:020000040800F2
:1080000098640020658100080DCB0008F1C10008CC
:1080100009CB0008A19B000845ED00080000000006
:1080200000000000000000000000000011D900085E
:10803000C1B400080000000075D10008E9DB0008A9
:10804000B9EE00087F8100087F8100087F81000869
:108050007F8100087F8100087F8100087F81000800
:108060007F8100087F8100087F8100087F810008F0
:108070007F8100087F8100087F8100087F810008E0
:108080007F8100087F8100087F810008299C00080B
:10809000A59B00087F810008C59B00087F81000820
:1080A0007F8100087F8100087F8100087F810008B0
:1080B0007F81000879DD00087F8100087F8100084A
:1080C0007F8100087F8100087F8100087F81000890
:1080D0007F810008E9E2000891E3000869E40008F4
:1080E0007F8100087F8100087F8100080000000078
:1080F0000000000000000000000000000000000080
:1081000000000000000000007F8100087F8100085F
:1081100009E1000801E200087F8100087F81000872
:108120007F8100087F8100087F8100087F8100082F
:108130007F8100087F8100087F810008919E0008F0
:108140007F810008FD9D0008219E00087F810008B6
:10815000DFF80CD000F048FC00480047451C01083F
:10816000986400200648804706480047FEE7FEE77F
:10817000FEE7FEE7FEE7FEE7FEE7FEE7FEE7FEE7D7
:10818000BDDC00085181000840EA01039B0703D0D1
:1081900009E008C9121F08C0042AFAD203E011F846
:1081A000013B00F8013B521EF9D27047D2B201E008
:1081B00000F8012B491EFBD270470022F6E710B5EC
:1081C00013460A4604461946FFF7F0FF204610BD45
:1081D00030B505462A460B4612F8010B13F8014B41
:1081E00008B1A042F8D01CB1002802D06D1CF1E704
:1081F000284630BD421C10F8011B0029FBD1801A13
:10820000704730B504460020034600E05B1C9342F3
:1082100003D2E05CCD5C401BF8D030BDF0B480EA06
:108220000102D40F4200B2EB410F02D202460846CF
:1082300011464A0042D0C30DDDB2C1F3C752AD1A98
:10824000202D35DAC1F3160141F4000204B1524287
:10825000C5F1200602FA06F12A411044B3EBD05FC3
:1082600023D0C4B1012DA0EBC35009DCF0BC4FF00A
:10827000004202EAC352DBB200F5000000F06ABA25
:10828000400000F1807000EBC350A0F1807040EA24
:10829000D170490009E0490841EAC071A0EBC35020
:1082A00000F50000400800EBC350F0BC00F049BAF4
:1082B0006142012202EB4101001BF6E7F0BC70476E
:1082C00081F00041AAE780F00040A7E780EA0102C0
:1082D00010B502F00043400022D04A001FD0010E2A
:1082E00001EB1261C0F35600C2F3560240F40000E5
:1082F00042F40002A0FB022000047F39140400D0E5
:10830000401C50EA124001D44000491EC2B20C0683
:1083100004EBD010401C4008802A02D003E000206B
:1083200010BD20F00100002900DA0020184310BD24
:1083300030B480EA010202F0004530F0004221F042
:10834000004013D090B1C30DD40DC2F31601C0F399
:108350001600E41A41F4000140F400027D34914219
:1083600001D3641C00E04900002C02DA30BC00207C
:1083700070474FF400000023914201D3891A034350
:1083800040084FEA4101F7D151B1914202D14FF07B
:10839000004105E002D24FF0010101E06FF0010160
:1083A00003EBC450284430BC00F0CBB92DE9FE4F9C
:1083B00081EA030404F0004421F0004100944FF0EE
:1083C000000B23F0004350EA01045ED052EA03049C
:1083D0005BD0C3F30A54C1F30A552C44A4F2F3341E
:1083E0000194A0FB0254C1F3130141F48011C3F3C3
:1083F000130343F4801301FB024400FB034E840A81
:10840000970A44EA815447EA8357A4FB0768029518
:108410008D0A05FB07854FEA932C04FB0C542705B6
:10842000029D4FEA065847EA1637B5EB08056EEB92
:10843000070C870E920E47EA811742EA8312A7FBC8
:108440000201B6EB0B0164EB00042B0D43EA0C3385
:108450005E1844EB1C50DA465146E7FB0201C5F3B7
:1084600013044FEA0B3343EA14534FEA0432019CDE
:1084700043EA0603A4F10C040294009CCDE900B485
:1084800000F0A5F903B0BDE8F08F00200146F9E740
:108490002DE9F04D81EA030404F0004B21F0004582
:1084A00014464FF0000A23F0004150EA050220D0A4
:1084B00054EA01021DD0C5F30A570246C5F313035F
:1084C000C1F31300C1F30A5640F4801543F480133E
:1084D000A7EB0608101BD64608F2FD3873EB050023
:1084E00002D308F1010801E092185B41B8F1000FD6
:1084F00003DA00200146BDE8F08D00204FF4801122
:10850000064684460EE0171B73EB050705D3121BC6
:1085100063EB050306434CEA010C49084FEA3000BF
:1085200092185B4150EA0107EDD152EA030012D0E4
:1085300082EA040083EA0501084305D0101BAB4121
:1085400006D20122002306E000224FF0004302E0A1
:108550006FF0010253101AEB06004CEB085110EBC0
:108560000A0041EB0B01BDE8F04D00F021B9C10F4D
:1085700080EAE0700844CA079623002100F0EAB8B8
:1085800096230022114600F0E5B80EB540F23341C3
:1085900002910021CDE900110A460B4600F017F9BF
:1085A00003B000BD20F00040C10DC0F3160040F440
:1085B00000007F2901DA00207047962903DCC1F111
:1085C0009601C840704796398840704700F00042D5
:1085D00030F000400AD0C10D01F56071C0F3160003
:1085E00042EA0151C208400711437047002001468A
:1085F0007047000030B5041E71F1000404DB4FF039
:108600000044404264EB0101141E73F1000405DBD9
:108610001C464FF00043524263EB04038B4208BFF9
:10862000824230BD30B5041E71F1000404DB4FF00E
:108630000044404264EB0101141E73F1000405DBA9
:108640001C464FF00043524263EB0403994208BFBB
:10865000904230BD01F0004330B421F0004150EAB7
:10866000010206D00A0DA2F56072C1F31301002ABF
:1086700002DC30BC00207047440F44EAC104C10052
:10868000E01830BC00EBC25000F05BB8002801DB02
:10869000C0F10040002901DBC1F100418142704777
:1086A000002801DBC0F10040002901DBC1F10041DD
:1086B0008842704730B50B46014600202022012435
:1086C00009E021FA02F59D4205D303FA02F5491BA0
:1086D00004FA02F52844151EA2F10102F1DC30BDB6
:1086E0002DE9F05F0546002092469B4688460646E7
:1086F000814640241BE0284641464746224600F07A
:1087000094F953465A46C01A914110D3114618465F
:10871000224600F07BF92D1A67EB01084F462246EE
:108720000120002100F072F917EB00094E41201ED4
:10873000A4F10104DFDC484631462A464346BDE841
:10874000F09F0029A8BF7047401C490008BF20F0D7
:108750000100704710B4B0FA80FC00FA0CF050EA47
:10876000010404BF10BC704749B1CCF1200421FAC8
:1087700004F411FA0CF118BF012121430843A3EBC3
:108780000C01CB1D4FEA00614FEA102042BF0020D0
:1087900010BC704700EBC35010440029A4BF10BCAC
:1087A0007047401C490008BF20F0010010BC704712
:1087B00010B5141E73F1000408DA401C41F10001E9
:1087C00092185B411A4301D120F0010010BD2DE940
:1087D000F04D92469B4611B1B1FA81F202E0B0FA37
:1087E00080F22032904600F011F904460F4640EA2C
:1087F0000A0041EA0B0153465A46084313D011467A
:1088000053EA010019D0C8F14002504600F00DF9BA
:1088100005460E4650465946424600F0F7F80843D2
:1088200005D0012004E020463946BDE8F08D002047
:10883000054346EAE0762C4337430A986305E40A89
:10884000A0EB08000022FD0A44EA47540A3002D592
:1088500000200146E9E7010510196941DDE90845F5
:1088600000196941BDE8F04DA2E72DE9FE4F8046B1
:1088700081EA0300C00F0C46009021F0004123F074
:108880000045B8EB0200A94105D24046214690467A
:108890001C460B46024623F00040104347D0270DEC
:1088A000C7F30A00C3F30A510290401A019040280E
:1088B0006BDAC3F3130040F4801B0098924620B19A
:1088C0000023D2EB030A63EB0B0B01985946C0F16E
:1088D0004002504600F09AF806460D46504659466A
:1088E000019A00F0B2F810EB08006141002487EA19
:1088F000115284EAE7731A4340D0009A62B3019A96
:10890000012A4FEA075215DC001B61EB02014FF010
:10891000004202EA0752CDE90042001C41F58011F5
:1089200032462B46FFF753FF03B0BDE8F08F4046B9
:108930002146F9E7001B61EB0201001C41F58013A1
:1089400000185B412018A2F5001747EB030140EA2D
:10895000D570B6196D4111E06D084FEA360645EA4B
:10896000C0754FEA0752001B61EB0201001C41F584
:10897000801149084FEA30000019514132462B4618
:1089800003B0BDE8F04FFFF713BF0098012240008D
:108990000023D0EB020263EBE073009821464FEA1C
:1089A000E074B8EB000061EB0401E9E783F00043F9
:1089B0005BE781F0004158E7C1F30A52C1F31301AC
:1089C00040F2FF3341F480119A4202DA002001465E
:1089D000704740F233439A42A2F2334202DC5242E1
:1089E00000F023B800F012B8064C074D06E0E0682E
:1089F00040F0010394E8070098471034AC42F6D3E6
:108A0000FFF7AAFB9C500108BC500108202A04DB98
:108A1000203A00FA02F1002070479140C2F1200391
:108A200020FA03F3194390407047202A04DB203AD0
:108A300021FA02F00021704721FA02F3D040C2F17E
:108A400020029140084319467047202A06DBCB17C5
:108A5000203A41FA02F043EAE07306E041FA02F3F9
:108A6000D040C2F12002914008431946704770B5CA
:108A70008C1810F8015B15F0070301D110F8013BC9
:108A80002A1106D110F8012B03E010F8016B01F850
:108A9000016B5B1EF9D12B0705D40023521E0DD4A8
:108AA00001F8013BFAE710F8013BCB1A921C03E0F6
:108AB00013F8015B01F8015B521EF9D5A142D8D32E
:108AC000002070BD10B503F0BDFE4FF4FA7002F047
:108AD000F8FC03F0CFFE10BD10B503F0BFFE4FF45D
:108AE000FA7002F0EEFC03F0C5FE10BD21B1826801
:108AF00042F00102826003E0826822F0010282609B
:108B0000704721B1826842F48072826003E082681B
:108B100022F4807282607047014600208A6802F069
:108B200004020AB1012000E0002070470146002045
:108B30008A6802F008020AB1012000E000207047B4
:108B400030B502460020002350680F4C20400D79BC
:108B50000C6844EA05242043506090680B4C204088
:108B6000D1E902542C434D7944EA450420439060F6
:108B7000D06A20F470000C7C641EE4B2234340EA07
:108B80000350D06230BD0000FFFEF0FFFDF7F1FFA3
:108B9000F0B504460D4600200021092D11DDE068E6
:108BA000A5F10A0606EB4607072606FA07F18843F1
:108BB000A5F10A0606EB460603FA06F10843E06053
:108BC0000CE0206905EB4507072606FA07F1884304
:108BD00005EB450603FA06F108432061072A0FDA80
:108BE000606B561E06EB86071F2606FA07F18843C0
:108BF000561E06EB860605FA06F10843606322E07E
:108C00000D2A0FDA206BD61F06EB86071F2606FA01
:108C100007F18843D61F06EB860605FA06F10843DE
:108C2000206310E0E06AA2F10D0606EB86071F261E
:108C300006FA07F18843A2F10D0606EB860605FA4F
:108C400006F10843E062F0BD816841F008018160EF
:108C5000704721B1826842F4A002826003E082681A
:108C600022F4A00282607047816841F004018160B3
:108C7000704700002DE9F05F7E490868FFF7A6FC09
:108C800004467D4A7D4BFFF7CDFC20D27948016830
:108C90007B48FFF71BFB83467A49FFF714FB8146AD
:108CA000744801687648FFF711FB82464946FFF792
:108CB0003FFB0446FFF78AFC0746734A734BFFF7F6
:108CC00075FB0546FFF7C6FC7149086049E0694934
:108CD0000868FFF77BFC04466E4A6F4BFFF7A2FC67
:108CE0002AD264490868FFF771FC0446624A634B64
:108CF000FFF780FC20D25F4801686148FFF7E6FA81
:108D000083466049FFF7DFFA81465A4801685C48AC
:108D1000FFF7DCFA82464946FFF70AFB0446FFF7F5
:108D200055FC07465D4A5E4BFFF740FB0546FFF7E3
:108D300091FC5749086014E04E4801685048FFF71D
:108D4000C5FA06464F49FFF7BEFA0446494801688E
:108D50004B48FFF7BBFA05462146FFF7E9FA4C49B5
:108D600008604B4800684F49086049480068FFF7B1
:108D70002DFC04464FF033324B4BFFF753FC11D21E
:108D800043480068FFF722FC04460022474BFFF7E8
:108D900031FC07D846484068401C454948600020DF
:108DA00088601AE03A480068FFF710FC0446414A20
:108DB000414BFFF71FFC10D835480068FFF706FC51
:108DC00004463E4A3E4BFFF72DFC06D838488068E3
:108DD000401C37498860002048602D480068FFF734
:108DE000F5FB0446334A344BFFF71CFC09D22848F4
:108DF0000068FFF7EBFB04460022324BFFF7FAFB5B
:108E000013D323480068FFF7E1FB0446294A2E4BA1
:108E1000FFF708FC09D31E480068FFF7D7FB04469C
:108E2000264A274BFFF7E6FB04D2002027490860BB
:108E3000BDE8F09F1E484068142803DC1C48806889
:108E4000142815DD1A484068142806DD002018494A
:108E5000486002201D490860EAE715488068142828
:108E600006DD002012498860012018490860DFE70C
:108E70000020DDE7CC0B0020AE47E17A14AE0240C3
:108E80000000E0400000A041B3B85A82E779EE3F0D
:108E900098000020105839B4C8760240A7E3D6499C
:108EA0002220EE3F640000203333114000001640C2
:108EB000A00B0020CDCCCCCCCCCC00409A99999979
:108EC0009999A93F00001040CCCC14409C00002090
:108ED000F8B505460E46002490208DF800000120CC
:108EE0008DF801008DF802608DF803500949086083
:108EF00003F094FA00BF08E01DF8040003F0C8FA7C
:108F00000A2000F029F8601CC4B2042CF4DB03F042
:108F1000A5FAF8BD9881214208B50121082004F086
:108F2000ADFAC020ADF8000003208DF8020010203B
:108F30008DF803006946054802F0ECFC0120044965
:108F400008600449C1F8980108BD0000000C014008
:108F50009C8121420080214200BF411E89B2081E2F
:108F6000FBD1704700B591B00121084604F056FAD4
:108F7000012140F2152004F081FA4FF4004004F082
:108F800041FA1F20ADF8400000208DF8430010A9E1
:108F9000424802F0BFFC0120ADF8400000208DF8EF
:108FA000430010A93E4802F0B5FC00200B900E9043
:108FB0004FF460200D9001208DF8310006208DF8CF
:108FC0003C0001208DF830000BA93648FFF7B8FDB2
:108FD000052301220A213348FFF7DAFD0523022287
:108FE0000B213048FFF7D4FD052303220C212D4827
:108FF000FFF7CEFD052304220D212A48FFF7C8FD07
:1090000005231A460E212748FFF7C2FD0523062235
:1090100000212448FFF7BCFD22484C300090801509
:10902000069000200490204801904FF48060079043
:1090300080200590002002900620039020200890B8
:1090400000200A904FF4805009906946174802F0BA
:10905000B9F90121154802F0A9F901211148FFF7DA
:1090600050FD01210F48FFF741FD0E48FFF7ECFDD1
:1090700000BF0C48FFF75AFD0028FAD10948FFF756
:10908000F3FD00BF0748FFF747FD0028FAD1012193
:109090000448FFF7DEFD11B000BD000000100140E4
:1090A0000008014000240140C00B002008000240DD
:1090B00070B502F0D5F80E4909780E4A52F8210031
:1090C00080470B4909780C4A52F821008047044632
:1090D0000748007800EB4000084901EBC00050F859
:1090E00024501DB12046A8470149087070BD0000FA
:1090F0005824002094070020B4070020D406002044
:10910000014601F00F000A0902EB820200EB420067
:10911000C0B2704710B5012004F0C0F9002004F07F
:10912000BDF910BD10B5A2B0002441F204000C49F5
:10913000A1F80500202048800A48007C401C09490D
:10914000087409A005F018FF01AA02A9044802F05A
:1091500057F90021094804F0CDFE22B010BD0000EF
:109160002A1E0020B01F002073656E6420436861D2
:1091700072676520646174610A0D0000F8050020C3
:1091800010B5114890F86600642804D1062002F05A
:1091900021FA002010BD0C4A906E926E91688847AB
:1091A00020B91C2002F016FA0020F3E7064A906E60
:1091B000926E1169884720B9212002F00BFA002035
:1091C000E8E70120E6E70000FC07002010B5A2B0A8
:1091D000002441F209000A49A1F805001220488044
:1091E0000848007C401C0749087407A005F0C4FE2D
:1091F00001AA02A9024802F003F922B010BD000042
:109200002A1E0020B01F002053656E642043686151
:109210007267696E6744617461200A0D0000000086
:1092200000B5A1B00020009041F203000E49A1F862
:1092300005000E4801780C48817204200A494880D4
:109240000B48007C401C0A4908740AA005F094FEF3
:109250006A4601A9044802F0D3F800210A4804F044
:1092600049FE21B000BD00002A1E0020700200202F
:10927000B01F002073656E64207374617465206490
:10928000617461200A0D0000F005002010B5242053
:1092900002F070F90021034804F02CFE002001F0D8
:1092A000D9FF10BD6824002010B5A2B0002441F2FF
:1092B00021001549A1F805001448007DC871134824
:1092C000808A010A1048017210484069010C0E485A
:1092D00041720E484069000E0B4988720420488094
:1092E0000B48007C401C0A4908740AA005F044FEA3
:1092F00001AA02A9044802F083F804210248C01D13
:1093000007F097FE22B010BD2A1E0020E4190020AD
:10931000B01F00200A0D7368656E676A6979696E0F
:10932000676461200A0D000010B5A2B000244FF45C
:1093300081500F49A1F805005520C871AA210C4899
:10934000017202200A4948800A48007C401C0949F1
:10935000087409A005F010FE01AA02A9044802F051
:109360004FF802210248C01D07F063FE22B010BD75
:109370002A1E0020B01F00204F54412041434B20A3
:109380000A0D000010B5A2B0002441F208001E49E9
:10939000A1F805001D481EA1096801601EA1096809
:1093A0004160194819490968C0F807101749496808
:1093B000C0F80B101548017A1348C173134800898F
:1093C000010A1148017411488068010C0E4841746B
:1093D0000E488068000E0C4988740C48017B0A48CE
:1093E000C1740D20084948800D48007C401C0C4980
:1093F00008740CA005F0C0FD01AA02A9024801F002
:10940000FFFF22B010BD00002A1E0020E221002034
:109410005332303100000000574C494E47000000E5
:10942000B01F002073656E6420626D7320766572D4
:1094300073696F6E0A0D0000F0B503460C46FF25F8
:10944000FF261512D6B209E013F8010B80EA0501D8
:109450000648405C80EA06050548465C201EA4F1EB
:109460000107BCB2F0D146EA0520F0BD384C010836
:10947000384D010870B502460C46FF25FF2309E070
:1094800012F8010B80EA05010648405C80EA0305FA
:109490000548435C201EA4F10106B4B2F0D143EAB2
:1094A000052070BD384C0108384D010810B5022167
:1094B00001A004F01CF910BD4154000010B50A21B0
:1094C00001A004F014F910BD41542B5354415445EC
:1094D0003D3F000070B504460E462546288845F6F7
:1094E000A521884202D1284608F0EAFD70BD00009F
:1094F00030B589B00446202101A8FEF75EFE202188
:1095000001A8FEF75AFE224606A101A805F044FD77
:1095100001A8FEF76FFE0546294601A804F0E7F80A
:1095200009B030BD41542B4E414D453D25730000DF
:1095300010B5092101A004F0DAF810BD41542B4EFA
:10954000414D453D3F00000010B50D2101A004F044
:10955000CEF810BD41542B554152545F4346473D10
:109560003F00000010B50B2101A004F0C0F810BDB1
:1095700041542B564552494F4E3D3F0010B52548AA
:109580000078012845D124480078062837D2DFE842
:1095900000F003170D36202A072220A12148FEF7EC
:1095A00030FE10B902201C49087028E00A221EA1D2
:1095B0001C48FEF726FE10B90120174908701EE06E
:1095C0001C491848FEF704FE10B104201249087027
:1095D00015E00B2218A11348FEF713FE10B9052061
:1095E0000D4908700BE00F480B494860154800888A
:1095F0000881144801880B48FFF76CFF00BF00BFCB
:109600000020044908700F49088080210548FEF7B2
:10961000D4FD10BD76020020B01F002041542B4F16
:109620004B0D0A00D41A002041542B4F4B0D0A3029
:10963000333033005415002041542B4F4B0D0A306A
:10964000310D0A007402002010B516480078072872
:1096500024D2DFE800F0040A07230D1F220000F0E7
:1096600077FA1CE000F078FA19E000F031FA16E021
:1096700000F05CFA0C4890F8760018B9002009490F
:10968000887006E0084890F87600012801D1054965
:10969000887004E000F00AF801E000E000BF00BFBD
:1096A00010BD0000B01F00204415002010B559481F
:1096B00090F8A800012808D15748007C0A2803DB4D
:1096C0000020544981F8A80010BD4FF47A70534926
:1096D00008805148007C14280EDD4E4890F8760032
:1096E00018B900204C49887006E04A4890F8760086
:1096F000012801D1484988704748807807287AD2E4
:10970000DFE800F004070E666782830000F0B0F91E
:109710007DE000F06DF900203E4981F8A80076E078
:109720003E4801883E4804F0E5FB01284FD13D4802
:109730000088401C3B49088008460088092801DD54
:10974000002008800021364804F0D4FB354800880A
:1097500010B900F021F93AE032480088012802D11E
:10976000FFF7E0FC33E02F480088022802D1FFF722
:1097700057FD2CE02B480088032828D02948008872
:10978000042802D100F050F821E02648008805287E
:1097900002D1FFF7F7FD1AE022480088062802D11F
:1097A000FFF714FD13E01F480088072802D106F0D8
:1097B000ADF90CE01B480088082802D106F040F9FA
:1097C00005E018480088092801D106F067F91EE075
:1097D0001DE01148417C407C401C0F4A5074142904
:1097E00011DD0020114608700A4890F8760018B97B
:1097F0000020887007E009E0064890F8760001280C
:1098000001D10549887002E001E000E000BF00BF1F
:1098100000BF59E744150020B01F0020DC050020E0
:10982000D8050020D405002010B5A2B0002001907A
:10983000002441F207004B49A1F805004A48808BFB
:109840004949C98B484342F2107190FBF1F084B250
:109850004548007F4349C8714348808B0112414805
:1098600001724148817F3F4841723F48C08B0112DD
:109870003C488172C4723C4890F829103948017301
:10988000394890F8281037484173202181735F21AF
:10989000C1733548C17E33480174334890F82610AF
:1098A000304841743048C08C01122E4881742E48D3
:1098B000C17E2C48C1742C48417A2A4801752A4837
:1098C000B0F809000112274841752748C17A254898
:1098D00081752548B0F80B0001122248C175224855
:1098E0004178204801762048B0F8010001121D4857
:1098F00041761D4841791B4881761B48B0F8050028
:1099000001121848C1761848C179164801771648DF
:10991000817C144841771448408A010A11488177B4
:10992000114890F82A100F48C1770F4890F82B1073
:109930000C4880F820100DA005F01EFB1A200949E4
:10994000488001AA02A9074801F05AFD0C48007C92
:10995000401C0B49087400210A4804F0CBFA22B0DD
:1099600010BD00002A1E0020240C002073656E64C8
:10997000204443444320646174610A0D00000000E8
:10998000B01F00201006002070B504460D46294681
:10999000204603F09FFE70BD00B5A1B000200090EE
:1099A0000AA005F0E9FA3A200E4948806A4601A962
:1099B0000C4801F025FD0C48007C401C0A49087445
:1099C00000210A4804F096FA21B000BD73656E6468
:1099D00020686561727462656174206461746120DD
:1099E0000A0D00002A1E0020B01F0020E8050020FC
:1099F00000B591B00020009040F6B831134804F053
:109A000079FA01281FD141F201001149A1F805009E
:109A100010A005F0B1FA0E48C01D1349CA6E0260CD
:109A2000096F416011490A6882604968C16010206D
:109A3000074948806A4601A9054801F0E1FC002178
:109A4000024804F057FA11B000BD0000E405002000
:109A50002A1E002073656E64204C6F67696E206457
:109A60006174610D0A00000044150020A84B010834
:109A700000B591B00020009041F288310C4804F00C
:109A800039FA012811D100030A49A1F80500002084
:109A9000488009A005F070FA6A4601A9054801F05E
:109AA000AFFC0021024804F025FA11B000BD00000F
:109AB000E00500202A1E002053656E642052656771
:109AC0006973746572656420646174610A0D0000D5
:109AD00010B54FF47A71124804F00CFA01281ED127
:109AE0001048007818B901200E49087013E00D489D
:109AF0000078012806D10C48FFF7FAFC022009493A
:109B0000087008E007480078022804D1FFF710FD2C
:109B10000020044908700021014804F0EBF910BD51
:109B2000CC050020C80500205415002010B540F6D3
:109B3000B831064804F0DEF9012805D1FFF7BEFC74
:109B40000021024804F0D6F910BD0000D005002025
:109B500010B5FFF7ABFC10BD10B54FF47A710E488D
:109B600004F0C8F9012815D10C48007828B9FFF78E
:109B7000F9FC01200949087008E00848007801282C
:109B800004D1FFF7E1FC00200449087000210248DD
:109B900004F0B0F910BD0000C4050020C30500208A
:109BA00000BFFEE700B585B06A460021044800F01A
:109BB00070FE6946002006F091FE05B000BD000071
:109BC0000064004010B54FF40071154800F01CFC13
:109BD00001280DD11349124800F0DAFB012802D107
:109BE000002006F059FF4FF400710D4800F0A4F971
:109BF0004FF480610A4800F007FC01280ED10949A2
:109C0000891C074800F0C4FB012802D1002006F09F
:109C100069FF4FF48061024800F08EF910BD00002A
:109C2000006400400200F01010B50021194800F057
:109C300057FF0446022C08D0012C00D100E0002080
:109C400002460021084606F085FE0121114800F079
:109C500047FF0446022C08D0012C00D100E0002070
:109C600002460121002006F075FE0221094800F09D
:109C700037FF0446022C08D0012C00D100E0002060
:109C800002460221002006F065FE0121014800F095
:109C900053F910BD0064004000B585B003F039FEF3
:109CA0000121092003F0EAFB0121480603F0C6FB6D
:109CB0000121880603F0C2FB0021494800F098FD0D
:109CC0004FF40050ADF8100003208DF8120018205A
:109CD0008DF8130004A9434801F01CFE4FF4805096
:109CE000ADF8100048208DF8130004A93D4801F09C
:109CF00011FE00208DF80A0001208DF80B000020D5
:109D00008DF80C008DF80D008DF80E008DF80F0009
:109D10008DF8060001208DF8070008208DF8080056
:109D200001208DF809000620ADF8040001A92C4897
:109D300000F003FC2C49002000F015FB012210214B
:109D4000274800F0F1FB41208DF8000001208DF83C
:109D5000010000208DF8020001208DF80300684604
:109D600002F0DCFE012211461D4800F0DDFB01225D
:109D700051021B4800F0D8FB01229102184800F064
:109D8000D3FB0122D103164800F0CEFB0121144879
:109D900000F02EFD3F208DF8000001208DF801001D
:109DA00000208DF8020001208DF80300684602F0C3
:109DB000B5FE42208DF8000001208DF80100002042
:109DC0008DF8020001208DF80300684602F0A6FE1F
:109DD00003F0A1FD05A005F0CFF8002005B000BDFF
:109DE00000680040000C01406406002063616E20A2
:109DF00032206F70656E210A0000000000B585B04A
:109E00006A460121054800F044FD9DF8090018B993
:109E10006946012006F062FD05B000BD0068004003
:109E200010B54FF40071184800F0EEFA012810D177
:109E30001649154800F0ACFA012805D106F02CFEB1
:109E40001249114800F05CF84FF400710E4800F020
:109E500073F84FF480610C4800F0D6FA012812D153
:109E60000A49891C084800F093FA012806D106F037
:109E700039FE0649891C044800F042F84FF480611D
:109E8000014800F059F810BD006800400200F010D1
:109E900010B50021194800F023FE0446022C08D01A
:109EA000012C00D100E0002002460021012006F034
:109EB00051FD0121114800F013FE0446022C08D088
:109EC000012C00D100E0002002460121084606F0E6
:109ED00041FD0221094800F003FE0446022C08D08F
:109EE000012C00D100E0002002460221012006F0F2
:109EF00031FD0121014800F01FF810BD006800404D
:109F000000220C4B994202D10023836111E0C1F37E
:109F1000130201F000730BB1C2600AE001F080632C
:109F20000BB1026105E001F000630BB1826000E05B
:109F3000426070477000F030B1F5007F3AD00FDC1E
:109F4000202928D006DC01291CD004291DD008298D
:109F500040D11DE0402921D0B1F5807F3AD126E0E3
:109F6000B1F5004F31D006DCB1F5806F25D0B1F5E9
:109F7000006F2FD124E0B1F5803F12D0B1F5003F42
:109F800028D111E0154A826025E00822C26022E053
:109F90001022C2601FE0082202611CE01022026150
:109FA00019E00822426016E01022426013E0042209
:109FB000426010E0042242600DE0042242600AE0A8
:109FC000002282610422426005E0002282610422B4
:109FD000426000E000BF00BF7047000001010100C7
:109FE00010B504460B48844209D10121480603F00C
:109FF00035FA00214FF0007003F030FA08E001213B
:10A00000880603F02BFA00214FF0806003F026FA57
:10A0100010BD0000006400402DE9F04104460D46EB
:10A0200017461E46ECB10020207220606060B5F536
:10A03000006F03D304202072656002E000202072CC
:10A04000256006B127B90020A0720220607208E0E6
:10A0500000206072A6723246394604F10B00FEF70A
:10A0600093F8BDE8F0812DE9F04104460D4617460E
:10A070001E46ECB10020207220606060B5F5006FD4
:10A0800003D304202072656002E000202072256066
:10A0900006B127B90020A0720220607208E00020FB
:10A0A0006072A6723246394604F10B00FEF76CF876
:10A0B000BDE8F08110B50021837A012202FA03F194
:10A0C0003D4A126842F001023B4B1A603A4A1C3288
:10A0D00012688A43384B1C331A60027BCAB9364A6D
:10A0E0000C3212688A43344B0C331A604288C3889E
:10A0F00042EA0343304A4032847A42F834300288DC
:10A10000838842EA03432C4A4032847A02EBC40239
:10A110005360027B012A19D1274A0C3212680A4384
:10A12000254B0C331A604288038842EA0343224AD3
:10A130004032847A42F83430C288838842EA03434A
:10A140001D4A4032847A02EBC4025360C27A3AB9A3
:10A15000194A121D12688A43174B1B1D1A6006E02C
:10A16000154A121D12680A43134B1B1D1A600289FF
:10A1700032B9114A143212688A430F4B14331A60F1
:10A180000289012A06D10C4A143212680A430A4B8A
:10A1900014331A60427B012A06D1074A1C32126826
:10A1A0000A43054B1C331A60034A126822F001026D
:10A1B000014B1A6010BD0000006600402DE9FF470A
:10A1C00006460F46B94600244FF00108404600F00D
:10A1D000D9FB8DF80A8001208DF80B008DF80C005A
:10A1E000ADF808008DF80D0000253EE0204604EB98
:10A1F000D0714910A4EB4101491C012902D0022968
:10A2000020D10FE056F83500042101EBC000000C0E
:10A21000ADF8000036F8350001EBC00080B2ADF8B3
:10A2200002000FE056F83500042101EBC000000CDD
:10A23000ADF8040036F8350001EBC00080B2ADF88F
:10A24000060000BF00BF641C204604EBD07149101B
:10A25000A4EB410141B96846FFF72CFF9DF80A00C5
:10A26000401CC0B28DF80A006D1C4D45BEDB204677
:10A2700004EBD0714910A4EB410111B16846FFF71E
:10A2800019FFBDE8FF872DE9FF4706460F46B9468F
:10A2900000244FF00108404600F074FB8DF80A805E
:10A2A00001208DF80B0000208DF80C000120ADF886
:10A2B00008008DF80D00002547E02046E11704EB6B
:10A2C00091718910A4EB8101491C012906D0022952
:10A2D0000DD0032914D0042924D11AE056F83500F2
:10A2E0004FF6FF7101EA4010ADF800001AE056F891
:10A2F00035004FF6FF7101EA4010ADF8020011E0A1
:10A3000056F835004FF6FF7101EA4010ADF8040031
:10A3100008E056F835004FF6FF7101EA4010ADF83D
:10A32000060000BF00BF641CE11704EB91718910A7
:10A33000A4EB810141B96846FFF7BCFE9DF80A0015
:10A34000401CC0B28DF80A006D1C4D45B5DBE1170D
:10A3500004EB91718910A4EB810111B16846FFF7FC
:10A36000A9FEBDE8FF8770B504460D460C2624B94A
:10A3700031462846FFF787FF08E0012C04D131461B
:10A380002846FFF71BFF01E0002070BD0120FCE71D
:10A3900010B50246002001F4700343B19369C1F384
:10A3A000130423400BB101202DE000202BE001F02D
:10A3B000807343B15368C1F3130423400BB10120F0
:10A3C00021E000201FE001F0006343B19368C1F376
:10A3D000130423400BB1012015E0002013E001F02D
:10A3E000007343B1D368C1F3130423400BB10120C0
:10A3F00009E0002007E01369C1F3130423400BB107
:10A40000012000E0002010BD70B504460D46002676
:10A4100060692840002871D0B5F5807F5CD010DCE1
:10A42000082D35D006DC012D20D0022D24D0042D9E
:10A4300072D127E0102D31D0202D35D0402D6BD199
:10A4400038E0B5F5004F60D009DCB5F5007F49D0A4
:10A45000B5F5806F4CD0B5F5006F5DD14FE0B5F527
:10A46000803F2DD0B5F5003F56D12FE0A0682D4993
:10A4700000F0E6FE064651E0E068032100F0E0FE51
:10A4800006464BE0E068082100F0DAFE064645E0AB
:10A49000E068102100F0D4FE06463FE02069032169
:10A4A00000F0CEFE064639E02069082100F0C8FE23
:10A4B000064633E02069102100F0C2FE06462DE07A
:10A4C0006068082100F0BCFE064627E060681021A5
:10A4D00000F0B6FE064621E0A069012100F0B0FEC2
:10A4E00006461BE0A069022100F0AAFE064615E020
:10A4F000A069042100F0A4FE06460FE00FE0A06969
:10A50000702100F09DFE064608E06068042100F01E
:10A5100097FE064602E0FFE7002600BF00E00026A7
:10A52000304670BD010101001AB143690B4343611C
:10A5300002E043698B434361704730B50246002017
:10A540000023146824F002041460146844F0010429
:10A55000146000E05B1C546804F001041CB94FF661
:10A56000FF74A342F6D1546804F001040CB9002032
:10A570006CE08C79012C04D1146844F080041460E0
:10A5800003E0146824F080041460CC79012C04D119
:10A59000146844F04004146003E0146824F040049C
:10A5A00014600C7A012C04D1146844F02004146067
:10A5B00003E0146824F0200414604C7A012C04D1C8
:10A5C000146844F01004146003E0146824F01004CC
:10A5D00014608C7A012C04D1146844F008041460CF
:10A5E00003E0146824F008041460CC7A012C04D130
:10A5F000146844F00404146003E0146824F00404B4
:10A6000014608C78A407CD7844EA05640D7944EA97
:10A6100005444D7944EA05540D886D1E2C43D461E0
:10A62000146824F001041460002300E05B1C5468EB
:10A6300004F001041CB14FF6FF74A342F6D1546834
:10A6400004F001040CB1002000E0012030BD2DE930
:10A65000F04107460C461546264616B1002128460D
:10A66000B047BDE8F08170B506460C461546E9B224
:10A67000E0B207F087F870BD00B589B00121052070
:10A6800002F0FCFE0121480602F0D8FE00215248EB
:10A6900000F0AEF84FF48050ADF8200003208DF8A4
:10A6A000220018208DF8230008A94C4801F032F947
:10A6B0004FF40060ADF8200048208DF8230008A971
:10A6C000464801F027F900208DF81A0001208DF886
:10A6D0001B0000208DF81C008DF81D008DF81E0059
:10A6E0008DF81F008DF816008DF817000C208DF8DE
:10A6F000180001208DF819000920ADF8140005A9F3
:10A700003548FFF71AFF00208DF80E008DF80F0076
:10A7100001208DF810000020ADF80400ADF806000F
:10A72000ADF80800ADF80A00ADF80C0001208DF876
:10A73000110001A8FFF7BEFC012202212648FFF705
:10A74000F3FE14208DF8000001208DF80100002098
:10A750008DF8020001208DF80300684602F0DEF952
:10A76000012211461C48FFF7DFFE012251021A4860
:10A77000FFF7DAFE012291021748FFF7D5FE01220A
:10A78000D1031548FFF7D0FE0121134800F030F83F
:10A7900013208DF8000001208DF8010000208DF8B5
:10A7A000020001208DF80300684602F0B7F9162078
:10A7B0008DF8000001208DF8010000208DF80200C6
:10A7C00001208DF80300684602F0A8F904A004F007
:10A7D000D3FB002009B000BD006400400008014028
:10A7E00063616E2031206F70656E210A00000000E9
:10A7F00010B502460B4600204FF6FF71BBB9146836
:10A8000024F0020444F00104146000E0491E54687E
:10A8100004F00304012C01D00029F7D1546804F09E
:10A820000304012C01D0002032E0012030E0012B94
:10A8300013D1146824F00304146000E0491E546826
:10A8400004F003040CB10029F8D1546804F00304A7
:10A850000CB100201CE001201AE0022B17D1146873
:10A8600024F0010444F00204146000E0491E54681E
:10A8700004F00304022C01D00029F7D1546804F03D
:10A880000304022C01D0002002E0012000E000209F
:10A8900010BD10B500F5D87303EB01131B6803F06E
:10A8A00004031372137A53B900F5D87303EB011341
:10A8B0001B6840F2FF7404EA5353136009E000F58B
:10A8C000D87303EB01131B686FF0604404EAD303F1
:10A8D000536000F5D87303EB01131B6803F0020308
:10A8E000537200F5D87303EB01135B6803F00F0399
:10A8F000937200F5D87303EB01135B681B0AD374E2
:10A9000000F5D87303EB01139B68D37200F5D8737D
:10A9100003EB01139B681C0A147300F5D87303EB57
:10A9200001139B681C0C547300F5D87303EB0113DF
:10A930009B681B0E937300F5D87303EB0113DB6860
:10A94000D37300F5D87303EB0113DB681C0A14748E
:10A9500000F5D87303EB0113DB681C0C547400F58D
:10A96000D87303EB0113DB681B0E937421B9C36822
:10A9700043F02003C36003E0036943F02003036155
:10A9800010BD00000B49096841F00101094A11603E
:10A990001146096843F60E729143064A116011464A
:10A9A000096841EA002111601146096821F001019E
:10A9B000116070470066004010B5024600209368A1
:10A9C00003F08063B3F1806F00D110E0936803F06F
:10A9D0000063B3F1006F01D1012008E0936803F038
:10A9E0008053B3F1805F01D1022000E004200428ED
:10A9F00074D002F5C07303EB00131B6803F001046D
:10AA000002F5C07303EB00131C600B7A7BB94B7A21
:10AA10000C8843EA445302F5C07404EB0014246824
:10AA2000234302F5C07404EB0014236010E00B7A9A
:10AA30004C6843EAC4034C7A234302F5C07404EB28
:10AA400000142468234302F5C07404EB001423604F
:10AA50008B7A03F00F038B7202F5C07303EB0013C4
:10AA60005B6823F00F0402F5C07303EB00135C6016
:10AA700002F5C07303EB00135B688C7A234302F585
:10AA8000C07404EB001463608B7B1C064B7B44EAB0
:10AA900003440B7B44EA0323CC7A234302F5C074BE
:10AAA00004EB0014A3608B7C1C064B7C44EA03443B
:10AAB0000B7C44EA0323CC7B234302F5C07404EBF4
:10AAC0000014E36002F5C07303EB00131B6843F04E
:10AAD000010402F5C07303EB00131C6010BD0000FD
:10AAE00010B50246002321B1012907D002290FD158
:10AAF00009E090681D4C00EA04030BE090681C4CD0
:10AB000000EA040306E090681A4C00EA040301E03E
:10AB1000002300BF00BF184C181BA34216D007DC4F
:10AB200083B16FF08060184470B1022818D111E031
:10AB3000B0F5007F10D0114C204448B1B0F5003F73
:10AB40000ED10BE002230DE000230BE0002309E00F
:10AB5000002307E0012305E0012303E0012301E0D6
:10AB6000002300BF00BFD8B210BD000003000004E6
:10AB70000003000800000310000100080001FFF7B7
:10AB800010B5012002494870024801F0EDFE10BDE9
:10AB9000D4070020C40A002010B5002002494870E4
:10ABA000024801F00CFF10BDD4070020C40A0020A9
:10ABB00070B51F48058904891E48006808B31E48FF
:10ABC00000683C21B0FBF1F01B49086008460068B2
:10ABD000C0001A49086008460068FDF7D1FC064627
:10ABE0001749FDF7A5FB17490860FEF743F816491A
:10ABF000087000200F4908600F4908600F4908607D
:10AC000014E0124800683C280AD20B48006820442F
:10AC1000094908600D480068401C0C49086005E0BF
:10AC200000200A49086001200249086070BD000048
:10AC3000C00B002090000020880000208C00002025
:10AC400000401C46CC0B0020600000209400002037
:10AC500030B503460C46002118785D7800EB0520DE
:10AC6000184DA5F81B009878DD7800EB052001B29F
:10AC7000B1F57A6F02DDA1F57A6001E0C1F57A6085
:10AC800001B2104DA5F81D100A2906DB2846B0F8C0
:10AC90001D000D4DA5F8070003E000200A4DA5F8A2
:10ACA000070018795D7900EB0520064DA5F81F0017
:10ACB0002846B0F81F00A5F81F00987985F82100F4
:10ACC000012030BD6C0C0020E60C002010B50346BE
:10ACD0001C78074880F827405C7880F828409C78EA
:10ACE00080F82940DC7880F82A40012010BD00005F
:10ACF0006C0C002070B505460C461646032C00DD92
:10AD00000324224629460248FDF73EFA012070BD81
:10AD10006C0C002030B503460C46002118785D7895
:10AD200040EA0520144D68829878DD7840EA0520D5
:10AD3000114DA88218795D7940EA052001B2B1F57C
:10AD40007A6F02DDA1F57A6001E0C1F57A6001B2A7
:10AD5000094DE9829879DD7940EA052001B2B1F523
:10AD60007A6F02DDA1F57A6001E0C1F57A6001B287
:10AD7000014D2983012030BD6C0C002010B5034625
:10AD8000082900DD082118780A4CE07058782071F5
:10AD90009C7808484471DC7884711C79C4715879B6
:10ADA000044C20729C7903484472DC79847201203F
:10ADB00010BD00006C0C002010B503461878024C42
:10ADC000A076012010BD00006C0C002010B50346D9
:10ADD0001879074C84F834005C79054880F83540D0
:10ADE0009C7980F83640DC7980F83740012010BD2E
:10ADF0006C0C002010B503461C78074880F82340EF
:10AE00005C7880F824409C7880F82540DC7880F8D5
:10AE10002640012010BD00006C0C002030B5034618
:10AE20000C461546082C00DD08241878FEF768F952
:10AE30001449C8725878FEF763F912490873987874
:10AE4000FEF75EF90F494873D878FEF759F90D49B6
:10AE500088731879FEF754F90A49C8735879FEF7D0
:10AE60004FF9084908749879FEF74AF9054948747A
:10AE700005480B310A6802608A888280897981716D
:10AE8000012030BD6C0C0020610C002010B5044680
:10AE900006A004F071F800F079FAFDF71DFE00F04D
:10AEA0006FF9FFF76DFE012010BD000054310D0A4F
:10AEB0000000000010B5044602A004F05DF8022076
:10AEC00010BD00005431300D0A00000010B50446DA
:10AED00002A004F051F8062010BD00005431310DDD
:10AEE0000A00000010B5044602A004F045F8062050
:10AEF00010BD00005431320D0A00000010B50446A8
:10AF000002A004F039F8012010BD00005431330DC7
:10AF10000A00000010B5044602A004F02DF800203D
:10AF200010BD00005431340D0A00000010B5044675
:10AF300004A004F021F8FFF72FFE044801F03FFDC4
:10AF4000072010BD5431350D0A000000880A00208A
:10AF500010B5044603A004F00FF8FFF711FE00201F
:10AF600010BD00005431360D0A00000010B5044633
:10AF700005A004F001F802F0E9FB0549486000F083
:10AF80000BF9022010BD000054320D0A0000000031
:10AF90000424002010B5044604A003F0EDFF02F0E5
:10AFA000D5FB04498860032010BD000054330D0A0E
:10AFB000000000000424002010B5044606A003F0A1
:10AFC000DBFFFDF77FFD00F0E9F902F0BFFB04496C
:10AFD000C860042010BD000054340D0A00000000B9
:10AFE0000424002010B5044602A003F0C5FF05208C
:10AFF00010BD000054350D0A0000000010B50446D5
:10B0000002A003F0B9FF062010BD000054360D0A5F
:10B010000000000010B5044605A003F0ADFF00F0ED
:10B02000AFF800F0B3F9FDF757FD002010BD0000A8
:10B0300054370D0A0000000010B5044602A003F0CA
:10B040009BFF022010BD000054380D0A00000000D4
:10B0500010B5044602A003F08FFF022010BD0000CF
:10B0600054390D0A0000000010B5252000F082FAC6
:10B070000021034802F03EFF012000F0EBF810BD74
:10B080006C24002010B52248406A00F0004018B13E
:10B0900020A003F071FF34E01D48406A00F08040BA
:10B0A00018B120A003F068FF2BE01948406A00F0B7
:10B0B000005018B120A003F05FFF22E01448406A5E
:10B0C00000F0805018B121A003F056FF19E010489D
:10B0D000406A00F0006018B11FA003F04DFF10E0BF
:10B0E0000B48406A00F0806018B11FA003F044FFD5
:10B0F00007E00748406A00F0007010B11DA003F09F
:10B100003BFF0348406A40F080700149486210BD2F
:10B1100000100240B5CDB9A6BAC4B8B4CEBB0D0A72
:10B1200000000000B4B0BFDABFB4C3C5B9B7B8B44B
:10B13000CEBB0D0A00000000B6C0C1A2BFB4C3C59B
:10B14000B9B7B8B4CEBB0D0A00000000C8EDBCFE14
:10B15000B8B4CEBB0D0A0000C9CFB5E72FB5F4B522
:10B16000E7B8B4CEBB0D0A00D2FDBDC5B8B4CEBBA6
:10B170000D0A0000424F52B8B4CEBB0D0A000000C9
:10B1800010B5012002490870024801F0EDFB10BD26
:10B19000D4070020600A002010B500200249087082
:10B1A000024801F00CFC10BDD4070020600A00200A
:10B1B00006480078052801D101207047034800782F
:10B1C000062801D10220F8E70020F6E758240020E5
:10B1D00010B51848007920B1012807D002280DD1F8
:10B1E00008E01121144800F023FB07E0124800F0AA
:10B1F00051FB03E0112000F05DFB00BF00BF3221D6
:10B200000E4802F077FE012805D104F0F3FD00217D
:10B210000A4802F06FFEFA210848083002F06AFE80
:10B22000012806D105F054F900210448083002F045
:10B2300061FE10BDF423002099FF00083C2400208B
:10B240000246002002EA01030BB1012000E00020C9
:10B2500070470000012201490A5470477024002001
:10B260000120704710B5044908698047022801D1C0
:10B27000012010BD0020FCE76400002010B51F492C
:10B28000C86880471E490988884204DD012000F013
:10B29000A1F9002010BD1949C868804740F6B831AF
:10B2A00088420ADA1549C8688047B0F5FA6F04DDAC
:10B2B000022000F08FF90020ECE71248B0F81D00E2
:10B2C000B0F5167F04DD052000F084F90020E1E7E9
:10B2D0000B48B0F8410020B9092000F07BF90020AC
:10B2E000D8E70748B0F84300322804DA0A2000F013
:10B2F00071F90020CEE70120CCE7000064000020B7
:10B30000FC0700206C0C002010B500240C480078CD
:10B3100000B913E00A480078012801D101240DE0AA
:10B3200007480078052803D005480078072801D190
:10B33000022403E000F00EF900B10324204610BD02
:10B340005824002010B541F288310F4802F0D2FD98
:10B35000012807D1252000F03DF9012002F0AAFBC9
:10B36000002010BD41F288310748001F02F0C2FDE5
:10B37000012807D1242000F02DF9002002F09AFBCB
:10B380000020EEE70120ECE76C24002010B5024815
:10B3900001F0EAFA10BD0000FC09002010B50248D7
:10B3A00001F00DFB10BD0000FC09002021B1026876
:10B3B00042F00102026004E002684FF6FE731A4098
:10B3C0000260704710B50022026847F6F0739A4396
:10B3D0000C6A8B6823430C6923434C6923438C69B3
:10B3E0002343CC6923434C6A23438C6A23431A4387
:10B3F0000260CB6843600B6883604B68C36010BD1C
:10B400002DE9F04706460C4692460025A946A84677
:10B4100006B114B90020BDE8F087708819301FFA12
:10B4200080F8A5222846691CCDB222545A2228460B
:10B43000691CCDB222542846691CCDB204F80080A4
:10B440004FEA18222846691CCDB2225420222846F1
:10B45000691CCDB22254601910221849FCF794FEE1
:10B4600005F11000C5B272792846691CCDB222548C
:10B47000B6F80500020A2846691CCDB2225470882D
:10B48000022807DB72886019F11DFCF77DFEB07899
:10B490002844C5B229462046FDF7ECFF074628465A
:10B4A000691CCDB227543A0A2846691CCDB22254F1
:10B4B00029462046FEF768FA0120ACE74415002033
:10B4C000704710B5044606E0142003F00BFD01F0B0
:10B4D00017F8601E84B2002CF6DC10BD10B51021E8
:10B4E0000648FCF76AFE0648002101600171002051
:10B4F000044908600449086010BD0000742400205D
:10B50000C0080020B8080020BC08002010B510E0DA
:10B510000A480B4A1268815C0AA003F02DFD084816
:10B520000068401C052190FBF1F201FB1200044968
:10B53000086006F027FB0028EAD010BDC0080020F4
:10B54000B8080020457272204E554D2069732025A1
:10B55000640D0A00002106E00548405C08B10120A6
:10B560007047481CC1B21029F6DB0020F8E7000044
:10B570007424002070B50546284600F0DFFA044622
:10B58000284600F0D1FA06460448005D0021B1408B
:10B59000084302490855012070BD000074240020B2
:10B5A0002DE9F0410446204600F0C8FA0546204641
:10B5B00000F0BAFA06460648405D0121B14000EAB3
:10B5C000010717B10120BDE8F0810020FBE7000072
:10B5D0007424002070B506463046FFF7E1FF10B92D
:10B5E000304604F05BF9304600F0A8FA04463046D5
:10B5F00000F09AFA05460448005D0121A94008437D
:10B6000001490855012070BD742400200149C8601B
:10B61000704700000020024030B5044604250F4862
:10B6200000F0AAF80546042D16D10D48006940F037
:10B6300002000B49086108464461006940F040007F
:10B640000861064800F098F805460548006941F68B
:10B65000FD71084002490861284630BDFFFF0F0018
:10B660000020024004200B49C96801F0010109B122
:10B6700001200EE00749C96801F0040109B1022068
:10B6800007E00449C96801F0100109B1032000E096
:10B6900004207047002002400348006940F0800009
:10B6A00001490861704700000020024070B504465F
:10B6B0000D4604264FF6FF7000F05EF80646042E95
:10B6C00012D10A48006940F001000849086125804C
:10B6D0004FF6FF7000F050F806460448006941F646
:10B6E000FE71084001490861304670BD00200240EB
:10B6F00078B506460C460425002000904FF6FF70F2
:10B7000000F03AF80546042D26D11448006940F0AF
:10B7100001001249086134804FF6FF7000F02CF8E8
:10B720000546042D11D1B01C0090200C0099088012
:10B730004FF6FF7000F020F805460848006941F612
:10B74000FE7108400549086106E00448006941F6B9
:10B75000FE71084001490861284678BD002002407A
:10B760000248034948600348486070472301674521
:10B7700000200240AB89EFCD00B502460423FFF75D
:10B7800071FF034603E0FFF76DFF0346521E012BD6
:10B7900001D1002AF7D102B90523184600BD0000E7
:10B7A0002DE9F041074620480088401E86B200255A
:10B7B00000241E4800EBC60041683846FCF766FFCF
:10B7C00007D31A4800EBC50041683846FCF768FF0C
:10B7D00003D240F6FF70BDE8F0811EE0A81900EB2F
:10B7E000D071C1F34F04114800EBC40041683846E2
:10B7F000FCF756FF02D2601E86B20EE00B4800EB4B
:10B80000C40041683846FCF741FF02D2601C85B293
:10B8100003E0064830F93400DDE7B542DEDD0348D9
:10B8200030F93500D7E700006200002038460108F3
:10B8300070B504460D466421124802F05BFB0128F6
:10B8400008D1A04700201049C872486000210D4867
:10B8500002F050FB0C48C07A112811D10A48407CF4
:10B86000A8420DD1084840686FF30F00074988428D
:10B8700006D100200449C8724860012004490871BB
:10B8800070BD00002C240020FC0C00200000EC1CEB
:10B89000F423002010B504460220A04702200349EB
:10B8A00008710021024802F025FB10BDF42300209E
:10B8B0003024002010B504461148C07A132812D154
:10B8C0000F48407CA0420ED10D4840686FF30F0036
:10B8D0000C49884207D100200949C87248600A49CA
:10B8E00008710A4988633221094802F003FB0128E4
:10B8F00004D10020044908710449886310BD000088
:10B90000FC0C00200000EC1CF42300206C0C002038
:10B91000302400202DE9F0410246002500260020B9
:10B9200000230024002791F803C00CF00F0591F8C4
:10B9300003C00CF0100CBCF1000F03D091F802C052
:10B940004CEA050591F800C0BCF1000F31D0146835
:10B9500000202BE04FF0010C0CFA00F3B1F800C00E
:10B960000CEA03069E4220D183004FF00F0C0CFA24
:10B9700003F7BC4305FA03FC4CEA040491F803C046
:10B98000BCF1280F06D14FF0010C0CFA00FCC2F8F4
:10B9900014C00AE091F803C0BCF1480F05D14FF084
:10B9A000010C0CFA00FCC2F810C0401C0828D1D3CE
:10B9B0001460B1F800C0BCF1FF0F34DD5468002002
:10B9C0002EE000F1080C4FF0010808FA0CF3B1F872
:10B9D00000C00CEA03069E4221D183004FF00F0CF9
:10B9E0000CFA03F7BC4305FA03FC4CEA040491F893
:10B9F00003C0BCF1280F05D100F1080C08FA0CF8BF
:10BA0000C2F8148091F803C0BCF1480F07D100F1CF
:10BA1000080C4FF0010808FA0CF8C2F81080401C1E
:10BA20000828CED35460BDE8F0810000F0B50A4686
:10BA3000002300240021002500F00046B6F1004F4D
:10BA400002D11D4EF16901E01B4E7168C0F3034540
:10BA500083B200F44016B6F5401F08D121F07061A2
:10BA6000154E766826F07066134F7E6012E000F483
:10BA70008016B6F5801F06D1032606FA05F4A14309
:10BA800041F0706106E0460D360103FA06F6B14357
:10BA900041F0706122B1460D360103FA06F63143DA
:10BAA00000F00046B6F1004F02D1034EF16101E013
:10BAB000014E7160F0BD0000000001400246002010
:10BAC00093680B400BB1012000E0002070474161FA
:10BAD00070470161704700002DE9F0470D48C488A8
:10BAE0000D4A0321204603F063F90B480068FCF778
:10BAF0006DFD07463A460B4608480949FCF7C8FC65
:10BB00000546FCF7A7FD8146FFF74AFE0549487246
:10BB1000BDE8F087C00B0020AC0000209A999999ED
:10BB200099991340CC0B002001460A46C81701EB37
:10BB30005070C010A1EBC000C0B2704701460A4669
:10BB4000C81701EB5070C0F3C700704702460021D0
:10BB500012E001EB410000EBC1000E4B03EB0010C3
:10BB60000078904206D101EB410000EBC10003EBED
:10BB700000107047481CC1B2022909D201EB4100F4
:10BB800000EBC100034B03EB00100078FF28E0D16D
:10BB90000020EEE7601300202DE9F0478246BAF15D
:10BBA000010F34D1EB21822006F00EF864490880A1
:10BBB00008460088B0F5004F0CDB08460088B0F559
:10BBC000803F07DA084600884FF6FF71081A5C4983
:10BBD000088008E05A4800884FF6FF71884202DB6F
:10BBE00000205749088056480088FCF7CEFC804664
:10BBF000544A554BFCF7DAFB06460022534BFCF740
:10BC000047FC0446FCF726FD5149086094E0BAF170
:10BC1000020F59D1E321B22005F0D6FF4849088030
:10BC200008460088B0F5004F0ADB0120494908802A
:10BC3000434800884FF6FF71081A4149088002E026
:10BC40000020444908803E480088FCF79EFC80465E
:10BC50003C4A3D4BFCF7AAFB064600223B4BFCF757
:10BC600017FC0446FCF7F6FC3949086008460068F2
:10BC7000FCF7ACFC06464FF03332374BFCF796FB33
:10BC80000446364A364BFCF703FC8046FCF7E2FCE0
:10BC90002F4908602F48008801284DD14FF4FA61E0
:10BCA000304802F027F9012806D12FA003F064F9EB
:10BCB00000212C4802F01EF9254801680020FCF7FD
:10BCC000FFFA2349086037E0BAF1030F34D1E321CA
:10BCD000B42005F079FF1A49088008460088B0F5BD
:10BCE000004F0CDB08460088B0F5803F07DA0846B5
:10BCF00000884FF6FF71081A1149088008E01048C3
:10BD000000884FF6FF71884202DB00200C49088052
:10BD10000B480088FCF739FC06460A4A1B4BFCF727
:10BD200045FB04460022094BFCF7B2FB8046FCF7BA
:10BD300091FC0749086000BF05480068BDE8F0872E
:10BD4000BE000020FCA9F1D24D622040E0FFEF4090
:10BD5000C0000020C4000020F308CA40F6285C8F11
:10BD6000C2F51340D80000204E656761746976659E
:10BD700020766F6C746167652073616D706C6520EF
:10BD80006661756C74210D0A000000004D62104060
:10BD90000146087870470146C878032801D1012080
:10BDA0007047C878042801D10020F9E70020F7E7A0
:10BDB00001468878012800D17047887808B90020AA
:10BDC000FAE70020F8E700000148407A70470000D9
:10BDD000CC0B002010B5054948680549FCF776FAF8
:10BDE0000446FCF7DFFB80B210BD0000CC0B002046
:10BDF000000020412DE9F041044661492046FCF74E
:10BE00004FFC04D200205F490870BDE8F0815D4816
:10BE1000007830B1012830D002284CD0032874D1EA
:10BE200078E059492046FCF731FC01D2012700E0B7
:10BE300000272046FCF7CAFB0546544A544BFCF742
:10BE4000F1FB01D2012000E0002007401FB10120DA
:10BE50004C49087010E04F492046FCF721FC08D2FD
:10BE60004D492046FCF712FC03D2022045490870D8
:10BE700002E00020434908707EE043492046FCF779
:10BE800005FC01D2012700E000272046FCF79EFBBD
:10BE900005463E4A3E4BFCF7C5FB01D2012000E0BF
:10BEA000002007401FB101203649087002E0002041
:10BEB0003449087060E04FF07F512046FCF7E6FB04
:10BEC00001D2012700E000272046FCF77FFB054652
:10BED0002E4A2F4BFCF7A6FB01D2012000E00020E8
:10BEE00007401FB103202749087012E04FF081413D
:10BEF0002046FCF7D5FB09D227492046FCF7C6FBB4
:10BF000004D202201F49087003E031E000201D49DF
:10BF1000087031E04FF07F512046FCF7B7FB01D2AB
:10BF2000012700E000272046FCF750FB0546174A92
:10BF3000174BFCF777FB01D2012000E000200740FF
:10BF40001FB103200F49087011E04FF081412046D6
:10BF5000FCF7A6FB08D210492046FCF797FB03D25A
:10BF600002200849087002E000200649087003E03A
:10BF700000200449087000BF00BF0248007844E771
:10BF800000002041940B0020000040407B14AE478D
:10BF9000E17A843F333353400000E0402DE9F84F0D
:10BFA0003F48D0F800A001460868FCF70FFB0446A4
:10BFB0003C4A3D4BFCF736FB20D2394801683B48F0
:10BFC000FCF784F93A490090FCF77DF98146344842
:10BFD00001683648FCF77AF983464946FCF7A8F928
:10BFE0000446FCF7F3FA0746324A334BFCF7DEF916
:10BFF0000546FCF72FFB3149086049E028490868ED
:10C00000FCF7E4FA04462E4A2E4BFCF70BFB2AD22F
:10C0100023490868FCF7DAFA0446224A224BFCF767
:10C02000E9FA20D21E4801682048FCF74FF9834600
:10C030001F49FCF748F98146194801681B48FCF77D
:10C0400045F949460090FCF773F98046FCF7BEFAC3
:10C0500006461D4A1D4BFCF7A9F90446FCF7FAFAFF
:10C060001649086014E00E4801681048FCF72EF9E4
:10C0700006460F49FCF727F90446094801680B48B2
:10C08000FCF724F905462146FCF752F90B490860F4
:10C090000A4800680E49086008480068BDE8F88F43
:10C0A000CC0B0020AE47E17A14AE02400000E04025
:10C0B0000000A041B3B85A82E779EE3F9800002013
:10C0C000105839B4C8760240A7E3D6492220EE3F83
:10C0D000640000200148007A70470000CC0B00206B
:10C0E00001464878012800D17047487808B90020F7
:10C0F000FAE70020F8E7000070B5FFF74FFF0646AB
:10C10000FFF778FE04460025012C01D1012506E049
:10C11000022C01D0032C01D1022500E00025124899
:10C120000078854205D00020104908700E4805703F
:10C1300017E00F480078854203D100200B490870B2
:10C140000FE00A480078401C08490870084600784B
:10C150001E2806DB044800780549087000200349C2
:10C1600008700348007870BDB5000020B4000020BE
:10C17000B6000020014601F00F01092903DD01F19D
:10C180003700C0B2704701F13000C0B2FAE7014693
:10C190000911092903DD01F13700C0B2704701F12F
:10C1A0003000C0B2FAE700002DE9F0410B484488A6
:10C1B0000B4A0121204602F0FBFD09480068FCF70C
:10C1C00005FA0546074A084BFCF762F90746FCF7F3
:10C1D00041FA06494860BDE8F0810000C00B00202C
:10C1E000A80000201361C3D32B65693FCC0B00204E
:10C1F00000BFFEE770B50446002500BF0025912072
:10C20000005D06281ED2DFE800F0031E4C4D5C7076
:10C2100094F85400032815DB04F1700008F006F8C8
:10C2200080B904F1940104F1700008F01FF840B1E6
:10C23000012191200155002084F890000021AC20BC
:10C240000155012567E094F899309422115920781E
:10C2500004F19A02A668B04784F8980094F8900018
:10C26000401C84F8900094F89800FF280ED002211A
:10C27000912001550021AC200155012594F854006E
:10C2800081280DD1032084F8540009E094F890101F
:10C2900094F84400814203DB0421912001550125DB
:10C2A00039E038E094F8901094F84400814203DBC0
:10C2B00004219120015502E0012191200155012521
:10C2C00029E0002191200155D4F8A80020B10121D6
:10C2D000D4E92902904706E0206D20B10121226DAA
:10C2E000D4F8A4009047012515E0002191200155C4
:10C2F000D4F8A80028B10220D4E9292104F0B6FC22
:10C3000007E0206D28B10220D4F8A420216D04F0AC
:10C31000ADFC012500BF00BF012D04D19120005DBF
:10C3200004287FF46BAF25B122780421012004F0AA
:10C330009DFC70BD10B504469120005D022811D10E
:10C3400094F8901094F84400814203DB042191207A
:10C35000015502E00321912001552278042101209A
:10C3600004F084FC10BD70B504460D469120005DBC
:10C37000022803D09120005D03280DD194F8980085
:10C38000A84209D105219120015594F854000328B1
:10C3900002DB2046FFF72EFF70BD000070B50024C1
:10C3A000002515E001201B4908600520FCF7D4FD9D
:10C3B0006006040E1848D0F81C0108B144F00104CE
:10C3C0000020144908600520FCF7C6FD681CC5B2B2
:10C3D000082DE7DB00200F4908600520FCF7BCFDB5
:10C3E00000200D49C1F89C010520FCF7B5FD012096
:10C3F000084908600520FCF7AFFD00200649C1F898
:10C4000098010520FCF7A8FD01200249091D0860DC
:10C41000204670BD988121420080214210B5012044
:10C420000C4908600520FCF797FD01200A49C1F876
:10C4300098010520FCF790FD0020064908600520C2
:10C44000FCF78AFD00200449C1F898010520FCF79B
:10C4500083FD10BD9C8121420080214210B5002047
:10C46000094908600520FCF777FD01200749C1F85C
:10C4700098010520FCF770FD0120034908600520A4
:10C48000FCF76AFD10BD00009C8121420080214222
:10C4900070B5044600201849086000251CE004F02F
:10C4A000800020B101201449091D086003E000202C
:10C4B0001149091D086001200F4908600520FCF79B
:10C4C0004BFD00200D49C1F898010520FCF744FD03
:10C4D0006006040E681CC5B2082DE0DB0120064989
:10C4E000091D08600549C1F898010520FCF734FDD5
:10C4F00000200149086070BD9881214200802142DE
:10C500007F2003490860002002490870704700003E
:10C51000002C00404D02002010B5002414E004EB74
:10C52000440101EBC4010F4A02EB0110B021FBF7FB
:10C5300044FEFF2004EB440101EBC401094A02EB75
:10C5400001110870601CC4B2022CE8D301F008FB92
:10C550000549012004F0A4FB0449022004F0A0FBDB
:10C5600010BD00006013002067A600084FA6000859
:10C5700010B548210E48FBF720FE28210D48FBF797
:10C580001CFE0D4801F074F9044624B11422214622
:10C590000848FBF7F9FD0848203001F069F9044626
:10C5A0002CB11422214603481430FBF7EDFD10BDD9
:10C5B000900F0020680F0020684B010810B521483B
:10C5C00000F064F9204800F061F9204800F05EF9BD
:10C5D0001F4800F05BF91F4800F058F91E4800F0B2
:10C5E00055F91E4800F052F91D4800F04FF91D485A
:10C5F00000F04CF91C4800F049F91C4800F046F9DD
:10C600001B4800F043F91B4800F040F91A4800F0BD
:10C610003DF91A4800F03AF9194800F037F919487D
:10C6200000F034F9184800F031F9184800F02EF9FC
:10C63000174800F02BF9174800F028F9164800F0C9
:10C6400025F910BDE8090020FC090020100A00208F
:10C65000240A0020380A00204C0A0020600A00202A
:10C66000740A0020880A00209C0A0020B00A0020DA
:10C67000C40A0020D80A0020EC0A0020000B002089
:10C68000140B0020280B00203C0B0020500B002036
:10C69000640B0020780B00208C0B00202DE9F0416A
:10C6A00080460D46164600244046FFF74FFA0446E2
:10C6B0000CB105B116B90020BDE8F081287818B199
:10C6C00094F85400012801D00020F5E795F82000E7
:10C6D00000F0010018B1A86A08B90020ECE795F84D
:10C6E000251084F8451094F8450010B9322184F8DB
:10C6F000451094F8451001EB4101C80005F04AFBD4
:10C70000C4F88C00D4F88C0048B194F84530182255
:10C7100004F17000D4F88C1007F09AFD01E00020BD
:10C72000CAE795F8200000F00100D8B994F8451048
:10C73000080105F02FFBC4F88800D4F8880048B140
:10C7400094F84530102204F15800D4F8881007F00E
:10C750007FFD07E0D4F88C0004F0E4FC0020C4F86E
:10C760008C00A9E7296A216404F1200720213846BA
:10C77000FBF723FD1F2229463846FBF705FDE86A33
:10C78000F862A86AB86295F8240087F82400286B3C
:10C790003863084830610848F0600848B0600848CD
:10C7A00070600848306008487061022084F85400C6
:10C7B000012081E7B9200108E51E0108651F010875
:10C7C0007F1F010809200108011E010838B5054630
:10C7D00001213C2000F052FE0121084600F04EFEEF
:10C7E00001211348FFF722F9AC681CB911A002F02F
:10C7F000C3FB38BD2088ADF8000010208DF8030081
:10C8000002208DF8020069466068FFF783F8207AFD
:10C81000012804D121886068FFF75BF905E0207AE0
:10C8200018B921886068FFF752F900BFE1E70000FE
:10C83000000230004F5053206973204E554C4C0D70
:10C840000A00000010B5034800F08EF8024800F01E
:10C85000B6F810BD640B0020780B002010B503481B
:10C8600000F0ADF8024800F07FF810BD640B002026
:10C87000780B002010B5034800F076F8024800F06D
:10C8800073F810BD640B0020780B002070B50546CE
:10C890002C68206800B970BD20462168884700BF19
:10C8A000F9E7000038B5054601213C2000F0E6FD1F
:10C8B000AC681CB910A002F05FFB38BD2088ADF851
:10C8C000000010208DF8030002208DF80200694658
:10C8D0006068FFF71FF8207A012804D1218860687A
:10C8E000FFF7F7F805E0207A18B921886068FFF7AC
:10C8F000EEF800BFE1E700004F5053206973204E6F
:10C90000554C4C0D0A00000038B5054601210420A5
:10C9100000F0B4FDAC6804B938BD2088ADF8000063
:10C9200010208DF8030003208DF80200694660682E
:10C93000FEF7F0FF207A012804D121886068FFF714
:10C94000C8F805E0207A18B921886068FFF7BFF8B9
:10C9500000BFE1E710B5044621886068FFF7B7F82B
:10C9600000202072012010BD70B504462068456883
:10C97000686808B9002070BD2268906869688847B7
:10C980000120F8E710B5044621886068FFF796F8A3
:10C9900010BD70B5044620684568A86808B9032032
:10C9A00070BD22689068A9688847F9E710B5044609
:10C9B00021886068FFF78DF80120207210BD70B5E6
:10C9C000044620684568286808B9002070BD2268C0
:10C9D0009068296888470120F8E738B505460121A5
:10C9E000102000F04BFDAC6804B938BD2088ADF8CC
:10C9F000000048208DF8030003208DF802006946EE
:10CA00006068FEF787FF00BFEFE770B504460020BF
:10CA100000BF14F8016B8E4204D1012A00D108E056
:10CA2000551EEAB203B904E0451CA8B25D1EABB2C4
:10CA3000EFE700BF70BD000010B51448C07E0128AC
:10CA400003D164201249086003E04FF47A70104962
:10CA500008600F4801680F4801F04CFA012813D113
:10CA60000D4801780068401C0B4A106001F001007D
:10CA700018B10A48FFF778FF02E00848FFF79FFF68
:10CA80000021044801F036FA10BD0000240C0020FB
:10CA9000080000200000002004000020EC0A002014
:10CAA00010B53221124801F045FA012812D111487F
:10CAB0000078401C0F4908700F4B0122084601788E
:10CAC000022001F05DFA0D4B02220A480178052090
:10CAD00001F056FA42F21071094801F00BFA30B930
:10CAE000084B032203480178052001F049FA10BDE4
:10CAF000CC060020C8060020D5CE000865D000086E
:10CB0000D006002001D1000800BFFEE7704710B535
:10CB10004FF4A06000F03AF810BD000070B500219D
:10CB200000230F22C47804B3154C246804F4E06495
:10CB3000C4F5E064210AC1F10403CA40447804FA50
:10CB400003F184781440214309010E4C0678A15565
:10CB5000047804F01F050124AC4005786D11AD0088
:10CB600005F1E025C5F8004109E0047804F01F054F
:10CB70000124AC40044D0678761145F8264070BD7E
:10CB80000CED00E000E400E080E100E00249014338
:10CB9000024A1160704700000000FA050CED00E049
:10CBA000024A0A400243024B1A60704780FFFF1F8F
:10CBB00008ED00E0014908627047000000000E42E5
:10CBC00010B5044604F10B03184607F08BFB1868F8
:10CBD000C0F309300A2190FBF1F0074981F86600A3
:10CBE0005868800C81B20448C1875868800C81B2B3
:10CBF00001480181012010BDFC07002070B50446EA
:10CC000004F10B05284607F06DFB6A68C2F3C262A7
:10CC1000D0B2034A926ED1698847012070BD0000EE
:10CC2000FC07002010B5044604F10B03184607F07A
:10CC300059FB988881B20548A0F860105868010C2B
:10CC40000248A0F86210012010BD0000FC0700207F
:10CC500010B5044604F10B03184607F043FB98880F
:10CC6000010A054880F864105868010E024880F8EF
:10CC70006510012010BD0000FC07002070B50546BE
:10CC8000FCF704FB05F10B04204607F02BFB606862
:10CC9000C0F3892000EB80004FF6FF7101EA4000ED
:10CCA0000549A1F841006068000D81B20248A0F872
:10CCB0004310012070BD0000FC07002010B50446A1
:10CCC00004F10B03184607F00DFB0449186888624D
:10CCD00002485968C162012010BD00008023002075
:10CCE00010B5044604F10B03184607F0FBFA04499B
:10CCF00018680863024859684163012010BD0000AC
:10CD00008023002010B5044604F10B03184607F0F9
:10CD1000E9FA04491868886302485968C163012028
:10CD200010BD00008023002070B5054605F10B04FE
:10CD3000204607F0D7FA2068C0F34040C1B214483B
:10CD400080F845106068000C0A2190FBF1F0104952
:10CD5000A1F83300A088C0F38D00088021780C482A
:10CD600041712088000A2838C1B2094880F83B1078
:10CD70006068010C0648A0F839102268C2F300422E
:10CD8000D0B2034A926E51688847012070BD0000FE
:10CD9000FC07002010B5044604F10B03184607F009
:10CDA000A1FA9888C0F38D0081B20948C180186843
:10CDB000000A07494880000C08715868000DA0F56A
:10CDC0007A6081B20248A0F83510012010BD000041
:10CDD000FC07002010B5044604F10B03184607F0C9
:10CDE00081FA0449186808650248596841650120BC
:10CDF00010BD0000802300202DE9F0412A4805885D
:10CE000001272A482A494860002008702B463A46E4
:10CE100020212648FFF7F9FD044625494C700846B5
:10CE2000416824A002F0A8F8AC4202D10120BDE87C
:10CE3000F081781CC7B231E01C48005D202802D187
:10CE4000601C84B22AE02646184801191848027866
:10CE5000083040F822102B463A4620211348FFF7AD
:10CE6000D4FD0446A01BC1B2114802781830815489
:10CE700018380378083050F823200838017811A0BA
:10CE800002F07AF80A480078401C09490870084600
:10CE90000078042800DB03E0781CC7B2AC42CBD199
:10CEA00000BF0120C3E70000820200209A1C00207E
:10CEB000941F0020696E6F757420636D643A25734A
:10CEC0000A000000256420706172616D3A25730AC2
:10CED000000000007CB500200090019000900190BF
:10CEE0004FF4457058490860486000200872487245
:10CEF000082088726C465548FFF74BFD012801D188
:10CF0000012200E00022D4E9000162F31961C4E9C2
:10CF100000014E48FFF73DFD012801D1012100E04D
:10CF20000021D4E9000261F39B62C4E90002484891
:10CF3000FFF72FFD012801D0012200E00022D4E9F3
:10CF4000000162F31D71C4E900014148FFF721FDB2
:10CF5000012801D0012100E00021D4E9000261F3A1
:10CF60009F72C4E900023B484078D4E9001260F3A4
:10CF70001142C4E9001237480078D4E9001260F386
:10CF80009342C4E90012FEF7BFF90146D4E900203C
:10CF900061F38B22C4E90020FEF70AF90246D4E9C6
:10CFA000000162F31551C4E900012B48B0F81B20C1
:10CFB000D4E9001062F35D51C4E900102648B0F8CE
:10CFC0001D20D4E9000162F31430C4E90001FEF72A
:10CFD00049F90246D4E9001062F3DF71C4E9001098
:10CFE0001E4908681E49FBF771F90646FBF7DAFA95
:10CFF000054642F21070854201D9014600E02946FB
:10D00000D4E9000261F30C02C4E900022420FEF717
:10D01000C7FA0146D4E9002061F39E72C4E90020FA
:10D020000022D4E9000162F3D751C4E9000120468F
:10D0300007F05FF904480B300099016001994160E5
:10D040000B3803F06BFF7CBDE0230020000B0020B9
:10D05000140B0020D40700206C0C0020640000207A
:10D0600000007A441CB500200090019000900190CF
:10D070004FF47A701F4908604860002008724872B7
:10D08000082088726C46FEF765FA0246D4E9000172
:10D0900062F38E31C4E90001174A906E926E916975
:10D0A0008847012801D1012200E00022D4E90001D3
:10D0B00062F3CF31C4E90001104948688047024655
:10D0C000D4E9000162F31F61C4E900011422D4E92C
:10D0D000000162F31741C4E90001204607F009F995
:10D0E00004480B3000990160019941600B3803F04E
:10D0F00015FF1CBDE0230020FC0700206400002079
:10D100001CB50020009001900090019040F23F403B
:10D110000A49086048600020087248720820887236
:10D120006C46204607F0E5F804480B300099016092
:10D13000019941600B3803F0F1FE1CBDE023002093
:10D1400070B5054605F10B04204607F0CBF82268C0
:10D15000C2F30362D0B2064A926E51698847626890
:10D16000920FD0B2024A926ED1688847012070BDFA
:10D17000FC0700207047000070B542A001F0FCFEE3
:10D180004B4A906E926E916988474A4951F8204007
:10D19000214649A001F0F0FE454890F866204C4831
:10D1A00000784C4B53F820104BA001F0E5FE4048AE
:10D1B00090F84500012801D14EA000E051A00146A1
:10D1C00054A001F0D9FE3A48B0F84320B0F841101D
:10D1D00053A001F0D1FE5A48B0F81D20B0F81B1042
:10D1E00058A001F0C9FE5F49C868FBF7EFF9044693
:10D1F00022460B465CA001F0BFFE6049886880476C
:10D2000004465E49486880470546224629465CA098
:10D2100001F0B2FE4FF400415F48FEF74FFC08B149
:10D220005EA000E05FA004464FF480415A48FEF73C
:10D2300045FC08B15BA000E058A0054622462946FF
:10D240005AA001F099FE6048407808B15FA000E064
:10D250005FA002465C48007808B15EA000E05EA0D6
:10D2600001465EA001F088FE44490868FBF7AEF96C
:10D27000044622460B465FA001F07EFEFEF746F90B
:10D2800070BD00000D0AA1AAA1AAA1AAA1AAA1AAE3
:10D29000A1AAA1AAA1AAA1AAA1AAA1AAA1AAA1AA36
:10D2A000A1AAA1AAA1AAA1AAA1AAA1AA0D0A0000A5
:10D2B000FC070020880800200D0A56435520576FB0
:10D2C000726B696E67204D6F64652025730D0A00CF
:10D2D00058240020680800204368617267696E67FF
:10D2E00020537461676520257309534F43202564DB
:10D2F0000D0A0000436F6E7374616E74566F6C7428
:10D3000061676500436F6E7374616E74437572720A
:10D31000656E74004D6F64652025730D0A00000072
:10D3200044656D616E6420766F6C7461676520255D
:10D33000642063757272656E742025640D0A0000A6
:10D340006C0C00204F757470757420766F6C74616E
:10D3500067652025642063757272656E742025648C
:10D360000D0A0000CC0B002053616D706C20766FAD
:10D370006C74616765202566200D0A00640000203A
:10D3800054656D70312025642047554E5F54454DDE
:10D39000502025640D0A000000100140436C6F739B
:10D3A000650000004F70656E0000000044435F524E
:10D3B000656C61792025732041435F52656C61790A
:10D3C0002025730D0A000000D407002043433200DB
:10D3D00043430000435000004343310043502D437A
:10D3E00043312025732043432D4343322025730DC1
:10D3F0000A000000434320522069732025660D0A6D
:10D400000000000001460020034A506820F440401C
:10D4100008435060704700000010024029B1064ADE
:10D4200052690243044B5A6104E0034A5269824341
:10D43000014B5A61704700000010024029B1064AB2
:10D44000D2690243044BDA6104E0034AD2698243A1
:10D45000014BDA61704700000010024029B1064A12
:10D4600012690243044B1A6104E0034A12698243C1
:10D47000014B1A61704700000010024029B1064AB2
:10D4800092690243044B9A6104E0034A9269824321
:10D49000014B9A617047000000100240014908608A
:10D4A00070470000400442422DE9F0410021002273
:10D4B000002500230026002400278C46DFF8608129
:10D4C000D8F8048008F00C0121B1042907D00829FC
:10D4D00059D109E0DFF84C81C0F8008058E0DFF84E
:10D4E0004481C0F8008053E0DFF83481D8F804802C
:10D4F00008F47012DFF82881D8F8048008F4803529
:10D50000920C0D2A01D0921C00E0062235B9DFF8FA
:10D51000188102FB08F8C0F8008033E0DFF80081D2
:10D52000D8F82C8008F48036DFF8F480D8F82C8006
:10D5300008F00F0808F1010446B9DFF8E880B8FBED
:10D54000F4F808FB02F8C0F800801BE0DFF8D08098
:10D55000D8F82C80C8F3031808F10107DFF8C08061
:10D56000D8F82C80C8F3032808F1020CDFF8B48047
:10D57000B8FBF7F808FB0CF8B8FBF4F808FB02F866
:10D58000C0F8008004E0DFF89C80C0F8008000BF95
:10D5900000BFDFF88C80D8F8048008F0F00109099A
:10D5A000DFF8888018F80130D0F8008028FA03F8F6
:10D5B000C0F80480DFF86880D8F8048008F4E061DF
:10D5C000090ADFF8688018F80130D0F8048028FADA
:10D5D00003F8C0F80880DFF84880D8F8048008F421
:10D5E0006051C90ADFF8448018F80130D0F804808F
:10D5F00028FA03F8C0F80C80DFF82480D8F80480FB
:10D6000008F44041890BDFF8288018F80130D0F881
:10D610000C80B8FBF3F8C0F81080BDE8F081000082
:10D620000010024000127A0000093D004906002067
:10D630005906002010B501460022002300204A119F
:10D64000012A02D1094C236806E0022A02D1074CC4
:10D65000236A01E0054C636A01F01F020124944033
:10D660001C400CB1012000E0002010BD0010024061
:10D670000149086070470000800442420149086087
:10D68000704700003C0442420249096A0143014AD2
:10D69000116270470010024010B50D48008F00F471
:10D6A000804058B90A4890F8380000F0200028B9A6
:10D6B000074890F8380000F0400030B12720FDF70F
:10D6C00089FF00200249886310BD0120FCE70000AB
:10D6D0006C0C002070B505460E46002400BF03E028
:10D6E000285D00F045FE641CB442F9DB70BD70B5E6
:10D6F00005460E46002400BF03E0285D00F038FE1A
:10D70000641CB442F9DB0D2000F032FE0A2000F068
:10D710002FFE002403E0285D00F0E6FC641CB44208
:10D72000F9DB70BD0348008840F010000149088013
:10D730007047000004280040034800884FF6EF714E
:10D740000840014908807047042800400021034830
:10D750000188001F008841EA004070471C280040F3
:10D7600010B501214FF0C050FFF768FE4FF4007074
:10D77000FFF78AFF0120FFF781FF0120FFF71AFA68
:10D78000FBF7C8FC0120FFF773FF00BF6120FFF724
:10D7900051FF0028FAD04FF40070FFF775FF012009
:10D7A000FFF76CFF00F024F800F018F849F63F404E
:10D7B00000F004F800F012F810BD000000B50246B9
:10D7C000FFF7B0FFC2F3034003490880091D0A8038
:10D7D000FFF7B2FF00BD00000828004000BF03486B
:10D7E000008800F020000028F9D07047042800408D
:10D7F000074800884FF6F77108400549088000BFC8
:10D800000348008800F008000028F9D070470000A5
:10D810000428004010B5012013490860FEF7FEFD02
:10D820009020FEF735FE0020FEF732FEFEF716FED2
:10D83000FEF7F4FD9120FEF72BFEFEF7AFFD0B493E
:10D840000880FEF7ABFD09494880FEF707FE074850
:10D8500040880649098840EA012000B2034908804F
:10D860000846008880B210BD98812142B80000208F
:10D8700070B505461DB1686808B1A86808B90020F0
:10D8800070BD00240EE004EB440000EBC4001B4913
:10D8900001EB001000782978884201D10020EFE7E1
:10D8A000601CC4B2022CEED3002422E004EB44003E
:10D8B00000EBC400114901EB00100078FF2816D1DD
:10D8C00004EB440101EBC4010C4A02EB01102022DD
:10D8D0002946FAF759FC012004EB440101EBC4018D
:10D8E000064A02EB011181F854000548C8E7601CA4
:10D8F000C4B2022CDAD30020C2E70000601300207B
:10D900003801002000200149088070478202002071
:10D91000704772B6704762B6704770B504460D46E0
:10D92000FFF714FF0646206818B9266020682844CF
:10D9300060606068B04201D8012070BD0020FCE743
:10D9400001460020086048600120704710B500F0D3
:10D9500001F810BD0CB5002001900090404800680F
:10D9600040F480303E49086000BF3D48006800F444
:10D97000003000900198401C0190009820B94FF6AB
:10D98000FF7101988842F0D13548006800F40030FA
:10D9900010B10120009001E00020009000980128C3
:10D9A0005CD13048006840F010002E4908600846FD
:10D9B000006820F0030008600846006840F002009C
:10D9C0000860274840682649486008464068486023
:10D9D0000846406840F4806048600846C06A2249B2
:10D9E00008401F49C8620846C06A204908431C49CC
:10D9F000C8620846006840F08060086000BF1848B0
:10DA0000006800F000600028F9D01548406820F454
:10DA10007C10134948600846406840F4E8104860AC
:10DA20000846006840F08070086000BF0C4800683D
:10DA300000F000700028F9D00948406820F0030089
:10DA4000074948600846406840F00200486000BF4F
:10DA50000348406800F00C000828F9D10CBD000014
:10DA6000001002400020024000F0FEFF14080100F8
:10DA7000014602480170012070470000D8070020CD
:10DA80000146032903D0042901D000207047024831
:10DA9000C1700120FAE70000D807002001460129E3
:10DAA00002D009B100207047014881700120FAE7D7
:10DAB000D8070020002201490A5470477024002032
:10DAC0000146012902D009B1002070470148417088
:10DAD0000120FAE7D807002010B5FFF78DF908B943
:10DAE000002010BD0020154908801DE0134A12884F
:10DAF00002EB4202124B03EB82025168114A50685A
:10DB0000FAF766FB58B10D48008800EB40000C495D
:10DB100001EB8000846804B1A0470120E1E70748D9
:10DB20000088401C05490880044800880B28DDD384
:10DB300005A001F021FA0020D3E700008C020020AC
:10DB4000B44B0108941F0020416E20756E7265630E
:10DB50006F676E697A656420434D4420210A000096
:10DB600010B50948006820B9084803F011F90649C2
:10DB700008600548006803F09EF920B90A210248B0
:10DB8000006803F08BF910BD4C01002061450108CD
:10DB900010B5FBF7F5FA20B908A001F0EDF9002067
:10DBA00010BDFDF7CFFB08B90020F9E7FDF766FBD4
:10DBB00008B90020F4E70120F2E70000424D5320AD
:10DBC000546865204368617267696E6720506861B8
:10DBD00073652053746F70732041626E6F726D6154
:10DBE0006C6C790A0D0000000F480068401C0E495B
:10DBF00008600E480068401C0C4908600A4800682C
:10DC00004FF47A71B0FBF1F201FB1200012804D14C
:10DC100007480068401C064908600648007810B9AB
:10DC2000012004490870704758020020500200206B
:10DC30005C0200205402002030B5164800684FF402
:10DC40007A72B0FBF2F1B1F1807F01D301201DE0C7
:10DC500021F07F40401E4FF0E022506150170F220C
:10DC6000002807DA13071D0E0B4B00F00F04241FCA
:10DC70001D5503E013071C0E084B1C5400BF002069
:10DC80004FF0E022906107201061002008B100BF32
:10DC9000FEE730BD0C00002018ED00E000E400E0DD
:10DCA00010B5FEF72DFC4FF417720249024802F03E
:10DCB0009DFD10BD4415002000F0010810B5164868
:10DCC000006840F0010014490860084640681349A4
:10DCD00008401149486008460068114908400E494B
:10DCE00008600846006820F4802008600846406804
:10DCF00020F4FE0048600846006820F0A05008604C
:10DD00004FF47F0088600020C862FFF71FFE4FF0CD
:10DD100000600449086010BD001002400000FFF0E0
:10DD2000FFFFF6FE08ED00E02DE9F0470D480488FE
:10DD30000D4A0021204601F03BF80B480068FAF735
:10DD400045FC07463A460B4608480949FAF7A0FB46
:10DD50000546FAF77FFC8146FDF722FD054908726A
:10DD6000BDE8F087C00B0020A40000209A99999983
:10DD700099991340CC0B002010B50121054800F003
:10DD80004CF830B10449086880470121014800F08F
:10DD900035F810BD00040040C40600207FB50546DC
:10DDA0000C4601210220FFF749FBADF80850ADF801
:10DDB00004400020ADF80A00ADF8060001A90E48A5
:10DDC00000F046F8012211460B4800F037F81D20FC
:10DDD0008DF8000001208DF8010003208DF802006D
:10DDE00001208DF803006846FEF798FE01210248E5
:10DDF00000F007F87FBD000000040040CA43028223
:10DE0000704721B1028842F00102028004E00288DA
:10DE10004FF6FE731A400280704730B5024600206C
:10DE200000230024158A05EA0103958905EA010407
:10DE300013B10CB1012000E0002030BD1AB183897C
:10DE40000B43838102E083898B4383817047000009
:10DE5000002202881D4B98420ED01D4B98420BD0D9
:10DE6000B0F1804F08D01B4B984205D01A4B984216
:10DE700002D01A4B984204D14FF68F731A404B8848
:10DE80001A43174B984207D0164B984204D04FF6CE
:10DE9000FF431A40CB881A4302808B8883850B8806
:10DEA00003850A4B98420BD0094B984208D00E4B81
:10DEB000984205D00D4B984202D00D4B984201D1AB
:10DEC0000B7A03860123838270470000002C0140F7
:10DED000003401400004004000080040000C0040F5
:10DEE0000010004000140040004001400044014088
:10DEF000004801400246002321B90D480068106027
:10DF0000012070470A4803681068984205D81068D5
:10DF1000181A884209D30120F3E71068C0F1FF30D6
:10DF20001844884201D30120EBE70020E9E7000014
:10DF3000580200200246002321B9104800681060F2
:10DF4000012070470D4803681068984208D810688F
:10DF5000181A88420FD30948006810600120F0E7C2
:10DF60001068C0F1FF301844884204D303480068A9
:10DF700010600120E5E70020E3E7000058020020E0
:10DF80002DE9F04104460F4615461E4697FBF4F076
:10DF900004FB1070A84200D1B047BDE8F08100003A
:10DFA0004F48007801280AD14E48C068401C4D49AE
:10DFB000C8600120087000204949087000E07047DF
:10DFC0004848C0680521B0FBF1F201FB120030B9EE
:10DFD0004448C06818B101204249487000E0EEE7AB
:10DFE0004048C0680A21B0FBF1F201FB120028B9D9
:10DFF0003C48C06810B101203A4988703948C0686F
:10E000001421B0FBF1F201FB120028B93548C068B9
:10E0100010B101203349C8703248C0683221B0FBCA
:10E02000F1F201FB120028B92E48C06810B101209E
:10E030002C4908712B48C0686421B0FBF1F201FB48
:10E04000120028B92748C06810B10120254948713D
:10E050002448C0684FF4FA71B0FBF1F201FB1200E2
:10E0600028B92048C06810B101201E4988711D4898
:10E07000C0684FF47A71B0FBF1F201FB120028B9CD
:10E080001848C06810B101201649C8711548C06809
:10E0900040F2DC51B0FBF1F201FB120028B911484B
:10E0A000C06810B101200F4908720E48C0684FF4D3
:10E0B000FA61B0FBF1F201FB120028B90948C0680F
:10E0C00010B10120074948720648C06841F27071DA
:10E0D000884202D300200349C86000BF6FE70000F8
:10E0E000540200203415002010B50446214605488E
:10E0F00000F01FFB00BF0348008800F080000028EC
:10E10000F9D010BD004C004010B540F225513948FF
:10E1100000F04FFAF8B1374800F006FBC4B23648B9
:10E120000088C82808DA344801880088401C324A30
:10E1300010803248445402E000202F4908800A2C05
:10E1400004D1FFF7C9FCFFF7DDFB10BD40F22551FC
:10E15000284800F006FA40F22441264800F029FA47
:10E1600048B1FFF7CFFB234800F0DEFA40F224412C
:10E17000204800F0F6F940F227711E4800F019FA25
:10E1800020B140F227711B4800F0EBF940F2266104
:10E19000184800F00EFA20B140F22661154800F050
:10E1A000E0F90821134800F0F7F9012806D1082109
:10E1B000104800F0CDF90F4800F0B6FA04210D48E0
:10E1C00000F0EAF9012806D104210A4800F0C0F95C
:10E1D000084800F0A9FA0221064800F0DDF90128FC
:10E1E00006D10221034800F0B3F9024800F09CFA7E
:10E1F00000BFAAE7004C0040820200209A1C0020C9
:10E2000010B540F22551334800F0D3F9E8B1314858
:10E2100000F08AFAC4B230480088C82808DA2E48CC
:10E2200001880088401C2C4A10802C48445402E08D
:10E2300000202949088000202949088029490870C0
:10E2400040F22551234800F08CF940F22441214846
:10E2500000F0AFF950B11F4800F066FA01202149E3
:10E26000087040F224411B4800F07BF940F226611F
:10E27000184800F09EF920B140F22661154800F0E0
:10E2800070F90821134800F087F9012806D1082108
:10E29000104800F05DF90F4800F046FA04210D48DF
:10E2A00000F07AF9012806D104210A4800F050F95B
:10E2B000084800F039FA0221064800F06DF90128FB
:10E2C00006D10221034800F043F9024800F02CFA7D
:10E2D00010BD00000050004088020020621D002098
:10E2E000840200208602002010B540F225511D480E
:10E2F00000F05FF910B31B4800F016FAC4B21A48D8
:10E30000008800F40040C8B91748008800F4804035
:10E3100060B10A2C03D000201349088020E0124885
:10E32000008840F400401049088019E00D2C06D107
:10E330000D48008840F480400B49088010E00A48EE
:10E340000088C0F30D0009490C5407480088401CA0
:10E350000549088008460088C72801DD002008809C
:10E3600010BD000000380140720200200C1A00208D
:10E3700010B504462146054800F0DBF900BF03480C
:10E38000008800F080000028F9D010BD0044004053
:10E3900010B540F22551304800F00BF9C0B12E48BD
:10E3A00000F0C2F9C4B22D480088FE2808DA2B48D4
:10E3B00001880088401C294A10802948445402E002
:10E3C00000202649088040F22551234800F0C9F872
:10E3D00040F22441204800F0ECF850B11E4800F013
:10E3E000A3F901201F49087040F224411A4800F0A7
:10E3F000B8F840F22661184800F0DBF820B140F28E
:10E400002661154800F0ADF80821134800F0C4F863
:10E41000012806D10821104800F09AF80E4800F0B3
:10E4200083F904210C4800F0B7F8012806D1042133
:10E43000094800F08DF8084800F076F902210648F6
:10E4400000F0AAF8012806D10221034800F080F864
:10E45000014800F069F910BD00440040740200203A
:10E46000D41A00207602002010B540F2255133481E
:10E4700000F09FF8E8B1314800F056F9C4B23048D6
:10E480000088C82808DA2E4801880088401C2C4AD9
:10E4900010802C48445402E00020294908800020C4
:10E4A000294908802949087040F22551234800F085
:10E4B00058F840F22441214800F07BF850B11F4841
:10E4C00000F032F901202149087040F224411B4834
:10E4D00000F047F840F22661184800F06AF820B1D1
:10E4E00040F22661154800F03CF80821134800F07E
:10E4F00053F8012806D10821104800F029F80F48E8
:10E5000000F012F904210D4800F046F8012806D168
:10E5100004210A4800F01CF8084800F005F902211F
:10E52000064800F039F8012806D10221034800F01E
:10E530000FF8024800F0F8F810BD00000048004055
:10E540007C020020D21B0020780200207A020020EA
:10E5500001F40072B2F5007F00D100BFCA4302800F
:10E56000704710B50022002340F66A14A14200D182
:10E5700000BF0A1201249440A3B2DC43048010BD02
:10E5800021B1828942F40052828104E082894DF6F1
:10E59000FF731A408281704702460020B1F5007F68
:10E5A00000D100BF13880B400BB1012000E0002018
:10E5B000704770B50246002400230025002040F675
:10E5C0006A16B14200D100BFC1F3421501F01F032A
:10E5D000012606FA03F3012D02D19689334006E0A5
:10E5E000022D02D1168A334001E0968A33400C1284
:10E5F000012606FA04F41688344013B10CB1012048
:10E6000000E0002070BDF0B5034600240026002580
:10E61000002040F66A17B94200D100BF1846C1F386
:10E62000421401F01F06012707FA06F5012C01D15B
:10E630000C3004E0022C01D1103000E014301AB18B
:10E6400007682F43076002E00768AF430760F0BD2B
:10E650002DE9F04786B005460E460024A24600BFCD
:10E66000A1460027B08900B100BF2F462C8A4CF686
:10E67000FF700440F08804432C82AC894EF6F310FE
:10E680000440B08831890843718908430443AC8150
:10E69000AC8A4FF6FF400440B0890443AC8201A825
:10E6A000FEF702FF1F48874202D1DDF810A001E00B
:10E6B000DDF80CA0A88900F4004040B10AEBCA00C4
:10E6C00000EB0A1031684900B0FBF1F807E00AEBF3
:10E6D000CA0000EB0A1031688900B0FBF1F8642031
:10E6E000B8FBF0F004012009642101FB1089A8891E
:10E6F00000F4004040B1322000EBC900B0FBF1F063
:10E7000000F00700044308E0322000EB0910642108
:10E71000B0FBF1F000F00F0004432C8106B0BDE81F
:10E72000F08700000038014001468888C0F30800E7
:10E730007047C1F308028280704700002DE9F74F4F
:10E7400084B00C4617460026FDF7DAFE0498002830
:10E7500056D12079DA49087060794870A0790006AE
:10E76000E17940EA0140217A40EA0120617A0843D8
:10E77000D3494860A07AE17A40EA0120D049088173
:10E78000E07B0006A17B40EA0140617B40EA01207A
:10E79000217B0843CA49C860207C617C40EA012093
:10E7A000C7490882701E88610020C86148624FF620
:10E7B000FF7008840020C3490870C148008AC0491E
:10E7C000C968BF4A1289CDE900210290BC4843685C
:10E7D00042780178BCA000F0CFFBB948008AB84964
:10E7E000C968B74A1289CDE900210290B44843684C
:10E7F00042780178C34800F0BFFBFAF795FD5CE171
:10E8000004980128FBD1AF48007810B107B0BDE8EB
:10E81000F08FE0780006A17840EA0140617840EA94
:10E82000012021780843A6494861FAF73DFDFDF72C
:10E8300067FEA3483A464169B3A000F09DFBA0489B
:10E8400080699F494969884272D09D4840699C49C6
:10E8500088610846C169A7F10D0008449849C8615C
:10E860000846C369808BC0F30A020846C069C10A22
:10E87000ABA000F081FBFCF773FF9148008C90493E
:10E88000C969B0EBD12F14D08D48C069C0F3CF2037
:10E890008B4908840846C069AD4908444FEAD0282E
:10E8A0004FEAC8284146ABA000F066FB4046FCF7A3
:10E8B000B3FE04F1040AA7F10D00C11700EB91713A
:10E8C000C1F3870BC11700EB91718910A0EB810197
:10E8D00069B1A7A000F050FBA7F1090108190322B4
:10E8E000FF21F9F763FC0BF1010000F0FF0B744806
:10E8F000406A974900EB01087148C0697049486255
:10E90000002540E0002614E05AF825104046FCF7A8
:10E91000EFFE042800D10DE0701CC6B2032E08DB08
:10E92000414699A000F028FB0120664908706DE778
:10E93000C1E0E9E700BFD8F80090012D03DBABF19F
:10E940000100A84206DC5AF825204B46414697A014
:10E9500000F012FB5AF8250048450DD09BA000F0AE
:10E960000BFB5AF825204B46414690A000F004FBD3
:10E9700001205449087049E708F10408032E00DB20
:10E9800003E0681CC5B25D45BCDB00BFFDF7B8FD08
:10E99000A7F10D0081B296480288201DFAF74CFDC0
:10E9A00093490880464801899148028891A000F067
:10E9B000E3FAFDF7A5FD424840694149C96888422C
:10E9C00077D13F4800898A490988884203D092A0BC
:10E9D00000F0D2FA1AE700263948C16898A000F082
:10E9E000CBFAA048FCF718FE0FE09F499D48FCF7C2
:10E9F0007FFE042800D109E0701CC6B2032E04DBA0
:10EA000098499AA000F0B8FA00E0EEE700BF9548F8
:10EA1000D0F800904B46944A014664A000F0ACFA4E
:10EA20009148814503D0012026490870EEE6002672
:10EA300012E0234841688B48001DFCF759FE04286A
:10EA400000D10AE0701CC6B2032E05DB8549091D02
:10EA50008FA000F091FA00E0EBE700BF8148001DB5
:10EA6000D0F8009016484B467E49091D426892A096
:10EA700000F082FA12484068484503D0012011494D
:10EA80000870C3E6FDF73CFDFAF70EFC93A000F01A
:10EA900073FA00BF9C48006800F4E0609B4908439B
:10EAA000001D99490860BFF34F8F00BF00BFFEE70C
:10EAB000FFE7FCF7F1FDFDF723FD00BFA6E6000030
:10EAC000E4190020C20500200D0A36363655706460
:10EAD0002D2D747970653A2564202C7665723A255F
:10EAE000642C54627974653A25642C204372633A2D
:10EAF00025642C5061673A25642C506C656E3A256C
:10EB0000640D0A003C4E01080A0D437572722042E2
:10EB100061673A25642C206C656E2025640A0D001F
:10EB200057726974652D616464723A207365637409
:10EB30006F722025642C2C6F6666736574202564C3
:10EB4000202C7265636C656E202530640D0A000010
:10EB50000060020834344375727220457261736537
:10EB60002D2D616464723A202530780D0A00000072
:10EB70000A0D6C6173742D2D2D2D2D62616721217D
:10EB800021212121210A0D0021323221212121219F
:10EB90002121212157726974652D4661696C2D61AF
:10EBA0006464723A202530780D0A00006164647252
:10EBB000202530782C2C5772697465202530782CEC
:10EBC0002C72656164202530780D0A000A0D2072D0
:10EBD00065616476616C20213D20557064646174C8
:10EBE000615B695D2921212121210A0D00000000BE
:10EBF000C0050020313232557064486561642E468C
:10EC0000696C654372633D2530782C544372633DD3
:10EC10002530780D0A000000557064486561642E47
:10EC200046696C6543726320213D20544372632022
:10EC30002121212072657475726E210D0A00000079
:10EC40002121217570642D696E666F212120577214
:10EC50006974652D746F74706167202564200D0AD6
:10EC6000000000000058020844332211557064442B
:10EC7000617461466C6167212057726974652D4625
:10EC800061696C2D616464723A202530780D0A0048
:10EC90002121217570642D696E666F2121205772C4
:10ECA0006974652D4661696C2D616464723A202532
:10ECB00030780D0A00000000316164647220253054
:10ECC000782C2C5772697465202530782C2C72654D
:10ECD0006164202530780D0A000000003232757022
:10ECE000642D616C6C207772697465204F4F4B4BBB
:10ECF00021217265737461727421212121212121E6
:10ED0000212121210D0A00000CED00E00000FA0590
:10ED100070B5C2B005460C46002641F20D00084908
:10ED2000A1F80500224629460548C01DF9F72CFA2E
:10ED30000348448001AA02A9FCF762FB42B070BDFF
:10ED40002A1E002000BFFEE710B5064A906E926EA4
:10ED5000116A884720B92620FCF73CFC002010BD32
:10ED60000120FCE7FC07002010B5074A906E926E68
:10ED700091698847042804D02220FCF72BFC00204E
:10ED800010BD0120FCE70000FC0700202DE9F04148
:10ED900004460E461546601BF9F7E9FB80463146EE
:10EDA000F9F7C6FA0746F9F7FDFB80B2BDE8F08136
:10EDB0002DE9FC4781460C46924604EB44003B4952
:10EDC00011F82000002843D004EB440001EB800040
:10EDD000408888B304EB440001EB80004088142194
:10EDE00090FBF1F004EB4401304A02EB81014880D2
:10EDF00004EB440102EB81014888F9F7C6FB0746A2
:10EE00004FF066322A4BF9F7D1FA05460022294B1A
:10EE1000F9F73EFBCDE90001F9F71CFC04EB4401D6
:10EE2000224A02EB8101886004EB4400114601EBA9
:10EE300080008068CAF80000002004EB44011B4AEF
:10EE400002EB8101488004EB440102F821002BE031
:10EE500004EB4400154901EB80000079401C04EBF1
:10EE60004401124A02EB8101087104EB440011468F
:10EE700001EB80004088484404EB440102EB81012F
:10EE8000488004EB4400114601EB8000007914280F
:10EE90000AD1012004EB440102F82100002004EB18
:10EEA000440102EB81010871BDE8FC87DC0B002006
:10EEB00066660A400000B040002008490860084823
:10EEC0000078401C06490870084600781E2803DCBC
:10EED0007F2002490839086070470000082C004074
:10EEE0004D02002044E032213EE000BF00BF00BFE1
:10EEF00000BF00BF00BF00BF00BF00BF00BF00BF1A
:10EF000000BF00BF00BF00BF00BF00BF00BF00BF09
:10EF100000BF00BF00BF00BF00BF00BF00BF00BFF9
:10EF200000BF00BF00BF00BF00BF00BF00BF00BFE9
:10EF300000BF00BF00BF00BF00BF00BF00BF00BFD9
:10EF400000BF00BF00BF00BF00BF00BF00BF00BFC9
:10EF500000BF00BF00BF00BF00BF00BF00BF00BFB9
:10EF600000BF00BF4A1ED1B20029BEDC421ED0B293
:10EF70000028B8DC704700000FB4054B10B503A99A
:10EF8000044A029800F0EEF810BC5DF814FB000093
:10EF9000A11001086C0200200FB4084B10B504A9A1
:10EFA00002AA039800F0DEF8044602A9002000F04F
:10EFB00070FC204610BC5DF814FB000093F80008BC
:10EFC00002E008C8121F08C1002AFAD17047704732
:10EFD000002001E001C1121F002AFBD17047000090
:10EFE0002DE9FF5F82B00021DDE90430020DDDF87C
:10EFF00040B0034318D044F61050A2F2FF3242430F
:10F000001514119801281FD0A5EB0B00401C5FEAD6
:10F01000000A4FF000064E4FDFF83891B0465046D8
:10F0200015D5CAF1000413E0119801244AA3012860
:10F0300001D16FEA0B010298119AC0E90031C0E9D1
:10F04000024206B0BDE8F09FCBF10000DFE70446C6
:10F050000021404A491842EB0450CDE9001012E06B
:10F06000E00707D032463B4640464946F9F79EF94D
:10F070008046894632463B4610461946F9F796F9CE
:10F0800006460F466410002CEAD1DDE90401DDE9F3
:10F090000023BAF1000F06DAF9F788F942464B4629
:10F0A000F9F784F905E0F9F7F3F942464B46F9F729
:10F0B000EFF904460E460022284BF9F7B3FA03D8BD
:10F0C0004FF0FF30014607E00022254B2046314635
:10F0D000F9F7CBFBF9F770FC102409E0002C0ADBF0
:10F0E0000A220023F9F7FCFA039B30321A55641EFA
:10F0F00050EA0102F2D1641C039AC4F111031444D2
:10F10000119A012A03D0012208430DD10AE00843D5
:10F1100004D000204FF0110B119072E7A3EB0B0508
:10F120006D1E0DE05B4504DD4FF0000205F10105A9
:10F1300004E003DA4FF00002A5F10105002AECD04B
:10F1400002981199C0E90231C0E9004579E7000051
:10F15000000014400000F03F300000000000F043C9
:10F160000000E03F2DE9FF4F95B09B4689460646DB
:10F1700000250FE2252877D100242746F84A0121EF
:10F18000059400E0044316F8013F203B01FA03F028
:10F190001042F7D130782A2811D06FF02F03307841
:10F1A000A0F13002092A16D8059A44F0020402EBB5
:10F1B000820203EB42021044761C0590EFE759F8F7
:10F1C000042B0592002A03DA504244F400540590BF
:10F1D00044F00204761C30782E2816D116F8010F60
:10F1E00044F004042A280DD06FF02F023078A0F1EB
:10F1F0003003092B09D807EB870302EB4303C71839
:10F20000761CF3E759F8047B761C30786C280FD015
:10F2100006DC4C2817D068280DD06A2814D104E0E9
:10F22000742810D07A280FD10DE044F400140AE0BD
:10F2300044F4801401E044F440147278824202D114
:10F2400004F58014761C761C307866280BD013DC0D
:10F25000582877D009DC002875D04528F6D04628F4
:10F26000F4D047281AD19DE118E0632835D06428EE
:10F2700079D0652812D195E1702873D008DC672811
:10F28000F1D069286FD06E280DD06F2806D1B5E077
:10F2900073282CD0752875D0782874D05A461799C1
:10F2A00090476D1C75E1C4F30250022809D0032871
:10F2B0000DD0D9F8001004280DD00D6009F1040913
:10F2C00067E1D9F80010EA17C1E90052F6E7D9F86A
:10F2D00000100D80F2E70D70F0E719F8041B8DF8AF
:10F2E000001000208DF80100EA46012003E059F8E3
:10F2F00004AB4FF0FF3061074FF0000102D40DE086
:10F3000008F101018846B9420FDA8045F8DB1AF8A6
:10F3100008100029F4D108E008F101018846814273
:10F32000FADB1AF808100029F6D105985B46A0EB25
:10F33000080721463846179A00F094FA284400EB53
:10F34000080507E04DE029E10DE01AF8010B5A46E7
:10F3500017999047B8F10108F7D25B462146384625
:10F36000179A13E142E00A220092C4F302524FF0CE
:10F37000000A022A08D059F804CB032A4FEAEC719C
:10F380000AD00DE029E02AE009F1070121F0070287
:10F39000F2E802C1914609E00FFA8CFC4FEAEC71E9
:10F3A000042A03D14FFA8CFC4FEAEC71002907DAEA
:10F3B0000A460021DCF1000C61EB02012D2202E083
:10F3C000220504D52B228DF80420012203E0E20758
:10F3D00001D02022F7E7904659E00A2102E01022EE
:10F3E0000DE010214FF0000A00910BE010224FF0C9
:10F3F000000A44F004040827009203E008224FF0BA
:10F40000000A0092C4F30252022A05D059F804CB34
:10F410000021032A08D009E009F1070121F00702C1
:10F42000F2E802C1914605E01FFA8CFC042A01D1E2
:10F430000CF0FF0C4FF00008220728D5702806D0EA
:10F44000009B83F0100353EA0A0305D00EE040222C
:10F450008DF80420012208E05CEA010206D0302287
:10F460008DF804208DF8050002229046009B83F061
:10F47000080353EA0A030AD15CEA010201D16207D8
:10F4800005D530228DF804204FF001087F1E582842
:10F4900004D034A003900EA802900DE036A0F9E746
:10F4A00053466046009AF9F71BF984460398825C3C
:10F4B0000298401E029002705CEA0100F0D10298AE
:10F4C00006A9081A00F1200A600702D524F4803446
:10F4D00000E00127574502DDA7EB0A0000E000200D
:10F4E00000EB0A01009005984144401A0590E003A2
:10F4F00006D45B462146179A059800F0B3F90544F7
:10F50000002706E001A85A46C05D179990476D1C78
:10F510007F1C4745F6DBE0030CD55B462146179A76
:10F52000059800F09FF9054404E030205A461799E9
:10F5300090476D1C0099481E00900029F5DC08E0FA
:10F54000029802995A460078491C029117999047EF
:10F550006D1CBAF10001AAF1010AF1DC65E10000BD
:10F560000928010030313233343536373839616299
:10F57000636465660000000030313233343536375D
:10F5800038394142434445460000000000F058F934
:10F590000544761C307800287FF4ECAD19B028467D
:10F5A000BDE8F08F620700D4062709F1070222F0B8
:10F5B000070CFCE80223E14603F000485FEA080C70
:10F5C00002D00FF2702C0DE05FEA045C02D50FF25E
:10F5D000682C07E05FEAC47C02D00FF2602C01E0E7
:10F5E000AFF2700C4FF0FF3823F00043CDF850C05D
:10F5F00065280CD006DC452809D046281DD04728B0
:10F600003DD13DE0662818D067287ED138E0002142
:10F61000112F01DB112000E0781CCDE9000106A9C3
:10F620000EA8FFF7DDFCDDE90F010E9A0391002122
:10F63000009207F1010A04914DE04FF0004000975D
:10F64000CDE9011006A90EA8FFF7CAFCDDE90F02FB
:10F6500003920E9B11990022DDF80CA000930492F6
:10F6600011B9791C00EB010AB7EB0A0004D4C0F110
:10F67000FF3007F1010A0490AAEB0700019044E073
:10F68000012F00DA01270021112F01DD112000E0F8
:10F690003846CDE9000106A90EA8FFF7A1FCDDE977
:10F6A0000F010E9A0391002104910092BA4621079E
:10F6B0000CD40399514500DA8A46BAF1010F05DDF1
:10F6C000009AAAF10101515C302908D0B84202DA4F
:10F6D00010F1040F06DA0121CDE9011015E0AAF1BD
:10F6E0000101E9E7002805DC049901440491AAEB33
:10F6F000000102E0411C514500DD8A460499401A90
:10F70000401C01904FF000400290200704D4019863
:10F71000504501DBCDF8048000208DF84F000298A1
:10F720000DF14F07B0F1004F25D02B200E9002981D
:10F730004FF0020800280CDA404202902D200E9073
:10F7400007E00A210298F8F7B5FF3031029007F878
:10F75000011DB8F10001A8F10108F2DC02980028AF
:10F76000EFD1791E0E980870307800F0200040F03C
:10F77000450007F8020D12A8C01B00F107081498F5
:10F78000007800B1012000EB0A01019801EBE07163
:10F7900005984144401A401E0590E00306D45B469C
:10F7A0002146179A059800F05DF8054414980078F2
:10F7B00018B15A46179990476D1CE00324D55B4653
:10F7C0002146179A059800F04DF805441CE004986E
:10F7D000002807DBDDE90301884203DD0098405C77
:10F7E000179901E0179930205A469047049805F17F
:10F7F0000105401C04900198401E019004D12E2068
:10F800005A46179990476D1CBAF10001AAF1010AF6
:10F81000DDDC05E017F8010B5A46179990476D1C7F
:10F82000B8F10001A8F10108F4DC5B462146179A03
:10F830000598ABE62D0000002B0000002000000022
:10F840002DE9F041044600251E461746880404D4DD
:10F8500005E039462020B0476D1C641EF9D52846C6
:10F86000BDE8F0812DE9F041044600251E46904692
:10F87000C80301D5302700E02027880404D505E01F
:10F8800041463846B0476D1C641EF9D52846BDE890
:10F89000F0810A68531C0B601070704710B5044665
:10F8A00002F07EF900B110BD0748084909684454C8
:10F8B00006480068401C052190FBF1F201FB120094
:10F8C0000249086000BFEEE7C0080020BC08002025
:10F8D00010B58CB001F0DEF926E09DF80C3004AADA
:10F8E00007A80699FAF7BFFB00208DF82F0001202A
:10F8F000244908700B98009007A80FC800F0E4F99D
:10F9000001280FD1142207A91F48F8F73DFC1D4814
:10F910000021CDE901101C48006900901A480FC869
:10F9200000F06EF9FCF7ECFD1848406840B117484C
:10F9300003AB04AA06A944680020A0470128CCD044
:10F9400011E09DF80C3004AA07A80699FAF78BFB82
:10F9500000208DF82F000B98009007A80FC800F02A
:10F9600027F9FCF7CDFD0948C06940B1074803AB52
:10F9700004AA06A9C4690120A0470128E1D00CB05F
:10F9800010BD00004C02002020150020D0140020E3
:10F9900010B520211A48F8F710FC30211948F8F763
:10F9A0000CFC01F071F9FCF7B7FDFCF7E1FD154A1D
:10F9B00015490020FCF772FE10B114A0FFF7DCFA25
:10F9C000104A183217490120FCF768FE10B116A042
:10F9D000FFF7D2FA0B48C06830B10A4800231A4634
:10F9E0001946C4681846A0470648406A30B1054821
:10F9F00000231A461946446A0120A04710BD0000A2
:10FA000000150020D01400201402002063616E3124
:10FA100020D0ADD2E9B3F5CABCBBAFB3C9B9A60D0E
:10FA20000A000000E001002063616E3220D0ADD2F8
:10FA3000E9B3F5CABCBBAFB3C9B9A60D0A00000053
:10FA400010B5A2B0002441F20B000D49A1F8050049
:10FA500000BF01E0601C84B2282CFBDB5020084969
:10FA600048800848007C401C0649087406A0FFF73F
:10FA700083FA01AA02A90248FBF7C2FC22B010BD1A
:10FA80002A1E0020B01F002053656E642063656C41
:10FA90006C2074656D70200A0D00000010B5A2B0D6
:10FAA000002441F20C001049A1F8050000BF06E057
:10FAB0000E48015D0C48C01D0155601C84B2082C25
:10FAC000F6DB0820084948800948007C401C0849AA
:10FAD000087408A0FFF750FA01AA02A90248FBF730
:10FAE0008FFC22B010BD00002A1E002079220020C9
:10FAF000B01F002073656E6420626D735F73746164
:10FB000074655F696E666F0A0D00000010B5A2B0E3
:10FB1000002441F20A001149A1F8050000BF09E0E4
:10FB200004EB44010E48084481780C48C01D01557F
:10FB3000601C84B2282CF3DB28200849488009483F
:10FB4000007C401C0749087407A0FFF715FA01AABA
:10FB500002A90248FBF754FC22B010BD2A1E002067
:10FB600001220020B01F002053656E642063656C85
:10FB70006C2074656D70200A0D00000070B505469C
:10FB8000002400BF0FE0094951F83410286888426A
:10FB900007D1064800EBC40041682846884700208A
:10FBA0002860601C44B20C2CEDD370BD64060020AC
:10FBB0000FB410B5142202A90D48F8F7E5FA0C4865
:10FBC0000468142201460B48F8F7DEFA80210A483F
:10FBD000FBF77FFF0948016805488847142104485E
:10FBE000F8F7EBFA00200249086010BC5DF814FB3E
:10FBF000540F0020180F0020001001406006002064
:10FC00000FB470B5DDE9095429484078142810DA9A
:10FC10002749497801EB81022549091D01EB820042
:10FC2000142204A9F8F7B0FA21484078401C204972
:10FC3000487005986FF30F001E49884218D19DF84F
:10FC40001B00102803D09DF81B00132804D19DF839
:10FC50001E001949087007E09DF81B00112803D108
:10FC60009DF81C00144908700A201449086015E02A
:10FC700005986FF30F00124988420FD19DF81B00C1
:10FC80000D490978884206D114200C4908600020EB
:10FC90000949087002E0322008490860002109483B
:10FCA000FEF728F90020207070BC5DF814FB0000FE
:10FCB0004C0D00200000EC1CFC000020E4000020A3
:10FCC0000000EB1CE00000200FB410B5142202A9C4
:10FCD0003848F8F759FA37484068374908603548D6
:10FCE000808880B24FF25641884204D04FF0FF30F6
:10FCF00010BC5DF814FB2F4840686FF30F002F49CC
:10FD0000884207D114222B492D48F8F73DFA4FF0CD
:10FD1000FF30EDE7274840686FF30F00294988421C
:10FD200007D1142223492648F8F72EFA4FF0FF3066
:10FD3000DEE721480068244988422CD01E4800682C
:10FD40002249884227D01C4800682149884222D095
:10FD5000194800681F4988421DD0174800681E498D
:10FD6000884218D0144800681C49884213D01248B1
:10FD700000681B4988420ED00F4800681949884224
:10FD800009D00D4800681849884204D00A48006824
:10FD9000164988420BD1142206491548F8F7F4F9A0
:10FDA00004498A7A002348680B3100F033FC0020B4
:10FDB0009EE70000400F0020F80000200000EC1C2F
:10FDC000FC0C00200000EB1C56F4261856F4011819
:10FDD00056F4071856F4081856F40A1056F4121878
:10FDE00056F41D1856F41F0856F41A1056F41A1833
:10FDF000380D002070B50020134908601348486092
:10FE0000042008720020487205208872FF22082111
:10FE10000D480B30F8F7CAF90D48B0F84140B0F87A
:10FE20004300C0F57A6085B20749CC72210A0648C2
:10FE300001734573290A8173054890F845100248FB
:10FE4000C17301F043F870BD100D0020F456101876
:10FE5000FC07002070B50446012C25D100204A493A
:10FE600008604A4848600420087200204872082050
:10FE70008872FF22082144480B30F8F797F91020C8
:10FE80004149C8720D21404801730021417302218C
:10FE90008173FF21C1730021017406214174002187
:10FEA000817401F013F86EE0022C6CD10020364909
:10FEB0000860374848600420087200204872082013
:10FEC0008872FF22082130480B30F8F76FF90120C3
:10FED0002D49C8722F4890F833102B4801732D48D4
:10FEE000B0F83300010A284841732A48B0F83500B9
:10FEF000C0F57A60C1B2244881732648B0F8350055
:10FF0000C0F57A60010A2048C173224890F8371082
:10FF10001D4801741F48B0F83700010A1A4841749F
:10FF20001C4890F839101848817400F0CFFF032066
:10FF3000FBF7C7FA02201449C8721648B0F8390016
:10FF4000010A11480173134890F83B100E484173A1
:10FF50001048808F00EB80004FF6FF7101EA4005EA
:10FF600009488573290AC1730A4890F83E1006486B
:10FF700001740848C08F010A03484174002181744C
:10FF800000F0A4FF00BF70BD100D0020F456EC1C63
:10FF9000F456EB1CFC07002010B50446012C25D1BB
:10FFA0000020564908605648486004200872002026
:10FFB000487208208872FF22082150480B30F8F759
:10FFC000F5F810204D49C87209214C4801730021F1
:10FFD000417302218173FF21C1730021017411213A
:10FFE00041740021817400F071FF86E0022CFCD185
:10FFF00000204249086043484860042008720020FD
:020000040801F1
:10000000487208208872FF2208213C480B30F8F71C
:10001000CDF801203949C8723B48B0F81B00B0F553
:10002000FA6F0EDD3848B0F81B003849B1F85910A6
:10003000884206DA3448B0F81B003549A1F80500BB
:1000400004E04FF47A603249A1F805003148008895
:10005000643880B240F480502D49A1F80900084668
:100060004179264801732A48B0F80500010A23485F
:1000700041732748B0F80700C0F57A60C1B21F4845
:1000800081732348B0F80700C0F57A60010A1B4865
:10009000C173214890F84A10184801741E48B0F8FE
:1000A0004A00010A154841741B4890F8661013482D
:1000B000817400F00BFF0320FBF703FA164890F859
:1000C0006600C0F1640081B21348A0F84D10022010
:1000D0000A49C872104890F84D10084801730E483C
:1000E000B0F84D00010A0548417300218173C173C6
:1000F00001744174817400F0E9FE10BD100D002000
:10010000F456EC1CF456EB1C6C0C0020441500203B
:10011000E60C0020D90C0020FC07002010B5044696
:1001200000200C4908600C48486004200872002038
:10013000487202208872FF22082106480B30F8F727
:1001400035F80449CC72210A0248017300F0BEFE62
:1001500010BD0000100D0020F456271810B586B011
:100160000446142101A8F8F728F8012C25D1002015
:100170009249086092484860042008720020487242
:1001800008208872FF2208218C480B30F8F70EF8FF
:1001900010208A49C87231218848017300214173B7
:1001A00007218173FF21C173002101740221417471
:1001B0000021817400F08AFEFEE0022CFCD10020B8
:1001C0007E4908607F484860042008720020487219
:1001D00008208872FF22082178480B30F7F7E6FFE5
:1001E00001207649C87200BF77488078087300BF45
:1001F0007548C078487300BF73480079887300BFA2
:1002000071484079C87300BF6F488079C1B26B48AC
:10021000017400BF6C48C088010A6848417400BF7F
:100220006948007AC1B26548817400F04FFE03202E
:10023000FBF747F902206149C87200BF6248008994
:10024000010A5E4801736048817A5C4841735E48E8
:10025000C17A5A4881735C48017B5848C1735A4837
:10026000417B5648017400214174817400F02EFED8
:100270000320FBF726F903205049C87201214F489B
:100280000173022141735048817C4C4881734E4870
:10029000C17C4A48C1734C48017D484801744A48B2
:1002A000417D464841744848817D4448817400F04E
:1002B0000DFE0320FBF705F90020444981F8870172
:1002C000084690F88701012806D112223E491A31CA
:1002D00001A8F7F759FF04E0FF22112101A8F7F761
:1002E00065FF04203549C8723748C17D3348017322
:1002F0003548017E31484173002181739DF8041017
:10030000C1739DF8051001749DF8061041749DF8A5
:100310000710817400F0DAFD0320FBF7D2F8052006
:100320002649C8729DF80810244801739DF80910E9
:1003300041739DF80A1081739DF80B10C1739DF8ED
:100340000C1001749DF80D1041749DF80E1081740D
:1003500000F0BCFD0320FBF7B4F806201749C87273
:100360009DF80F10154801739DF8101041739DF80A
:10037000111081739DF81210C1739DF81310017450
:100380009DF8141041741021817400F09FFD03202A
:10039000FBF797F807200949C8720A21074801733B
:1003A0000B21417307218173E021C173FF21017487
:1003B0004174817400F08AFD06B010BD100D00205C
:1003C000F456EC1CF456EB1CFC07002044150020EE
:1003D00010B5044600200A4908600A484860042015
:1003E00008720020487201208872FF220821044808
:1003F0000B30F7F7DBFE0248C47200F067FD10BD5A
:10040000100D0020F456091010B5044600202849AC
:1004100008602848486004200872002048720720BD
:100420008872FF22082122480B30F7F7BFFE4B20CD
:10043000214908804A2021490880214890F89701E5
:10044000012820D11F48C07A1949C8721E48017876
:10045000174801731C4800880112154841731B4856
:100460000178134881731948008801121048C1733C
:10047000124801780E4801740F4801780C48417405
:1004800000F024FD12E00F48C07A0949C8724C21DF
:100490000748017304214173B02181730421C173A2
:1004A000642101746521417400F010FD10BD00004D
:1004B000100D0020F4561C180C0100200E01002025
:1004C00044150020E60C00200A010020080100204D
:1004D0002DE9F04781460024002500260027A0468C
:1004E00000201A4908601A48486004200872002059
:1004F000487207208872FF22082114480B30F7F752
:1005000055FE144890F89701012806D105244B2583
:1005100004264A274FF0030805E005244B2504264E
:100520004A274FF003080948C4720573467387735E
:1005300080F80F80002101740748007C0007010E3D
:100540000248417400F0C2FCBDE8F087100D0020A5
:10055000F456131844150020E60C00202DE9F04154
:10056000074600240025002600202549086025486C
:100570004860042008720020487204208872FF221C
:1005800008211F480B30F7F711FE1F48C07A642876
:1005900003D01E4800781C2802D144F0010400E07A
:1005A00000BF1A4800781E2802D144F0100400E071
:1005B00000BF16480078032802D144F0400400E050
:1005C00000BF12480078182802D145F4806500E089
:1005D00000BF0D48B0F807000D49B1F885108842FA
:1005E00002DB46F0010600E000BF0548C472057357
:1005F000290A4173867300F069FCBDE8F0810000B0
:10060000100D0020F4561910E60C00207002002096
:10061000441500202DE9F04105460E461746984640
:100620000024FAF721FD5649681A8D424CD015DC9A
:100630005449A5EB01008D4273D008DC5248284490
:1006400000286CD051490844002869D14AE050493B
:100650000844E8B1B0F5C02FF7D127E0B0F5202F5E
:100660004ED0B0F5901F5DD0B0F5A81F68D0B0F5A2
:10067000F01FEAD1424639463046FAF73BFB0446C2
:100680002CB14448806B40F480404249886374E058
:10069000424639463046FAF771FB04462CB13D48D4
:1006A000806B40F001003B49886366E04246394672
:1006B0003046FAF7B3FB04462CB13648806B40F065
:1006C00002003449886358E0424639463046FAF71A
:1006D00021FB04462CB12F48806B40F004002D49CB
:1006E00088634AE0424639463046FAF765FB0446DD
:1006F0002CB12848806B40F00800264988633CE014
:10070000424639463046FAF7A3FA04462CB121484E
:10071000806B40F010001F4988632EE001E01DE06F
:100720002AE000BF424639463046FAF763FB0446EA
:100730002CB11848806B40F02000164988631CE0FB
:10074000424639463046FAF741FB04462CB111487F
:10075000806B40F040000F4988630EE04246394606
:100760003046FAF7B3FA04462CB10A48806B40F0E1
:1007700080000849886300E000BF00BFBDE8F08149
:1007800056F4081856F41A10AA0BE0F7000015F8F2
:10079000000019F86C0C0020F0B5034698180F4FB4
:1007A000B84201D90320F0BD0AB90020FBE70126B9
:1007B00000240BE01D780878A84204D0FF2D01D05A
:1007C0000220F0E700265B1C491C641C9442F1D314
:1007D000012E01D10020E6E70120E4E70000020835
:1007E00001460020C80AC002704700002DE9F84FFA
:1007F00006460F4614464FF0040B30192A4988422A
:1008000002D90120BDE8F88F0CB90020FAE704F006
:10081000010000B1641C224639463046FFF7BCFF98
:100820008046B8F1000F01D10020EBE7012080F3F2
:10083000108800BFFAF794FF3520FAF7E7FE30463C
:10084000FFF7CEFF0090FAF7E7FE83464FF47A7A7F
:1008500000BFBAF10000AAF101011FFA81FAF8D134
:10086000002511E017F815906800401C385C49EA33
:10087000002949463046FAF719FF8346BBF1040FB9
:1008800000D004E0B61C6D1CB5EB540FEAD300BFDA
:10089000FAF702FF002080F3108800BFBBF1040FBD
:1008A00000D1AFE70220ADE70000020810B5044612
:1008B0003CB900210748F9F79BFF0648F9F790FB80
:1008C00006E000210448F9F793FF0348F9F788FB95
:1008D000012010BD006400400068004070B505466E
:1008E0000C46022D00DB70BD05EB85000D4901EBC8
:1008F0008000006988B1A37A207A042801D1606859
:1009000000E02068014605EB8500064A02EB800006
:1009100004F10B0206692846B047284600F060F94A
:1009200000BFE0E7680F002070B505460E460DB920
:10093000064900E0064908463146FAF73DF8044604
:10094000042C00D1FF24204670BD0000006400404C
:100950000068004070B504460D461646022C00DBC8
:1009600070BD04EBC400144901EB8000C068012194
:10097000A9400840F0B104EBC4000F4901EB80002E
:10098000C0680121A940884304EBC4010A4A02EB74
:100990008101C860204600F023F904EB8400074978
:1009A00051F8200030B104EB840051F82020294692
:1009B0002046904700BFD3E7900F0020680F00202B
:1009C00070B504460D4614B9F9F756FE01E0F9F783
:1009D00063F9012070BD000010B50446832C00D0DF
:1009E00010BD0A48007C01280ED00948C06A18B121
:1009F0000748C16A01208847012004490874002182
:100A000002481430FDF776FA00BFE9E70015002030
:100A1000D01400202DE9F04105460E4626BB2F4696
:100A200000240FE0124800EB04100068B84207D120
:100A30000F4901EB041101F10C000021FDF75AFAF6
:100A4000601C84B2092CEDD300BF0A48807F0028C7
:100A50000BDD0848007C022807D10021054881777A
:100A60001830FDF747FA00E000BFBDE8F081000054
:100A7000500100200015002010B50446002004EBB2
:100A8000C401044A02EB810188602046FFF70EFF93
:100A900010BD0000900F002010B50446022C00DBB2
:100AA00010BD04EB84000D4901EB8000806890B11B
:100AB00004EBC4000A4B03EB8000C06808B10120BE
:100AC00000E00020014604EB8400044B03EB8000AF
:100AD00082682046904700BFE2E70000680F0020D0
:100AE000900F002010B50446022C00DB10BDFCF76F
:100AF00010FF04EB84000F4901EB8000C06838B19F
:100B000004EB84000A4602EB8000C1682046884757
:100B1000FCF701FF04EBC400074901EB8000C0684B
:100B200030B1002004EBC401034A02EB8101C8602C
:100B300000BFDBE7680F0020900F00202DE9F04197
:100B400004460D4616461F46022C02DB0020BDE877
:100B5000F081012004EBC401204A02EB810188608E
:100B6000002004EBC40102EB8101487104EBC400D6
:100B7000114601EB8000077104EBC40001EB80001B
:100B8000C67004EBC40021F82050002004EBC4011F
:100B900002EB8101C86004EBC40002EB8001204637
:100BA000FFF70EFF38B1022004EBC4010B4A02EB41
:100BB0008101886006E0002004EBC401074A02EBD3
:100BC0008101886004EBC400044901EB8000806867
:100BD000022801D10120BAE70020B8E7900F0020D9
:100BE000022800DB704700BFFCE700002DE9F04160
:100BF00004460E4617469846022C07DA04EBC4005A
:100C0000194901EB80008068022802D00020BDE86D
:100C1000F08104EBC401144A02EB810101F11000E0
:100C200043463A463146F9F7F7F904EBC4000E4A59
:100C300002EB800000F110012046FFF775FE05462B
:100C4000FF2D0ED004EBC400074901EB8000C16802
:100C50000120A840014304EBC400034A02EB8000DA
:100C6000C1602846D3E70000900F0020FEB504467F
:100C70000D4616460094019502966946014803F018
:100C800012FBFEBD5812002010B500F0A9F800F0CC
:100C900047F810BD10B500F055F800F0ABF810BDE6
:100CA00010B502460B4612B94FF0FF3010BD0021BF
:100CB00014E01A4850F8310090420ED1174800EB6A
:100CC000C1004360154800EBC100406818B900201E
:100CD000124C44F831000020E8E7491C1429E8D3FD
:100CE00013B94FF0FF30E1E7002111E00B4850F855
:100CF000310020B1094800EBC100406838B907480D
:100D000040F8312000EBC10043600020CEE7491CD1
:100D10001429EBD34FF0FF30C8E70000D80F0020B4
:100D200010B54FF426710648F7F747FA28230C222E
:100D30000349A03101F5F07003F08AFA002010BDDC
:100D4000D80F00203EB518E069460F4803F08EFA30
:100D500000240FE00D4850F834000099884208D173
:100D60000A4800EBC400456815B19DE80700A84794
:100D700002E0641C142CEDD300BF034803F056FAC4
:100D80000028E1D000203EBD58120020D80F0020DE
:100D900010B502460AB9002010BD002119E001EB90
:100DA00041000E4B03EB8000806880B901EB4100ED
:100DB00003EB80008260002001EB4103074C44F804
:100DC000230001EB4100234603EB8000E4E7481CCD
:100DD00081B21429E3D30020DEE700007012002066
:100DE00010B5F0210248F7F7E8F9002010BD000027
:100DF00070120020F8B5002700216846FDF77AF848
:100E00000098B84203D0781C0099814201D100209B
:100E1000F8BD009F00243BE004EB44001E4901EBB9
:100E20008000866804EB440051F820507DB376B30F
:100E300004EB4401184A02EB8101081D2946FDF725
:100E400059F8012823D104EB4400134901EB800039
:100E50008068A8B104EB440001EB80004068009971
:100E6000081AB0FBF5F004EB44010B4A02EB8101D8
:100E7000496800FB051004EB440102EB8101486066
:100E80002EB104EB4401044A02EB8100B047641C1C
:100E9000142CC1D30020BBE77012002070B50446AB
:100EA0000E46254605B970BD2E600021281DFDF7B0
:100EB00021F800BFF7E701460A460AB9002070474B
:100EC000106808B10120FAE70020F8E77CB5044675
:100ED000002611480068E0B10021207A042801D1E1
:100EE000606800E02068CDE90001607A08B9A07A66
:100EF00000E000200346207A042801D1606800E069
:100F000020680146044804F10B0205680020A84748
:100F10007CBD0020FCE70000D01400207CB5044616
:100F2000002612488069F0B10021207A042801D1FE
:100F3000606800E02068CDE90001607A08B9A07A15
:100F400000E000200346207A042801D1606800E018
:100F500020680146054804F10B0285690120A84775
:100F600008B100207CBD0020FCE70000D014002068
:100F700010B50A48008840B9012008490880F7F7F1
:100F8000A1FD07A0FDF7F8FF07E000200349088056
:100F9000F7F7A2FD07A0FDF7EFFF10BDAA0500209F
:100FA000B9D8B1D5BDBBC1F7BCCCB5E7C6F70D0A02
:100FB00000000000BFAAC6F4BDBBC1F7BCCCB5E7BA
:100FC000C6F70D0A000000007047704710B50A48C8
:100FD000008840B9012008490880FAF7D7F907A02E
:100FE000FDF7CAFF07E0002003490880FAF7D6F9A9
:100FF00007A0FDF7C1FF10BDA8050020B9D8B1D5E5
:10100000D6B1C1F7BCCCB5E7C6F70D0A00000000A9
:10101000BFAAC6F4D6B1C1F7BCCCB5E7C6F70D0A76
:101020000000000070477047704770477047704776
:1010300070472DE9F04705460E460D20FDF754F8A0
:101040000A20FDF751F82C46002710E02078FBF726
:101050009EF880462078FBF78DF881464046FDF7E4
:1010600043F84846FDF740F8641C781C87B2B74245
:10107000ECDB0D20FDF738F80A20FDF735F8BDE868
:10108000F0870022002107E042F6E06200E0521EF5
:10109000002AFCD14B1C99B28142F5DB704700005D
:1010A00070B504460D46E1B21948FDF742FB00BF9A
:1010B0001748008800F080000028F9D0154890F803
:1010C000A800012822D11448807802281AD1134898
:1010D0000078962808DA114802780078401C0F4BF7
:1010E00018700F48845411E00C4801780C48FDF743
:1010F0000FFE0948007C401C07490874002007497E
:10110000087003E00020034981F8A800204670BD64
:10111000004C004044150020B01F00209E05002018
:101120008122002010B5002821D0114B0022001F81
:10113000196803E0814203D80A4649680029F9D1B9
:1011400052B11368841A9C4204D10068184410609C
:10115000104602E0506000E0186039B102680B1AD6
:10116000934203D10B681A4402604968416010BD84
:10117000980B002010B50D4A906E926E91698847C9
:101180000446022C01D0032C01D1002010BD41F2F5
:1011900088310748FCF7AEFE012805D1002104483C
:1011A000FCF7A8FE0120F1E70020EFE7FC07002094
:1011B0005024002010B5134890F8380000F00100CA
:1011C00040B111484079012804D110A0FDF7D4FEA8
:1011D000012010BD0B4890F8380000F0010038B134
:1011E0000220094948710FA0FDF7C6FE0120F0E773
:1011F000124908698047022801D00220E9E700204F
:10120000E7E700006C0C0020F4230020424D535F00
:1012100050524F544F43414C5F4742323031350AB0
:101220000D000000424D535F50524F544F43414C0C
:101230005F4742323031310A0D0000006400002067
:101240000348807B012800D170470020FCE70000A4
:10125000F423002010B50E49086980470446022C8B
:101260000DD1FDF781FD50B120210A48F6F7A5FF09
:10127000FAF734F908A0FDF77FFE012010BD012C1C
:1012800004D10AA0FDF778FE0220F7E70020F5E779
:101290006400002004240020BDF8C8EBD6B1C1F7DB
:1012A000B3E4B5E7C1F7B3CC0D0A0000BDF8C8EB55
:1012B000BDBBC1F7B3E4B5E7C1F7B3CC0D0A00007D
:1012C00010B50F48C078AA2804D10EA0FDF754FE2F
:1012D000012010BDFCF7E0F920B911A0FDF74CFE8C
:1012E0000220F6E71C48816980680A30814204D3F5
:1012F0001AA0FDF741FE0320EBE70020E9E700001C
:101300006C0C002052455620445F43445A5F4841CC
:101310004E44494E475F43524D2041410A0D000063
:1013200052656164792D53746174652052656365FB
:101330006976656420546865204368617267696EE8
:10134000672050696C652041626F7274204D65732F
:10135000736167650A0D0000042400205245414472
:10136000592054494D45204F55540A0D00000000A6
:1013700010B5FCF70DFC08B9012010BDFCF78CF985
:1013800020B906A0FDF7F8FD0320F6E7F9F7DAFF2C
:1013900008B90320F1E70020EFE7000052756E6EF8
:1013A000696E672D53746174652052656365697653
:1013B000656420546865204368617267696E6720C0
:1013C00050696C652041626F7274204D6573736162
:1013D00067650A0D0000000010B5FCF75DF920B943
:1013E00015A0FDF7C9FD022010BDF7F7C9FE20B911
:1013F0001FA0FDF7C1FD0320F6E7FDF7A5FC20B90E
:1014000026A0FDF7B9FD0420EEE72B48807EAA2830
:1014100004D12AA0FDF7B0FD0120E5E72E48C169FF
:10142000C0680A30814204D32CA0FDF7A5FD052039
:10143000DAE70020D8E7000053746172742D53740A
:1014400061746520526563656976656420546865DA
:10145000204368617267696E672050696C6520413E
:10146000626F7274204D6573736167650A0D0000C9
:10147000424D5320446F6573204E6F74204D656557
:101480007420546865204368617267696E67204301
:101490006F6E646974696F6E730A0D00424D53205C
:1014A000557070657220566F6C7461676520466177
:1014B000696C7572650A0D006C0C002043445A5F1C
:1014C0005F43524F20414120746F2043686172672F
:1014D000696E670A0D000000042400205354415235
:1014E000542054494D45204F55540A0D000000002A
:1014F0001CB50A216846FCF710FA20B16846FCF7D3
:101500001FFA01201CBD0020FCE770B504460D4603
:10151000002629462046F7F7DBFC0520FFF7B1FD42
:10152000FCF778F90646304670BD01460720704743
:10153000704701460220704710B5FCF707F91349C0
:1015400048611348008F00F4804078B100201049B2
:10155000886301200F49487100BF0F480088044686
:10156000FEF7DCFD0DA0FDF707FD0EE04FF4FA617C
:1015700008480830FCF7BEFC38B10DA0FDF7FCFCB4
:10158000002104480830FCF7B5FC10BD04240020FD
:101590006C0C0020F4230020FC070020445F43442F
:1015A0005A5F48414E44494E475F43484D0D0A003B
:1015B0004E4F2048616E647368616B6520536967A4
:1015C0006E616C0A0D0000000146002070477047F4
:1015D0000146012070477047014603207047000014
:1015E00010B5FCF7B3F80C4988610C48007920B1BC
:1015F000012807D002280DD108E002210848FAF797
:1016000017F907E00648FAF745F903E00220FAF770
:1016100051F900BF00BF10BD04240020F4230020B6
:101620005D01010801460520704710B5F9F7D0FDAE
:1016300010BD01460420704770B5FCF787F82F49AC
:10164000C8612F48007920B1012807D002280DD1A8
:1016500008E006212B48FAF7EBF807E02948FAF7EB
:1016600019F903E00620FAF725F900BF00BF0026AC
:1016700005212548FCF751F908B1AA2600E000260B
:1016800035462C46214890F8380000F0020030B171
:101690001E48806B20F002001C4988632CE01B4828
:1016A00090F8380000F00400B8B134B91848FBF7DE
:1016B0005BF91848FBF758F905E01548FBF77FF987
:1016C0001448FBF77CF92046FEF782FE0F48806B3A
:1016D00020F004000D4988630EE00C4890F83800B3
:1016E00000F0080040B10CA0FDF746FC0748806BF5
:1016F00020F008000549886370BD00000424002024
:10170000F423002055FE00088C2400206C0C0020DF
:10171000380A00204C0A002043445A5F48414E4496
:10172000494E475F43524D2041410A0D00000000E1
:10173000014606207047000010B500200F4948718F
:1017400032210F48FCF7D6FB012806D10020FEF716
:1017500005FF00210A48FCF7CDFBFA2108481030AC
:10176000FCF7C8FB012807D10020FEF74DFE002141
:1017700003481030FCF7BEFB10BD0000F42300202E
:101780003C24002070B505460E463046FAF7DEF9D7
:10179000044604B970BD812D26D004DC042D07D089
:1017A000802D4DD116E0822D0AD0832D48D128E01E
:1017B00094F85400032802DB2046FAF71BFD40E0B2
:1017C00094F85400032804DBE06C10B18220E16C33
:1017D000884736E094F85400032804DBE06C10B12D
:1017E0008020E16C88472CE094F85400032807DB44
:1017F0002046FAF79FFDE06C10B18120E16C88472C
:101800001FE094F85400032819DB9120005D0228A2
:1018100006D104219120015522780120FFF726FAF4
:10182000E06C18B18320E16C884708E0207800F074
:10183000E7FA207800231A46194600F053FB00E02F
:1018400000BF00BF00BFA5E770B506460D46304695
:10185000FAF77CF904461CB394F85400022805DC1E
:10186000E068E8B13046E168884719E094F8540030
:10187000812808D13DB184F85400324681210120ED
:10188000FFF7F4F90CE094F85400812808D03DB932
:10189000802084F85400324680210120FFF7E6F9C9
:1018A00070BD70B504460D4629462046FFF7CCFFB3
:1018B00070BD70B505462846FAF748F904468CB164
:1018C00094F85400022805DCE06858B12846E16825
:1018D000884707E0832084F854002A4683210120AA
:1018E000FFF7C4F970BD00002DE9F04107460D4631
:1018F00090461E463846FAF729F90446002C39D09E
:1019000094F85400032835DB94F85400802802D161
:10191000032084F8540094F8400000F0010038B12E
:10192000A06C38B3324641462846A36C984721E064
:101930001248056006710079002809DD0F4800791A
:10194000082805DC0D4802794146401DF6F71CFCCD
:101950000A4904F1580002F0A6FC04F1580002F014
:101960006EFC38B1822084F854003A46822101206E
:10197000FFF77CF90120BDE8F0810000C0140020D1
:1019800070B506460C463046FAF7E0F805461DB13C
:10199000E1B22846FAF7E7FC70BD000010B514204C
:1019A0006E4981F8660041F2883008800120887015
:1019B00001216A48C1700171032141714FF47A71AC
:1019C000C18041F268010181422181725921C172B5
:1019D000442101735421417300218173C17301219A
:1019E000017402214174192181740B21C1740A21EF
:1019F00001750021417581751021C17500210176A5
:101A00004176112256A11A30F6F7BEFB53482B300F
:101A100058A10A680260496841604FF4D2704F498A
:101A2000A1F833004FF47A714C48A0F835104FF408
:101A30009B71A0F8371041F22431A0F839106E21C3
:101A400080F83B10142181874FF47A61C187002010
:101A5000424981F840004FF47A60A1F841004FF408
:101A600016713E48A0F84310022180F8451000206E
:101A70003A49A1F8460000213848A0F84810B0F8CB
:101A80004A006FF30B0000F5A2703449A1F84A0038
:101A9000084690F84B0020F0F00110312F4880F8F4
:101AA0004B103C21A0F84D1001202C4981F84F002B
:101AB0006FF0310232490A20FDF768F9C1B22748B8
:101AC00080F85010032180F851106FF031022C493A
:101AD0000520FDF75BF9C1B2204880F852100421BF
:101AE00080F85310002180F8541080F8551080F8C9
:101AF000561080F8571080F8581080F8591080F868
:101B00005A100120154981F85B0000211348A0F804
:101B10005C1080F85E106420104981F85F0040F28C
:101B200059110E48A0F8601040F26311A0F862103D
:101B30006FF0310212491920FDF728F9C1B20748A8
:101B400080F864106FF031020D491C20FDF71EF97A
:101B5000C1B2024880F8651010BD0000FC070020EB
:101B60004C4656324132314B3641333039323339BB
:101B7000390000005330303148303031000000006F
:101B8000CDCCCC3D0448006804490968884201D1A5
:101B9000012070470020FCE7B8080020BC080020A6
:101BA00007480068401C052190FBF1F201FB120080
:101BB00004490968884201D1012070470020FCE7F0
:101BC000BC080020B808002070B504460D4618482F
:101BD0000078B0B929462046FFF797FC15490968F7
:101BE000084414490860144801780078401C124ADF
:101BF0001070092902DB01200D4908700F48008888
:101C000070BD00200A4908700A4800680C49086045
:101C100000200849086008490870094800680A213E
:101C2000B0FBF1F00549088008460088E8E70000AD
:101C3000D5000020CC000020D4000020C8000020E7
:101C4000D000002086B0FCF739F84FF400410803BB
:101C5000FAF7A6FFFBF7F0FF01A8FBF725FCFAF760
:101C600056FFFAF7ABFC40F2CF2140F2F310FCF73D
:101C700095F8F7F777F9F7F74FF94FF47A3002F064
:101C80003FFB4FF4E13002F095FBFFF787FEFDF7D5
:101C90007FFEFBF765FDF9F7F5F9012032498873FE
:101CA00061E0FCF77DF9FDF713FE3048007801286C
:101CB00013D100202D490870F7F7FAF9F7F75EFC09
:101CC0002B49086880472A4948688047284988681E
:101CD00080472749C868804745E024484078012864
:101CE00005D1002021494870FAF70AFC3BE01F4863
:101CF0008078012808D100201C4988700220F9F75B
:101D00004BFF1C49C8602EE01848C078012803D159
:101D100000201649C87026E014480079012805D132
:101D2000002012490871FAF787FE1CE00F4840793D
:101D3000012803D100200D49487114E00B48C079F7
:101D4000012810D100200949C8710B48FAF70CFE90
:101D5000F7F77AFCFBF710FAFBF7F8FC044621468C
:101D600006A0FDF709F99CE7F423002034150020B4
:101D700078000020CC0B0020280B00205254435F39
:101D8000476574436F756E746572206973202564AE
:101D90000D0A0000F0B50B30154D20F007010024AE
:101DA000144A0FE003688B420BD38B4205D95E1AAD
:101DB00043184768C3E9006700E04368136002C046
:101DC00004E0021D10680028ECD12046002802D152
:101DD000286808B10020F0BD064A07481060074A8D
:101DE000121A22F00702C0E9002401202860D7E778
:101DF0009C0B0020980B00209C240020984400207D
:101E000070B505462846F9F7A1FE04461CB194F8C2
:101E10005400022801DC002070BD022084F8540028
:101E2000E06810B12846E16888479120005D0028ED
:101E300034D0D4F8A800B0B19120005D052804D1B9
:101E40000021D4E92902904728E09120005D042870
:101E500004D10121D4E9290290471FE00321D4E9EC
:101E6000290290471AE0206DC0B19120005D05283D
:101E700005D10021226DD4F8A40090470EE09120F6
:101E8000005D042805D10121226DD4F8A4009047FB
:101E900004E00321226DD4F8A400904715E004F17A
:101EA000940104F1700002F0E1F970B1D4F8A800D7
:101EB00020B10321D4E92902904706E0206D20B12A
:101EC0000321226DD4F8A400904704F1700002F0C1
:101ED000ADF90028E3D0202104F19000F6F76DF968
:101EE000012099E72DE9F04105460E461746984630
:101EF0002846F9F72BFE04461CB194F8540001283B
:101F000002DC0020BDE8F081606848B343463A46F1
:101F100031462846D4F804C0E04708B3D4F88C0012
:101F200040B194F84530182204F17000D4F88C10B8
:101F300002F08EF994F8400000F0010058B9D4F88E
:101F4000880040B194F84530102204F15800D4F8CC
:101F5000881002F07DF9032084F854000120D1E7B5
:101F60000020CFE770B5054600242846F9F7EEFDBE
:101F7000044614B194F8540070BD0020FCE72DE92C
:101F8000FF4180460E4615461F464046F9F7DEFDE6
:101F900004464CB194F85400022805DD25B194F8AC
:101FA000400000F0010018B1002004B0BDE8F0814D
:101FB00004F1580002F03AF908B10020F5E769464B
:101FC00004F1580002F052F908B90020EDE700983A
:101FD00030609DF8040038709DF8040000280ADD88
:101FE0009DF80400082806DC9DF804200DF1050189
:101FF0002846F6F7C9F894F85400822802D1032045
:1020000084F854000120D0E72DE9F04786B08046DF
:102010000F4615461E46DDE90E9A00244046F9F7A4
:1020200095FD044654B194F85400022806DD082EAC
:1020300004DC04F1700002F002F918B1002006B0CF
:10204000BDE8F087FBF765FC94F85400832803D0C3
:1020500094F85400032803DAFBF75DFC0020EEE758
:10206000CDF814A000978DF80560CDF8109015B943
:1020700000208DF805009DF8050000280ADD9DF878
:102080000500082806DC9DF8052029460DF106000C
:10209000F6F77AF8FF208DF80400694604F1700025
:1020A00002F001F99120005D10B92046FAF7A2F87C
:1020B000FBF731FC0120C2E7034600207047000017
:1020C0002DE9F04F99B0834600201890402106A8D2
:1020D000F6F773F8002005904FF6FF7004905C4609
:1020E0000020F1490874B4F8050048F22001884244
:1020F00004D0B4F80500491C884243D1CDF80CB097
:10210000B4F802A0B4F8050002906088B0F5967F9C
:1021100004DC6288E11DE548F6F736F85146E348ED
:10212000FEF787FFAAF1020003990A5C401C085CD5
:1021300042EA00201690AAF1020081B20398F7F754
:1021400099F91790DAA0DDE91612FCF715FFDDE921
:102150001601884205D0DCA0FCF70EFF19B0BDE8DF
:10216000F08F0020D04948740299E031C8B252463D
:10217000CE49FCF7E3FA6420DB4908800420CA4911
:102180008870EBE7B4F80500B0F5004F5FD034DCA1
:10219000B0F5D06F01F0C38714DCB0F5607F72D06A
:1021A00009DC802854D0B0F5C07F79D0B0F5207F0D
:1021B00041F0E68783E0B0F5906F66D0B0F5B06F80
:1021C000F6D1AAE0B0F5286F01F0D2870CDCB0F5AB
:1021D000F06F01F0B787B0F5086F01F0B887B0F580
:1021E000186FE5D101F0B8BFB0F5025F01F0C58707
:1021F000B0F5065FDCD101F0C2BF48F20702811AD8
:10220000904201F09E870DDC6FF4004108440628DF
:1022100081F0B687DFE810F04300520061006600ED
:102220008000820F062901F09C8709DC012901F05A
:102230008D87022901F08F870329B9D101F090BF62
:10224000192901F099871A29B2D101F097BF00BF6F
:10225000E07901281ED194498870A44981F876005C
:1022600008460021C1660167A0F874100146A26803
:10227000CA66E068086701208B4988709C4908702D
:102280009A496C3102E029E00AE02CE099A0FCF7C1
:1022900073FE02E09FA0FCF76FFE01F072BF00BF6B
:1022A000E079012806D102207F4988709EA0FCF7C2
:1022B00063FE02E0A1A0FCF75FFEEEE700BFE1795C
:1022C000A2A0FCF759FEA649D4F809200A60B4F888
:1022D0000D208A80E07B8871DFE700BFA1A0FCF7BA
:1022E0004BFEDAE700BFA5A0FCF746FE207A0128E6
:1022F00001D1A8A000E0A9A00146AAA0FCF73CFEDD
:10230000207A40B90120AA490870AA48007810B97B
:102310000420A8490870C0E700BF0120A649087042
:10232000E07918B9A5A0FCF727FE02E0A7A0FCF70A
:1023300023FEE079012841F07786267A3146A7A06E
:10234000FCF71AFE012E14D1607A40B90120984999
:1023500008709848007810B9042096490870607A8F
:10236000012801D1A1A000E0A2A00146A3A0FCF792
:1023700003FE022E09D1607A012803D1A3A0FCF745
:10238000FBFD02E0A5A0FCF7F7FD042E1BD104F134
:102390000900F5F72FFF85B2102D0FD22A4604F160
:1023A000090152481030F5F7EFFE04F109019FA032
:1023B000FCF7E2FD01204E49087004E004F1090138
:1023C0009FA0FCF7D9FD072E0AD1657A2946A3A064
:1023D000FCF7D2FD4548A0F8695001204449087037
:1023E000062E0ED1657A2946A3A0FCF7C5FD3F480D
:1023F000A0F84D50A0F84F50A0F8515001203C4992
:102400000870082E03D1657A012039490870092E19
:102410001DD104F10900F5F7EDFE85B2102D0ED2A5
:102420002A4604F109013148F5F7AEFE04F109012D
:1024300097A0FCF7A1FD01202D49087004E004F1EC
:10244000090199A0FCF798FD0120294908700A2E7E
:1024500014D1657A012D07D10120244981F8870024
:1024600098A0FCF789FD06E00020204981F887004C
:1024700094A0FCF781FD01201D4908700B2E00D1AE
:10248000657A0C2E0FD1657A012D07D101201749ED
:1024900081F8890091A0FCF76FFD32E1002013491B
:1024A00081F889002AE12FE1B01F0020B62000202A
:1024B0000A0D44637263202530782C5663726320C2
:1024C0002530780A0D0000000A0D2028446372634D
:1024D00020213D2056637263292072657475726EE7
:1024E00021212121210A0D009C05002044150020F6
:1024F0006002002072656769737465726564207399
:1025000075636365737365642C436F64652025731D
:102510000A0D0000726567697374657265642066F0
:1025200061696C65640A0D004C6F67696E205375B4
:10253000636365737365640A0D0000004C6F67691F
:102540006E204661696C65640A0D00006865617201
:102550007420636F756E742025640A0D00000000FE
:10256000610C00207265636569766520737461741F
:10257000652064617461200A0D0000007265636566
:1025800069766520636861726765206461746120A3
:102590000A0D0000456E61626C650000446973615C
:1025A000626C65006368617267652025730A0D00BF
:1025B00099050020700200209A0500207061726168
:1025C0006D20726561640A0D000000007061726127
:1025D0006D2077726974650A0D0000007061726188
:1025E0006D20616464722025780A0D00656E616259
:1025F0006C65000064697361626C65006368617298
:1026000067696E672025730A0D000000636C6F73A5
:10261000652072656C61790A0D0000006F70656E4F
:102620002072656C61790A0D00000000626C7565AE
:10263000746F6F7468206E616D652025730A0D00DC
:10264000626C7565746F6F7468206E616D65206D66
:10265000697374616B652025730A0D0048656172AA
:102660007420426561742054696D652025642020C2
:102670007365630A0D0000004F76657254656D70D6
:1026800056616C75652025642020200A0D0000002D
:102690005379735061726150696C65442E736E3A60
:1026A00025730A0D00000000537973506172615068
:1026B000696C65442E736E206661756C7420257399
:1026C0000A0D0000517569636B204368617267658C
:1026D00020456E61626C650A0D00000074726963CA
:1026E0006B6C65204368617267696E6720536F6326
:1026F00020456E61626C6520310A0D00F3A0FCF785
:102700003BFC0120F94908700D2E14D1657A642D27
:1027100007DAF74981F88A502946F6A0FCF72CFC25
:1027200006E0FAA0FCF728FC5A20F14981F88A005B
:102730000120EE4908700E2E15D1657A0A2095FB0E
:10274000F0F100FB115001900A2095FBF0F0009091
:102750000146F4A0019AFCF70FFCE54880F88B5085
:102760000120E24908700F2E0ED1657A2946F3A0A8
:10277000FCF702FC05EB85004006000EDC4981F801
:102780008C000120D9490870102E37D1617AA07AC7
:1027900041EA00252946EFA0FCF7EEFBD448B0F84B
:1027A000590005EB8501B0EB410F0CDD05EB850011
:1027B0004FF6FF7101EA4000CD49A1F883000120E6
:1027C000CA4908701AE0CA48B0F8592005EB8500DC
:1027D0004100E4A0FCF7D0FBC548B0F8590014381C
:1027E000C349A1F883000846B0F883000A2190FB92
:1027F000F1F001460190E2A0FCF7BEFB112E25D1BD
:10280000617AA07A41EA00252946E2A0FCF7B4FBF0
:10281000B748B0F85B0005EB8501B0EB410F0CDD6C
:1028200005EB85004FF6FF7101EA4000B049A1F8C1
:1028300085000120AD49087008E0AD48B0F85B2084
:1028400005EB85004100D8A0FCF796FB122E13D1B2
:10285000617AA07A41EA00252946D9A0FCF78CFBD1
:1028600005EB85004FF6FF7101EA4000A049A1F891
:10287000590001209D490870132E13D1617AA07A66
:1028800041EA00252946D3A0FCF776FB05EB85003D
:102890004FF6FF7101EA40009549A1F85B00012065
:1028A00092490870142E19D1657A2946CEA0FCF7FA
:1028B00063FBD2488078202802DD2020CF49887031
:1028C000CE48807800EBC001CC48C01C00EB410032
:1028D0008580CA488078401CC8498870162E18D157
:1028E000617AA07A41EA00258148A0F863500A2065
:1028F00095FBF0F100FB115001900A2095FBF0F0E0
:1029000000900146BEA0019AFCF736FB01207749F2
:1029100008701D2E17D1657A012D01D0022D0FD11F
:10292000734981F88D50012D01D1BBA000E0BBA0FF
:102930000146BBA0FCF720FB01206C49087002E0B7
:10294000BCA0FCF719FB1E2E20D1657A05EB850093
:102950004FF6FF7101EA40006549A1F853000846AF
:10296000B0F853000A2190FBF1F201FB1200019034
:102970005F48B0F8530090FBF1F000900146B3A01F
:10298000019AFCF7F9FA0120584908701F2E50D11E
:10299000657A5748B0F890005549B1F8531088420D
:1029A00027DD5348B0F853000A2190FBF1F0019065
:1029B0004F48B0F8900090FBF1F000900146A9A0BC
:1029C000019AFCF7D9FA4A48B0F853000A38484946
:1029D000A1F890000846B0F890000A2190FBF1F0B1
:1029E00001460190AAA0FCF7C7FA01203F490870F0
:1029F0001FE005EB85004FF6FF7101EA40003C49FE
:102A0000A1F890000846B0F890000A2190FBF1F27E
:102A100001FB120001903648B0F8900090FBF1F0F5
:102A200000900146A0A0019AFCF7A6FA01202F49C8
:102A30000870202E1DD1657A05EB85004FF6FF71D9
:102A400001EA40002A49A1F8B3000846B0F8B300F3
:102A5000642190FBF1F201FB120001902448B0F8D0
:102A6000B30090FBF1F00090014696A0019AFCF7AC
:102A700083FA212E20D1657A05EB85004FF6FF7190
:102A800001EA40001A49A1F8B1000846B0F8B100C7
:102A9000642190FBF1F201FB120001901448B0F8A0
:102AA000B10090FBF1F0009001468DA0019AFCF777
:102AB00063FA01200D490870222E06D1657A0C4870
:102AC000A0F8B750B0F8B71018E11DE1747269634F
:102AD0006B6C65204368617267696E6720536F6332
:102AE00020456E61626C6520300A0D006002002096
:102AF00044150020747269636B6C6543686172678A
:102B0000696E67536F6325640A0D00007472696310
:102B10006B6C654368617267696E67536F632039D8
:102B2000300A0D00747269636B6C6520706F776595
:102B3000722025642E25646B770A0D007472696318
:102B40006B6C652063757272656E742564410A0D45
:102B500000000000426D734D6178566F6C742564FF
:102B6000200A0D00256420426D734D6178566F6C0C
:102B700074202564206661696C640A0D0000000001
:102B8000426D52657175697265566F6C742025646B
:102B9000200A0D00426D734D617843757272656E47
:102BA00074202564200A0D00726571202564206F51
:102BB000766572206D6178202564200A0D00000082
:102BC000426D734D6178566F6C74202564200A0D38
:102BD00000000000426D734D617843757272656E3E
:102BE000742564200A0D000073657474696E672093
:102BF000736F63282564290A0D000000A0170020C8
:102C0000754261744D6178456E65726779202564FF
:102C10002E25640A0D0000004343000043560000C7
:102C20004368617267696E674D6F64653A2573200A
:102C30000A0D00004368617267696E674D6F6465D5
:102C4000204661756C740A0D000000004F766572B5
:102C5000506F776572203A25642E25646B77680A79
:102C60000D00000052657175697265506F7765726D
:102C7000202564206B77204F766572506F776572E0
:102C8000203A25646B772C6661756C740A0D000020
:102C900052657175697265506F7765722025642081
:102CA0006B77200A0D0000005265717569726550DE
:102CB0006F776572203A25642E25646B77680A0D5C
:102CC000000000004261745261746564566F6C7458
:102CD000616765203A25642E2564560A0D000000C0
:102CE0004261744D6178436861726765566F6C200C
:102CF0003A25642E2564560A0D000000EDA0FCF76D
:102D00003BF90120EF490870232E1CD1617AA07A8B
:102D100041EA0025EC48A0F85F50B0F85F000A21B6
:102D200090FBF1F201FB12000190E748B0F85F0060
:102D300090FBF1F000900146E4A0019AFCF71CF929
:102D40000120E0490870242E1CD1617AA07A41EA62
:102D50000025DD48A0F85950B0F859000A2190FB31
:102D6000F1F201FB12000190D748B0F8590090FB36
:102D7000F1F000900146DCA0019AFCF7FDF801207B
:102D8000D0490870252E0CD1657A2946DBA0FCF7C6
:102D9000F3F805F13200CC4981F8B5000120C949AA
:102DA0000870262E0CD1657A2946DBA0FCF7E4F8E2
:102DB00005F13200C44981F8B6000120C14908700C
:102DC000272E33D1657AC04880F8B050012D02D14A
:102DD000D8A0FCF7D1F8022D02D1DCA0FCF7CCF88A
:102DE000032D02D1DFA0FCF7C7F8042D02D1E4A027
:102DF000FCF7C2F8052D02D1E7A0FCF7BDF8062DBF
:102E000002D1EBA0FCF7B8F8072D02D1EEA0FCF739
:102E1000B3F8082D02D1F4A0FCF7AEF8FF2D02D1D3
:102E2000F7A0FCF7A9F80120A6490870282E13D1B5
:102E3000617AA07A41EA0025A348A0F85D50B0F875
:102E40005D000A2190FBF1F001460190F2A0FCF731
:102E500093F801209B490870292E19D1657A0A2D13
:102E60000BDB642D09DC984981F89350084690F8F3
:102E70009310EEA0FCF780F807E02946F4A0FCF7D9
:102E80007BF80020904981F8930001208D4908705B
:102E90002A2E1FD1617AA07A41EA0025B5F57A7F02
:102EA00011DB40F6AC5085420DDC8748A0F8A650F7
:102EB000B0F8A6000A2190FBF1F001460190EAA0CB
:102EC000FCF75AF803E02946EFA0FCF755F801207B
:102ED0007C4908702B2E19D1657A012D03D17A49CE
:102EE00081F8A85003E00020774981F8A8007648CF
:102EF00090F8A800012801D1EDA000E0EEA0014665
:102F0000EFA0FCF739F801206E490870302E1CD173
:102F1000617AA07A41EA00256B48A0F86350B0F8C6
:102F200063000A2190FBF1F201FB12000190664858
:102F3000B0F8630090FBF1F000900146E7A0019A21
:102F4000FCF71AF801205F490870312E23D1617A0D
:102F5000A07A41EA002505EB85004FF6FF7101EAF2
:102F600040005949A1F88E000846B0F88E000A21A9
:102F700090FBF1F201FB120001905348B0F88E0073
:102F800090FBF1F000900146DAA0019AFBF7F4FF04
:102F900001204C490870322E0BD1657A4A48A0F8BE
:102FA0004D50B0F84D10DAA0FBF7E6FF012045497F
:102FB0000870332E0BD1657A4348A0F84F50B0F813
:102FC0004F10D9A0FBF7D8FF01203E490870342EDE
:102FD0000BD1657A3C48A0F85150B0F85110D8A0F8
:102FE000FBF7CAFF012037490870352E1BD1657ADF
:102FF000012D03D1344981F8925003E00020324979
:1030000081F89200304890F89200012802D1AFF682
:103010007C2001E0AFF67C200146CFA0FBF7ACFF9F
:10302000012028490870362E18D1112126489530E4
:10303000F5F7C3F824481D30D4F809208267D4F886
:103040000D20C267B4F81110A0F8801004F1090136
:10305000C7A0FBF791FF01201A490870372E12D143
:1030600019489530D4F80920C0F80A20B4F80D208A
:10307000C281E17B017404F10901C3A0FBF77CFF6D
:10308000012010490870502E11D1657A012D03D10D
:103090000D4981F8745103E000200B4981F8740157
:1030A000094890F87401012802D1BFA085E18BE1A5
:1030B00082E10000426174436F756E74203A2564AA
:1030C0000A0D00006002002044150020546F746156
:1030D0006C4361706163697479203A25642E2564BC
:1030E00041480A0D00000000426D734D6178566F33
:1030F0006C743A25642E2564760A0D00754261745D
:103100004D617854656D70506C75733530203A257B
:1031100064200A0D00000000754261744D696E5410
:10312000656D70506C75733530203A2564200A0D3A
:10313000000000007563426174547970653AC7A657
:10314000CBE1B5E7B3D8200A0D00000075634261FA
:1031500074547970653AC4F8C7E2B5E7B3D8200A69
:103160000D0000007563426174547970653AC1D7EF
:10317000CBE1CCFAEFAEB5E7B3D8200A0D000000E2
:103180007563426174547970653AC3CCCBE1EFAE9C
:10319000B5E7B3D8200A0D007563426174547970A5
:1031A000653AEEDCCBE1EFAEB5E7B3D8200A0D000F
:1031B0007563426174547970653AC8FDD4AAEFAE64
:1031C000B5E7B3D8200A0D00756342617454797075
:1031D000653ABEDBBACFCEEFEFAEC0EBD7D3B5E7E3
:1031E000B3D8200A0D0000007563426174547970F1
:1031F000653AEED1CBE1EFAEB5E7B3D8200A0D00CA
:103200007563426174547970653AC6E4CBFBB5E7E7
:10321000B3D8200A0D000000546F74616C566F6CB7
:10322000746167653A256420200A0D005265717546
:10323000697265566F6C746167654469666665722C
:10324000656E63652825642956200A0D000000007C
:10325000202825642956206F7665722072616E677A
:1032600065200A0D0000000053696D756C6174657E
:103270006443757272656E74426174566F6C74202B
:103280002564560A0D00000053696D756C61746504
:103290006443757272656E74426174566F6C74200B
:1032A0002564562D2D3130302D333530560A0D0022
:1032B0004F50454E00000000434C4F534500000066
:1032C00025732044656275675F506167655F667549
:1032D0006E6374696F6E200A0D00000075426174A0
:1032E0004D6178456E65726779202564202E2564CE
:1032F000200A0D0053746F70566F6C7461676520FF
:103300003A25642E2564205620200A0D0000000076
:103310004F76657254656D703056616C75653A25EF
:103320006420200A0D0000004F76657254656D70B0
:103330003156616C75653A256420200A0D00000045
:103340004F76657254656D703256616C75653A25BD
:103350006420200A0D0000005369676E616C4C6F99
:103360007373466C616720257320200A0D000000EE
:103370005665686963686C65496E666F28302D39DB
:10338000293A25730A0D00005665686963686C6503
:10339000496E666F2056494E2831302D3137293A13
:1033A00025730A0D0000000070726F666573736903
:1033B0006F6E616C00000000F4A00146F5A0FBF701
:1033C000DBFD0120F8490870512E2DD1617AA07AD9
:1033D00041EA0025302D0CDBB5F5967F09DA05EBC7
:1033E00085004FF6FF7101EA4000F049A1F8750130
:1033F00003E02946EEA0FBF7BFFDEC48B0F87501ED
:103400000A2190FBF1F201FB12000190E748B0F8AD
:10341000750190FBF1F000900146EEA0019AFBF7D8
:10342000ABFD0120E0490870522E2CD1617AA07AC0
:1034300041EA00250A2D0BDD642D09DA05EB850034
:103440004FF6FF7101EA4000D849A1F8770103E087
:103450002946E7A0FBF790FDD448B0F877010A2190
:1034600090FBF1F201FB12000190D048B0F8770117
:1034700090FBF1F000900146E7A0019AFBF77CFD7C
:103480000120C9490870532E23D1657A0A2D05DD24
:10349000962D03DAC548A0F8795103E02946E4A047
:1034A000FBF76AFDC148B0F879010A2190FBF1F2FF
:1034B00001FB12000190BD48B0F8790190FBF1F0DA
:1034C00000900146E2A0019AFBF756FD0120B649A3
:1034D0000870542E0BD1657AB44880F87B5190F86F
:1034E0007B11E1A0FBF748FD0120AF490870552E84
:1034F0000BD1657AAD4880F87C5190F87C11E0A042
:10350000FBF73AFD0120A8490870562E2CD1617AAC
:10351000A07A41EA0025302D0BDBFA2D09DA05EB04
:1035200085004FF6FF7101EA4000A049A1F87D0136
:1035300003E02946D7A0FBF71FFD9C48B0F87D01AA
:103540000A2190FBF1F201FB120001909748B0F8BC
:103550007D0190FBF1F000900146D7A0019AFBF7A6
:103560000BFD012090490870572E2CD1617AA07A6A
:1035700041EA0025142D0BDB6E2D09DA05EB8500E1
:103580004FF6FF7101EA40008849A1F87F0103E08E
:103590002946D0A0FBF7F0FC8448B0F87F010A214F
:1035A00090FBF1F201FB120001908048B0F87F011E
:1035B00090FBF1F000900146CFA0019AFBF7DCFCF4
:1035C000012079490870582E0ED1657A962D02DABD
:1035D000764981F88151754890F88111CDA0FBF7AB
:1035E000CBFC012070490870592E0ED1657A962DBA
:1035F00002DA6E4981F882516C4890F88211CBA0B2
:10360000FBF7BAFC0120684908705A2E1AD1657A76
:10361000012D03D1654981F8905103E000206349F1
:1036200081F89001614890F89001012801D1C448C7
:1036300001E0C34808300146C2A0FBF79DFC012011
:1036400059490870602E1AD1657A012D03D1574966
:1036500081F8875103E00020544981F887015348DD
:1036600090F88701012801D1B54801E0B44808303D
:103670000146BAA0FBF780FC01204B490870612E7F
:103680001AD1657A012D03D1484981F8885103E0A8
:103690000020464981F88801444890F888010128B3
:1036A00001D1A74801E0A64808300146AFA0FBF7CA
:1036B00063FC01203C490870622E25D1657A032DF8
:1036C00003DC3A4981F8895103E00020374981F849
:1036D0008901364890F88901012802D1A8A0FBF79A
:1036E0004BFC324890F88901022802D1A9A0FBF7CF
:1036F00043FC2E4890F88901032802D1AAA0FBF7C9
:103700003BFC012028490870632E24D1617AA07AFD
:1037100041EA0025254890F88901012803D129466E
:10372000A6A0FBF729FC214890F88901022803D1C3
:103730002946A8A0FBF720FC1C4890F88901032823
:1037400003D12946A9A0FBF717FC1848A0F88A5115
:10375000012015490870642E02D101201249087019
:10376000652E11D1657A012D03D1104981F88C5154
:1037700003E000200D4981F88C010C4890F88C0181
:10378000012802D16E483EE144E13BE16561737975
:1037900000000000576F726B4D6F64656C202573DD
:1037A00020200A0D000000006002002044150020C7
:1037B000444352657175697265566F6C7420256457
:1037C0003A4F7665722834382D3330302920202046
:1037D0000A0D0000444352657175697265566F6C3D
:1037E000743A25642E2564205620200A0D0000001E
:1037F00044435265717569726543757272656E7482
:103800002564413A4F7665722831302D3130304190
:10381000292020200A0D0000444352657175697209
:103820006543757272656E74256441200A0D00004F
:1038300044434D6178506F7765722564203A4F7626
:10384000657228312D31356B2909200A0D000000E1
:1038500044434D6178506F7765723A25642E256434
:10386000206B77090A0D000044435F496E6475635D
:1038700074616E636554656D70202564200A0D00C7
:1038800044435F4947425454656D70202564200AC3
:103890000D00000044434D6178566F6C7420256420
:1038A000563A4F7665722834382D323030562920FA
:1038B00020200A0D0000000044432044434D61785D
:1038C000566F6C743A25642E2564205620200A0D0C
:1038D0000000000044432044434D617843757272F8
:1038E000656E7425643A4F7665722832302D313119
:1038F00030292020200A0D0044432044434D6178A4
:1039000043757272656E743A25642E2564204120D9
:10391000200A0D0043617061636974616E636554D0
:10392000656D7031202564200A0D00004443426F0C
:103930007854656D7032202564200A0D0000000067
:1039400094250108446F75626C65426174746572F8
:10395000794D6F64652025730A0D000056494E208D
:103960005472616E732025730A0D0000426C7565F8
:103970005369676E616C4C6F737325730A0D000099
:103980004368617267654D6F64652D2D6B77680ABA
:103990000D0000004368617267654D6F64652D2DF1
:1039A00074696D650A0D00004368617267654D6F4B
:1039B00064652D2D534F430A0D000000436861726A
:1039C00067654D6F64652D6B7768282564290A0D3E
:1039D000000000004368617267654D6F64652D7477
:1039E000696D65282564290A0D000000436861722D
:1039F00067654D6F64652D534F43282564290A0D73
:103A000000000000F9480146F9A0FBF7B5FA0120D3
:103A1000FE4908706D2E1ED1657A012D06D1012058
:103A2000FB4981F89701FBA0FBF7A6FA022D06D10E
:103A30000220F74981F89701FBA0FBF79DFA032DBF
:103A400006D10320F24981F89701FCA0FBF794FA14
:103A50000120EE4908706E2E1DD1617AA07A41EAEC
:103A60000025EB48A0F89851C82D0BDDB5F53E7F39
:103A700008DA05EB85004FF6FF7101EA4000E449E2
:103A8000A1F85900E248B0F89811F1A0FBF774FAD8
:103A90000120DE4908706F2E1CD1617AA07A41EABC
:103AA0000025C82D0BDDB5F53E7F08DA05EB850056
:103AB0004FF6FF7101EA4000D549A1F85D00D448F6
:103AC000A0F89A51B0F89A11E9A0FBF755FA012035
:103AD000CE490870702E0DD1617AA07A41EA002596
:103AE000CB48A0F89C512946E9A0FBF745FA0120F4
:103AF000C6490870712E0DD1617AA07A41EA00257D
:103B0000C348A0F89E512946EBA0FBF735FA0120E7
:103B1000BE490870722E0DD1617AA07A41EA002563
:103B2000BB48A0F8A0512946E3A0FBF725FA0120E5
:103B3000B6490870732E0DD1617AA07A41EA00254A
:103B4000B348A0F8A2512946E3A0FBF715FA0120DB
:103B5000AE490870742E0DD1617AA07A41EA002531
:103B6000AB48A0F8A4512946DBA0FBF705FA0120D9
:103B7000A6490870752E0DD1617AA07A41EA002518
:103B8000A348A0F8A6512946D3A0FBF7F5F90120D8
:103B90009E490870762E0DD1617AA07A41EA0025FF
:103BA0009B48A0F8A8512946CBA0FBF7E5F90120D6
:103BB00096490870772E0DD1617AA07A41EA0025E6
:103BC0009348A0F8AA512946C3A0FBF7D5F90120D4
:103BD0008E490870782E0DD1617AA07A41EA0025CD
:103BE0008B48A0F8AC512946BBA0FBF7C5F90120D2
:103BF00086490870792E0DD1617AA07A41EA0025B4
:103C00008348A0F8AE512946B3A0FBF7B5F90120CF
:103C10007E4908707A2E0DD1617AA07A41EA00259A
:103C20007B48A0F8B0512946ABA0FBF7A5F90120CD
:103C3000764908707B2E0DD1617AA07A41EA002581
:103C40007348A0F8B2512946A3A0FBF795F90120CB
:103C50006E4908707C2E0DD1617AA07A41EA002568
:103C60006B48A0F8B45129469BA0FBF785F90120C9
:103C7000664908707D2E0DD1617AA07A41EA00254F
:103C80006348A0F8B651294693A0FBF775F90120C7
:103C90005E4908707E2E0DD1617AA07A41EA002536
:103CA0005B48A0F8B85129468BA0FBF765F90120C5
:103CB000564908707F2E0DD1617AA07A41EA00251D
:103CC0005348A0F8BA51294683A0FBF755F90120C3
:103CD0004E490870802E0DD1617AA07A41EA002504
:103CE0004B48A0F8BC51294683A0FBF745F90120B9
:103CF00046490870812E0DD1617AA07A41EA0025EB
:103D00004348A0F8BE51294681A0FBF735F90120B0
:103D10003E490870822E0DD1617AA07A41EA0025D1
:103D20003B48A0F8C051294679A0FBF725F90120AE
:103D300036490870832E0DD1617AA07A41EA0025B8
:103D40003348A0F8C251294671A0FBF715F90120AC
:103D50002E490870842E0DD1617AA07A41EA00259F
:103D60002B48A0F8C451294669A0FBF705F90120AA
:103D700026490870852E0DD1617AA07A41EA002586
:103D80002348A0F8C651294661A0FBF7F5F80120A9
:103D90001E490870862E0DD1617AA07A41EA00256D
:103DA0001B48A0F8C851294659A0FBF7E5F80120A7
:103DB00016490870872E0DD1617AA07A41EA002554
:103DC0001348A0F8CA51294651A0FBF7D5F80120A5
:103DD0000E490870882E07D1617AA07A41EA002541
:103DE0000B48A0F8CC519FE0A6E000009C250108FC
:103DF0006869676820766F6C74616765206D6F64B1
:103E0000756C652025730A0D00000000600200201B
:103E100044150020536F6353696D756C615479705C
:103E2000652D310A0D000000536F6353696D756C89
:103E300061547970652D320A0D000000536F635391
:103E4000696D756C61547970652D330A0D00000041
:103E50000A0D20536F6353696D756C614D6178561F
:103E60006F6C7420202564205620200A0D0000006D
:103E70000A0D20536F6353696D756C614D696E5601
:103E80006F6C7420202564205620200A0D0000004D
:103E90000A0D20536F6343616C6962726174696FCC
:103EA0006E566F6C74202025642028302E312956E0
:103EB00020200A0D000000000A0D20536F634361AB
:103EC0006C6962726174696F6E566F6C7420202524
:103ED00064205620200A0D00536F6343616C6962B1
:103EE000726174696F6E566F6C7420202564205661
:103EF00020200A0D00000000536F6343616C69626B
:103F0000726174696F6E2020256420200A0D000004
:103F1000536F6343616C6962726174696F6E2020D4
:103F200025642020200A0D002946AFF21C00FBF773
:103F300023F8012095490870892E0ED1617AA07A64
:103F400041EA00259248A0F8CE512946AFF2400040
:103F5000FBF712F801208D4908708A2E0ED1617A84
:103F6000A07A41EA00258A48A0F8D0512946AFF24C
:103F70006000FBF701F80120844908708B2E0ED1F8
:103F8000617AA07A41EA00258148A0F8D2512946F9
:103F9000AFF28400FAF7F0FF01207C4908708C2E04
:103FA0000ED1617AA07A41EA00257948A0F8D4516F
:103FB0002946AFF2A400FAF7DFFF01207349087029
:103FC0008D2E0ED1617AA07A41EA00257048A0F8C2
:103FD000D6512946AFF2C800FAF7CEFF01206B494F
:103FE00008708E2E0ED1617AA07A41EA00256848C9
:103FF000A0F8D8512946AFF2E800FAF7BDFF01203A
:10400000624908708F2E0ED1617AA07A41EA0025AC
:104010005F48A0F8DA512946AFF20C10FAF7ACFF6E
:1040200001205A49087078E0E079E8BB94F80880EC
:10403000414658A0FAF7A0FF5B4880F8008000785E
:104040000D2804D1002058490870584948800020A4
:104050005649488000F00EFA00273BE0B81CE11DED
:104060000E5C4FF0000930E0514810F83900B042C2
:1040700027D14F4800EBC900427831464DA0FAF7EE
:104080007BFF08F10203DFF824C1BCF802C09C44A6
:10409000464BDB1D0CEB0300454B03EBC9035A7881
:1040A000434B03EBC90300E037E05968F4F76CF8C1
:1040B0003E4840883E4901EBC901497808443B49E4
:1040C000488009F1010000F0FF09B9F1610FCBD37D
:1040D000781CC7B24745C1DB3448418808F102006B
:1040E00008443249488041F20500A1F80500E07912
:1040F000C871084680F80880002707E0B81CE11D59
:104100000A5C2A49C91D0A54781CC7B24745F5DB29
:1041100005AA06A92548F7F773F932E000BFE07950
:1041200001280DD100201A4981F8B90078211848DA
:10413000BA30F4F742F8F9F7B3FD27A0FAF71CFFFD
:104140001FE000BF2AA0FAF717FF1AE000BF28A05F
:10415000FAF712FF15E000BF25A0FAF70DFF10E0F7
:1041600000BF2AA0FAF708FF00202F49087408E0D2
:104170001FA0FAF701FF04E000BF02E000BF00E06B
:1041800000BF00BF00BFFDF7E9BF000060020020D4
:10419000441500205265616420706172616D206E6B
:1041A000756D2025640A0D00980500202A1E002048
:1041B000900200207265616420706172616D2061FF
:1041C000646472203078257820706172616D206C93
:1041D000656E2025640A0D00526563656976652069
:1041E0007265636F7264732061636B0A0D00000077
:1041F0005265636569766520444344432073746166
:1042000074652061636B0A0D0000000052656365F0
:104210006976652044454255472044434443206124
:10422000636B0A0D00000000B01F002001464888A3
:1042300008B1886808B9012070470020FCE70146F2
:1042400048880A88904201DB012070470020FCE783
:1042500010B50380002444808160828002FB031437
:10426000C460846804618468446110BD70B504460C
:104270000D46608808B1A06808B9002070BDA2880A
:1042800028466169F3F780FFA1886069084460618E
:10429000E1686069884201D3A06860616088401E5F
:1042A0006080A088EAE770B504460D4660882188E2
:1042B000884201DAA06808B9002070BDA2882946AA
:1042C0002069F3F761FFA188206908442061D4E9DF
:1042D0000310884201D3A06820616088401C608080
:1042E0000120EAE7026811BA426812BA026041602E
:1042F0007047026811BA426812BA026041607047A2
:1043000010B586B0044601210420F9F7B7F8012161
:104310004804F9F793F80420ADF8140003208DF851
:10432000160018208DF8170005A92048F7F7F2FAB3
:104330000820ADF8140048208DF8170005A91B4887
:10434000F7F7E8FA26208DF8000001208DF801002B
:104350008DF802008DF803006846F8F7DFFB019442
:104360000020ADF80800ADF80A00ADF80C00ADF87B
:1043700010000C20ADF80E0001A90D48FAF768F9FD
:10438000012240F225510A48FAF73DF9012240F294
:1043900024410748FAF737F901210548FAF7F0F800
:1043A00080210348FAF7D4F806B010BD0008014098
:1043B0000044004010B586B0044601211120F9F7F1
:1043C0005DF80121C804F9F739F84FF48060ADF8C1
:1043D000140003208DF8160018208DF8170005A989
:1043E0002248F7F797FA4FF40060ADF81400482020
:1043F0008DF8170005A91D48F7F78CFA34208DF8C1
:10440000000003208DF801008DF8020001208DF8D6
:1044100003006846F8F782FB01940020ADF808001D
:10442000ADF80A00ADF80C00ADF810000C20ADF8A6
:104430000E0001A90E48FAF70BF901210C48FAF712
:104440009FF8012240F225510948FAF7DCF80122D1
:1044500040F226610648FAF7D6F8012240F22441DC
:104460000348FAF7D0F806B010BD00000010014074
:10447000004C00403848B0F859000A2190FBF1F098
:10448000364908803448B0F85B000A2190FBF1F00F
:10449000324948803048B0F883000A2190FBF1F09F
:1044A0002E4908822C48B0F853000A2190FBF1F005
:1044B0002A4908832848B0F88E000A2190FBF1F0C1
:1044C000264988822448B0F885000A2190FBF1F043
:1044D00022494882204890F88B000A2190FBF1F095
:1044E0001E4988761C4890F88C000A2190FBF1F058
:1044F0001A49C8761848B0F890000A2190FBF1F0EC
:104500001649C8821448B0F8B1000A2190FBF1F0B6
:10451000124988831048B0F8B3000A2190FBF1F0EB
:104520000E49C8830C48B0F8B1000A2190FBF1F0A5
:104530000A498883084890F8B600323881F821008B
:10454000054890F8B500323881F82000024890F80C
:10455000790181F822007047441500209220002044
:1045600070B50546002462E004EB440000EBC40093
:10457000304901EB001090F85400032800DA54E0B1
:1045800004EB440000EBC4002A4901EB001090F852
:10459000910001280AD104EB440000EBC40001EBB8
:1045A0000010027804210120FCF760FB04EB4400BA
:1045B00000EBC4001F4901EB001090F891000228A5
:1045C00032D104EB440000EBC40001EB001090F882
:1045D000AC00401CC1B204EB440000EBC400154A1F
:1045E00002EB001080F8AC1004EB440000EBC400B8
:1045F000114601EB001090F8AC00022814DB0321F7
:1046000004EB440000EBC40002EB001080F89110B2
:1046100004EB440000EBC400114601EB00100278EB
:1046200004210120FCF722FB00BF601CC4B2022C55
:104630009ADB70BD60130020D8FF0000F8339F4361
:10464000D9FF000058699543DAFF0000BA298C436E
:10465000DBFF0000C77B8343DCFF000071BD7643B6
:10466000DDFF0000A09A6743DEFF00000080594391
:10467000DFFF0000E75B4C43E0FF0000E71B404327
:10468000E1FF00001BAF3443E2FF00005A042A435D
:10469000E3FF00008B0C2043E4FF00001DBA16432B
:1046A000E5FF000042000E43E6FF0000B6D30543DD
:1046B000E7FF00007B54FC42E8FF0000C3F5ED4239
:1046C000E9FF00005879E042EAFF000068D1D342D8
:1046D000EBFF0000E6EEC742ECFF0000AFC5BC42B6
:1046E000EDFF0000C749B242EEFF00002E70A84265
:1046F000EFFF0000B22E9F42F0FF0000C07B964209
:10470000F1FF00008A4E8E42F2FF0000AB9E86420F
:10471000F3FF00009AC87E42F4FF000007307142A8
:10472000F5FF0000FE656442F6FF0000645D58423C
:10473000F7FF0000230A4D42F8FF0000C560424227
:10474000F9FF00006D563842FAFF000048E12E42A2
:10475000FBFF0000B5F72542FCFF000000911D4261
:10476000FDFF0000DDA41542FEFF00009F2B0E425E
:10477000FFFF0000011E0742000000005A750042C2
:1047800001000000A156F441020000005474E84109
:10479000030000005238DD4104000000FC98D241C3
:1047A000050000004A8CC84106000000D509BF4141
:1047B00007000000CE08B64108000000D881AD41D6
:1047C00009000000916DA5410A00000039C59D4116
:1047D0000B000000758296410C0000008A9F8F41FB
:1047E0000D000000F01689410E00000088E38241B0
:1047F0000F00000069007A4110000000B7D16E413F
:10480000110000006132644112000000CE195A41CB
:10481000130000006F815041140000007C6147418B
:104820001500000039B43E411600000019733641EE
:1048300017000000F6972E41180000004F1E274178
:1048400019000000000020411A000000DA38194168
:104850001B00000028C412411C000000939D0C4165
:104860001D00000020C106411E000000022B014176
:104870001F00000025AFF74020000000D786ED4064
:1048800021000000A1D6E340220000009E98DA40FB
:1048900023000000E7C6D14024000000145CC9409A
:1048A000250000001153C14026000000DFA6B940DA
:1048B00027000000FC52B240280000001153AB401A
:1048C00029000000DBA2A4402A000000963E9E4082
:1048D0002B0000007D2298402C0000000A4B9240E3
:1048E0002D000000E1B48C402E000000E65C874003
:1048F0002F00000010408240300000002CB77A40AA
:10490000310000006059714032000000D061684001
:104910003300000092CB5F403400000010925740FB
:1049200035000000DEB04F4036000000E223484072
:10493000370000002EE740403800000027F73940DC
:1049400039000000DF4F33403A00000063EE2C4096
:104950003B0000006CCF26403C000000B3EF20403D
:104960003D000000984C1B403E00000054E3154001
:104970003F0000001CB1104040000000D0B30B40CD
:1049800041000000A7E8064042000000D34D02406D
:1049900043000000BEC1FB3F44000000FB3FF33F6B
:1049A000450000001B12EB3F460000002B35E33FA3
:1049B00047000000E8A4DB3F480000005F5ED43FF2
:1049C000490000004A5ECD3F4A000000B6A1C63F44
:1049D0004B0000000326C03F4C0000003EE8B93FFA
:1049E0004D00000075E5B33F4E000000041CAE3FD3
:1049F0004F000000A488A83F50000000062AA33FF3
:104A00005100000037FD9D3F520000009300993F88
:104A1000530000002332943F54000000EF8F8F3F7B
:104A20005500000001188B3F5600000008C9863F62
:104A30005700000062A1823F580000002D3E7D3FDC
:104A400059000000AE81753F5A0000004E0B6E3FCA
:104A50005B0000001FD7663F5C0000002AE35F3F59
:104A60005D000000CF2C593F5E00000018B2523F9D
:104A70005F00000065704C3F600000001765463F16
:104A800061000000DE8E403F620000001CEB3A3FF8
:104A900063000000D977353F640000006E34303F7A
:104AA00065000000931D2B3F66000000A032263FEA
:104AB000670000009F71213F6800000040D91C3F43
:104AC000690000008C67183F6A000000331B143F28
:104AD0006B000000E5F20F3F6C00000052ED0B3F51
:104AE0006D0000002D09083F6E000000CC45043F1A
:104AF0006F00000038A1003F700000009335FA3EBF
:104B0000710000006362F33E720000008FC7EC3E4C
:104B1000730000007862E63E740000007F30E03EE3
:104B200075000000A531DA3E76000000FA61D43E3F
:104B3000770000007FC1CE3E78000000944DC93E52
:104B4000790000003A06C43E7A00000082E7BE3ECB
:104B50007B0000006BF1B93E7C0000005721B53EA0
:104B60007D0000009678B03E000000003D0B01087B
:104B7000ED0B0108790A01080000000000000000A8
:104B80000000000000000000010000003D0B0108D3
:104B9000ED0B0108790A0108000000000000000088
:104BA00000000000000000004134305530350000A6
:104BB0000000000001000000D04E0108C90F0108EC
:104BC00001000000884E01082710010801000000C4
:104BD000804E01082510010801000000C44E0108A4
:104BE0002910010801000000BC4E01082F10010827
:104BF00001000000B04E01082D1001080100000066
:104C0000904E01082B100108010000009C4E010885
:104C1000CB0F010801000000AC4E01083110010863
:104C200001000000A84E0108CD0F0108010000009E
:104C3000D44E0108710F010800C1814001C08041BC
:104C400001C0804100C1814001C0804100C181405C
:104C500000C1814001C0804101C0804100C181404C
:104C600000C1814001C0804100C1814001C080413C
:104C700001C0804100C1814001C0804100C181402C
:104C800000C1814001C0804100C1814001C080411C
:104C900001C0804100C1814000C1814001C080410C
:104CA00001C0804100C1814001C0804100C18140FC
:104CB00000C1814001C0804101C0804100C18140EC
:104CC00000C1814001C0804100C1814001C08041DC
:104CD00001C0804100C1814000C1814001C08041CC
:104CE00001C0804100C1814001C0804100C18140BC
:104CF00000C1814001C0804100C1814001C08041AC
:104D000001C0804100C1814001C0804100C181409B
:104D100000C1814001C0804101C0804100C181408B
:104D200000C1814001C0804100C1814001C080417B
:104D300001C0804100C1814000C0C101C30302C263
:104D4000C60607C705C5C404CC0C0DCD0FCFCE0ECB
:104D50000ACACB0BC90908C8D81819D91BDBDA1A3B
:104D60001EDEDF1FDD1D1CDC14D4D515D71716D6AB
:104D7000D21213D311D1D010F03031F133F3F2321B
:104D800036F6F737F53534F43CFCFD3DFF3F3EFE8B
:104D9000FA3A3BFB39F9F83828E8E929EB2B2AEAFB
:104DA000EE2E2FEF2DEDEC2CE42425E527E7E6266B
:104DB00022E2E323E12120E0A06061A163A3A262DB
:104DC00066A6A767A56564A46CACAD6DAF6F6EAE4B
:104DD000AA6A6BAB69A9A86878B8B979BB7B7ABABB
:104DE000BE7E7FBF7DBDBC7CB47475B577B7B6762B
:104DF00072B2B373B17170B050909151935352929B
:104E000096565797559594549C5C5D9D5F9F9E5E0A
:104E10005A9A9B5B99595898884849894B8B8A4A7A
:104E20004E8E8F4F8D4D4C8C4484854587474686EA
:104E30008242438341818040A55A00000D0A3737E2
:104E4000375570642D2D747970653A253078202C93
:104E50007665723A2530782C54627974653A25303B
:104E6000782C204372633A2530782C5061673A25BC
:104E700030782C506C656E3A2530780D0A000000B1
:104E80004F464644434443004F4E4443444300008E
:104E900053455441504E5057440000004348495038
:104EA0004445434F444500004F46460043414E00B1
:104EB00053455441504E55534552000054455354A8
:104EC000424D5300524541444D41535300000000B0
:104ED00053455400414363757400000048414E44FB
:104EE0000000000049444C450000000053544F505E
:104EF00000000000494E4954000000005354415244
:104F0000540000006368617267655F4D6F64655FA0
:104F100031325600524541445900000052657365D4
:104F20007276656400000000526573657276617484
:104F3000696F6E5F41435F6368617267655F6D6F44
:104F40006465000044435F6368617267655F6D6F0D
:104F50006465000041435F646973636861726765FB
:104F60005F6D6F646500000044435F64697363684C
:104F7000617267655F6D6F64650000004E6F726DF2
:104F8000616C5F6D6F64650052656D6F74655F6322
:104F90006F6E74726F6C5F6D6F64650063686172D1
:104FA00067655F626174746572795F686561745F7B
:104FB0006D6F64650000000052656D6F74655F621F
:104FC0006174746572795F686561745F6D6F646543
:104FD0000000000044656661756C745F6D6F646508
:104FE0000000000041435F436861726700000000F9
:104FF0004B433130000000004B43313100000000D2
:105000004B4331004B433132000000004B43320030
:105010004B433300505752335F3300004B4334004F
:105020004B4335004B4336004B4337004B4338006E
:105030004B43390043414E325F535442000000005D
:1050400043414E5F535442004B435F41435F4F46E1
:105050004600000043414E325F454E004B435F41E6
:10506000435F4F4E000000004D43555F52554E00C8
:1050700041435F666565646261636B0044435F66DC
:105080006565646261636B004B4331426C756574A6
:105090006F6F74685F706F7765720000BC500108B5
:1050A00000000020A00B00006E8A00082C560108AA
:1050B000A00B0020F8580000D0EF00088133E8036F
:1050C00084A24A0400092C01020304060708091AF5
:1050D000FF018130089EC97F7F1EAB8252A613D587
:1050E000C01408C9BD1B08D5041AF90C1329DD1416
:1050F00008A9C11408D9BA1408B1AB026C0802435C
:1051000001180A8119010849180108A3041AB304F7
:105110001AE90441235C06A3E8031A8A0CB264DA94
:105120008B10DA8C10DA8D10DA8E10CB980560DADD
:105130009910DA9A1000091CD5FBB3B5D0ADD2E9AD
:1051400063030A08092AD9090108150A010834016C
:10515000501B0201F412025B2001085A03082305C8
:10516000101364151B2004081A54082306021A9110
:10517000081A07081AAD081A08281AAF081A0920D1
:105180001A44081A0A101ACB081A0F081AD0081A5B
:105190000E081ACF081A0D081ACE081A0C081ACDD4
:1051A000085A0B601A13481A9F101A12081A9D0801
:1051B0001A11081AC9081A10081AC7081A14082957
:1051C000281A16081AA7101A18381AF4081A1F08ED
:1051D00013A8201B201E081AAA081A1D081AD11885
:1051E0001A20081AB0101A21081AAE081A22081A32
:1051F000FB185A24601A23081AA3085A27481A26AB
:10520000081AB3281A25081AB2081A28201AA11851
:105210001A29101AD7081A2A101AEA081A2B101A73
:10522000EC085A30881A31081AA6301A32181A9126
:10523000101A33081A93081A34081A95081A3508F0
:105240001AD60823360A1AD9082337071AE3081A88
:10525000501813B8161B2051401AB9081A52081AD0
:10526000BB081A53181ABD081A54081ABF081A5551
:10527000081AC0081A56201AC1081A57081AC30873
:105280001A58181AC5081A59081AC6081A5A081AB4
:10529000D4081A60081ACB081A61081ACC081A62D6
:1052A000081ACD081A63381ACE081A65101AD008E1
:1052B0001A66081AD1081A6D081ADB081A6E201A25
:1052C000DC081A6F081ADE081A70081AE0081A714A
:1052D000081AE2081A72081AE4081A73081AE6088B
:1052E0001A74081AE8081A75081AEA081A76081AC9
:1052F000EC081A77081AEE081A78081AF0081A79D2
:10530000081AF2081A7A081AF4081A7B081AF6081A
:105310001A7C081AF8081A7D081AFA081A7E081A60
:10532000FC081A7F081AFE081A80081112171B20A1
:1053300081081A02081A82081A04081A83081A0631
:10534000081A84081A08081A85081A0A081A86080A
:105350001A0C081A87081A0E081A88081A10081A50
:1053600089081A12081A8A081A14081A8B081A16B9
:10537000081A8C081A18081A8D081A1A081A8E08A2
:105380001A1C081A8F081A1E0801261AFF01011A92
:10539000036FE8032D01020304043009060708091E
:1053A00002040608137DFB2408040113C1CB1B086B
:1053B00009081AFD081A57981325CC1B0858081A13
:1053C00051081A59081A7D081A5D081ABD081A5F93
:1053D000081AE108239B051305CD1B08E6101A29BE
:1053E000081AE7081A95081A80181AD5081A1150D1
:1053F0001341D11408A1CA296B91CFC91501088D99
:10540000AE14411AD118136DAF1B082D049AFD205C
:105410001A3318DA9514411AD9181AB918DB51B091
:10542000301D160108E5181AB5141ACD045A153C9A
:105430001A25181AFD0C1A39309AE5301E31170159
:1054400008151401101A2B601A513001101ACF18C8
:105450001AD7041A39042AE10819581A2B041A39E0
:10546000481A31101E4112010855041EB5110108D9
:10547000C1081ED913010871041EF1140108751426
:1054800081139DDA1408B1BD1B08C10813E1C01BCC
:105490000871081A91101A81081A9708016813D820
:1054A000071F20E44E0108F4041ADC041E144F0107
:1054B00008FC081E6C500108EC081AE4101AD40409
:1054C0001A7C041A34041A54041A44041A68041A7C
:1054D00028041A04041A88041A9C041AB8041A1C12
:1054E00004011013ADC91B0855041A850442204459
:1054F00010014042014A0C0C9A020C9A040C11292A
:1055000006590C42104A080C3948590C3905590CF7
:10551000393C5A143C2931596C3919594839A16917
:10552000602918593C3985690C4A803C3998291200
:10553000690C2905A990190C39C829051924390CB9
:10554000292469782911A9B4593C13A5C81408C89D
:10555000081B20D4041BDC091B6C500108141AE042
:10556000041AF0149A0C141AEC0413040A9B201069
:10557000141AF8041A18149A1C141A04381A2C1441
:105580009A20141A10141A40149A24141A1C141A6B
:1055900054149A28141A28141A68149A2C141A34B9
:1055A000141A7C149A30141A40141A90148BF04F69
:1055B000141A4C141AA4149AF8141A58141AB81479
:1055C0001A043C4BCDC7141A64141ACC141A88144C
:1055D0004B09C9141A70141AE0141A68145ADB140F
:1055E0001A7C141AF4149A70141A88141B080B1CD1
:1055F000998C1A94141A1C149A14141AA0141A30A0
:10560000149A34141AAC141A44149A54141AB81470
:105610001A58149A5C141AC4141A6C149A48141A5E
:0C562000D0141A80141A4014C1000000BD
:04000005080081511D
:00000001FF
